:020000040001F9
:200000000000022075030100B5030100B7030100B9030100BD030100C1030100000000008E
:20002000000000000000000000000000C5030100C703010000000000CB03010017820100C3
:20004000CF030100D3030100D7030100DB030100DF030100E3030100E7030100EB03010098
:20006000EF030100F3030100F7030100FB030100FF03010003040100070401000B04010075
:200080000F04010013040100170401001B0401001F04010023040100270401002B04010050
:2000A0002F04010033040100370401003B0401003F04010043040100B103010047040100CB
:2000C0004B0401004F0401005304010057040100B10301005B0401005F04010063040100E7
:2000E000670401006B040100B10301006F04010073040100770401007B0401007F04010003
:20010000B103010083040100870401008B0401008F04010093040100970401009B0401001E
:200120009F040100A3040100A7040100AB040100AF040100B3040100B7040100BB0401002F
:20014000BF040100C3040100C7040100CB040100CF040100D3040100D7040100DB0401000F
:20016000DF040100E3040100E7040100EB040100EF040100F3040100F7040100FB040100EF
:20018000FF04010003050100070501000B0501000F05010013050100170501001B050100C8
:2001A0001F05010023050100270501002B0501002F05010033050100370501003B050100A7
:2001C0003F05010043050100470501004B0501004F05010053050100570501005B05010087
:2001E0005F05010063050100670501006B0501006F05010073050100770501007B05010067
:200200007F05010083050100870501008B0501008F05010093050100970501009B05010046
:200220009F050100A3050100A7050100AB050100AF050100B3050100B7050100BB05010026
:20024000BF050100C3050100C7050100CB050100CF050100D3050100D7050100DB05010006
:20026000DF050100E3050100E7050100EB050100EF050100F3050100F7050100FB050100E6
:20028000FF05010003060100070601000B0601000F0601001306010017060100B10301002C
:2002A000B1030100B10301001B0601001F06010023060100270601002B0601002F060100CC
:2002C00033060100370601003B0601003F06010043060100470601004B0601004F060100DE
:2002E00053060100570601005B0601005F06010063060100670601006B0601006F060100BE
:2003000073060100770601007B0601007F06010083060100870601008B0601008F0601009D
:2003200093060100970601009B0601009F060100A3060100A7060100AB060100AF0601007D
:20034000B3060100B7060100BB060100BF060100C3060100C7060100CB060100CF0601005D
:20036000D3060100D7060100DB060100DF060100E306010072B6DC48DC4901600A6882F35A
:200380000888DB488047DB49DB4ADC4B9A4204D00431043208681060F8E7D949D94A002034
:2003A000914202D004310860FAE762B6D6480047FFF7FEBFFEE7FEE7FFF7FEBFFFF7FEBFBA
:2003C000FFF7FEBFFEE7FFF7FEBFFEE70000CF480047CF480047CF480047CF480047CF485E
:2003E0000047CF480047CF480047CF480047CF480047CF480047CF480047CF480047CF480D
:200400000047CF480047CF480047CF480047CF480047CF480047CF480047CF480047CF48EC
:200420000047CF480047CF480047CF480047CF480047CF480047CF480047CF480047CF48CC
:200440000047CF480047CF480047CF480047CF480047CF480047CF480047CF480047CF48AC
:200460000047CF480047CF480047CF480047CF480047CF480047CF480047CF480047CF488C
:200480000047CF480047CF480047CF480047CF480047CF480047CF480047CF480047CF486C
:2004A0000047CF480047CF480047CF480047CF480047CF480047CF480047CF480047CF484C
:2004C0000047CF480047CF480047CF480047CF480047CF480047CF480047CF480047CF482C
:2004E0000047CF480047CF480047CF480047CF480047CF480047CF480047CF480047CF480C
:200500000047CF480047CF480047CF480047CF480047CF480047CF480047CF480047CF48EB
:200520000047CF480047CF480047CF480047CF480047CF480047CF480047CF480047CF48CB
:200540000047CF480047CF480047CF480047CF480047CF480047CF480047CF480047CF48AB
:200560000047CF480047CF480047CF480047CF480047CF480047CF480047CF480047CF488B
:200580000047CF480047CF480047CF480047CF480047CF480047CF480047CF480047CF486B
:2005A0000047CF480047CF480047CF480047CF480047CF480047CF480047CF480047CF484B
:2005C0000047CF480047CF480047CF480047CF480047CF480047CF480047CF480047CF482B
:2005E0000047CF480047CF480047CF480047CF480047CF480047CF480047CF480047CF480B
:200600000047CF480047CF480047CF480047CF480047CF480047CF480047CF480047CF48EA
:200620000047CF480047CF480047CF480047CF480047CF480047CF480047CF480047CF48CA
:200640000047CF480047CF480047CF480047CF480047CF480047CF480047CF480047CF48AA
:200660000047CF480047CF480047CF480047CF480047CF480047CF480047CF480047CF488A
:200680000047CF480047CF480047CF480047CF480047CF480047CF480047CF480047CF486A
:2006A0000047CF480047CF480047CF480047CF480047CF480047CF480047CF480047CF484A
:2006C0000047CF480047CF480047CF480047CF480047CF480047CF480047CF480047CF482A
:2006E0000047CF48004700BF08ED00E0000001009D900100D8F4010090090020AC0F002031
:20070000AC0F00202C640020B7850100E94F0100FD4F010011500100255001003950010029
:200720004D5001006150010075500100895001009D500100B1500100C5500100D950010099
:20074000ED500100015101001551010029510100B1030100B103010095640100817F0100C1
:200760008F510100E97001007158010081580100176E0100276E0100376E0100576E010012
:20078000476E0100676E0100776E0100876E0100A76E0100976E0100B76E0100C76E010079
:2007A000D76E0100F76E0100E76E0100076F0100176F0100276F0100476F0100376F010044
:2007C000B1030100B1030100B1030100B1030100B1030100B1030100E9330100FD3301008D
:2007E0001134010025340100393401004D3401006134010075340100893401009D34010099
:20080000B1340100C5340100D9340100ED3401000135010015350100293501003D35010074
:200820005135010065350100793501008D350100A1350100B5350100C9350100DD35010050
:20084000F135010005360100193601002D3601004136010055360100693601007D36010029
:2008600091360100A5360100B9360100CD360100E1360100F5360100093701001D37010006
:200880003137010045370100593701006D3701008137010095370100A9370100BD370100E0
:2008A000D1370100E5370100F93701000D3801002138010035380100493801005D380100BB
:2008C000713801008538010099380100AD380100C1380100D5380100E9380100FD38010098
:2008E0001139010025390100393901004D3901006139010075390100893901009D39010070
:20090000B1390100C5390100D9390100ED390100013A0100153A0100293A01003D3A01004B
:20092000513A0100653A0100793A01008D3A0100A13A0100B53A0100C93A0100DD3A010027
:20094000F13A0100053B0100193B01002D3B0100413B0100553B0100B57C0100C57C0100EA
:20096000D57C0100E57C0100F57C0100057D0100157D0100257D0100357D0100457D010022
:20098000557D0100657D0100757D0100857D0100957D0100A57D0100F3790100037A01008A
:2009A000137A0100237A0100B15A0100C15A010061520100715201008152010091520100B3
:2009C000A15201004D7401008768010093680100B1030100CD7D0100BD4B0100D14B01004F
:2009E000E54B0100936B01009F6B0100693B01007D6001008D6001009D600100AD6001003F
:200A0000BD600100CD600100DD600100ED600100B1030100B1030100D5490100CD6A01003D
:200A2000D96A010010B402464FEA82024EF6A433C0F201031A44126801F01F034FF00104A9
:200A400004FA03F34FF00004202901D213631BE0402901D2D36217E0602908D2062801D008
:200A6000072801D153670FE04FF001040CE0802908D2062801D0072801D1136704E04FF07C
:200A8000010401E04FF00104204610BC704700004DF8048D4FF00001082801D8014621E0DC
:200AA0000F281FD80FF20408D8E800F01C1C1C1C1C1C1C1C1C080B0E1114171A4FF00C018C
:200AC00010E04FF010010DE04FF014010AE04FF0180107E04FF0200104E04FF0300101E0D7
:200AE0004FF0400108465DF8048B7047A1B39AB3082801D803462DE00C2804D84FF0090035
:200B00004FF00C0326E0102804D84FF00A004FF010031FE0142804D84FF00B004FF014031B
:200B200018E0182804D84FF00C004FF0180311E0202804D84FF00D004FF020030AE03028F7
:200B400004D84FF00E004FF0300303E04FF00F004FF0400308601360704710B402464FEA70
:200B600082024EF6C433C0F201031A4413684FF000021C6804F07F04A14208D8062802D226
:200B80004FF0400401E04FF08004A14201D34FF00102B2B9186810F0005F12D05B6B4FEA0A
:200BA00003134FEA137303F1010003464FEAC30318464FEA900000F10500814201D84FF02B
:200BC0000102104610BC704710B401464FEA810108464EF6C431C0F20101084401684FF044
:200BE00000024FF001030C6844F080440C600C6844F080540C60086810F0004F0AD00C68E3
:200C00006FF3DF740C6005E002F10102086810F0006F05D144F64030C0F24C008242F3D3F1
:200C200044F64030C0F24C00824202D34FF0010311E04FF0000208E002F10102086810F0B0
:200C4000807F02D04FF0000305E044F64030C0F24C008242F0D3184610BC704710B4014681
:200C60004FEA810108464EF6C431C0F20101084401684FF000024FF001040B686FF31C73E0
:200C80000B600B686FF39E730B6008E002F10102086810F0807F02D14FF0000403E042F21E
:200CA00010708242F2D3204610BC704702464FEA820210464EF6C432C0F20102104402683A
:200CC000106810F4006F38D061B9D2F8002C4FEA82324FEA927202F103004FF0010101FAB5
:200CE00000F22CE001290CD1D2F8002C4FEAC2224FEA927202F103004FF0010101FA00F27B
:200D00001DE002290CD1D2F8002C4FEA02224FEA927202F103004FF0010101FA00F20EE02C
:200D2000D2F8002C4FEA42124FEA927202F103004FF0010101FA00F201E04FF00802D0B223
:200D40007047F0B581B005464FF008064FF4007728464FF00001FFF7A9FF3044B7FBF0F45E
:200D600028464FF00101FFF7A1FF3044B7FBF0F00444062D01D0072D11D128464FF0020116
:200D8000FFF794FF3044B7FBF0F0044428464FF00301FFF78BFF3044B7FBF0F00444E0B26B
:200DA00001B0F0BD2DE9F04F85B004460D461646039320464FEA80004EF6C431C0F20101B0
:200DC0000844D0F80080CDF808804FF008098DF802904FF40079CDF804904FF0000A4FF02E
:200DE00000004FF0000B16B14FF000013170062C2CBF032101218DF803104FF0000726E0BA
:200E0000C0B2A5EB0000C5B2F8B201462046FFF74DFF9DF8028008EB0001DDF80480B8FBA9
:200E2000F1F00EB1FAB2327085420CD201FB05F05044DDF8088008F180010844DDF80C8016
:200E4000C8F8000007E00AF5007A07F101079DF803804745D4D9062C02D24FF4806001E017
:200E60004FF40060824501D34FF0010B584605B0BDE8F08F2DE9F04F87B004468DF8071000
:200E800015469B46DDF840A020464FEA80004EF6C432C0F20102104407684FF0000604AB9C
:200EA0000DF106029DF807102046FFF77BFF012802D14FF0010628E16878402802D94FF0FD
:200EC000010622E1049800F10809CDF814909DF807102046FFF741FE012802D14FF0010678
:200EE00013E1386810F4006F08D06879012805D1D7F8000C40F00040C7F8000C9DF8061072
:200F00002046FFF7D3FE6A78824202D94FF00106FBE003AA02A96878FFF7E8FDBAF1000F35
:200F20006ED068784FEAA000C0B202464FF0000030E0049C03464FEA830304F108042344A1
:200F400004464FEA8404544424784FEA046407464FEA870707F1010757443F784FEA0747C4
:200F600047EA040407464FEA870707F1020757443F784FEA072747EA040407464FEA87071D
:200F800007F1030757443F7847EA04041C6000F10100C0B29042CCD310464FEA8000C0B2F2
:200FA00013E020F0030200F00303C3F103031A4402F03F02D2B2DDF81480424400EB0A037D
:200FC0001B78137000F10100C0B26A789042E8D3687811E020F0030200F00303C3F1030392
:200FE0001A4402F03F02D2B2DDF8148042442B79137000F10100C0B29DF80C209042E9D313
:2010000004984FF00002026004984FF000024260049B029A18686FF3134002F00F024FEA66
:20102000024240EA02001860287801281BD104982BF060424260049B58686FF35F709DF8F3
:20104000488008F007024FEA427240EA02005860049A106840F400101060049A10686FF3B4
:201060009650106023E0049B58686FF39C4040F2FF720BEA02024FEA824240EA02005860FD
:20108000049B58686FF35F709DF8488008F007024FEA427240EA02005860049A10686FF319
:2010A00055501060049A10686FF396501060A878012804D1049A106840F480101060049A47
:2010C00010686FF31B601060E878012804D1049A106840F000401060049B6A7918686FF393
:2010E0009E7002F001024FEA827240EA02001860049B18686FF31B60DDF8448008F00F027E
:201100004FEA026240EA02001860304607B0BDE8F08F2DE9F04C83B004460E4617469A46DD
:20112000DDF828B04FF0000501AB0DF1030231462046FFF737FE012802D14FF0010546E0A0
:2011400031462046FFF709FD012802D14FF001053DE001984FF00001016001984FF0000145
:201160004160012F0ED101982AF0604141600199086840F400100860019908686FF39650C2
:20118000086016E0019A50686FF39C4040F2FF710AEA01014FEA814140EA01005060019958
:2011A00008686FF355500860019908686FF396500860BBF10F0F0AD0019A10686FF31B6002
:2011C0000BF00F014FEA016140EA01001060284603B0BDE8F08CF0B401464FEA81014EF6A2
:2011E000C432C0F2010211440C6801464FEA81014EF6A432C0F2010211440B6803F180026C
:20120000062804D24FF480774FF0400503E04FF400774FF08005616B41F0805161634FF0DA
:20122000000109E00E464FEA860616444FF0000CC6F800C001F10101B942F3D303F5086271
:201240004FF0000108E00E464FEA860616444FF0FF37376001F10101A942F4D34FF0FF31D2
:2012600019614FF0FF3159614FF0FF3199614FF0FF31996401464FEA81014EF6C432C0F208
:2012800001021144096801F528624FF0000108E00B464FEA830313444FF000051D6001F1C3
:2012A00001010629F4D301464FEA81014EF6C432C0F201021144096801F52A624FF00001BD
:2012C00008E00B464FEA830313444FF0FF351D6001F101010429F4D301464FEA81014EF6A1
:2012E000C432C0F201021144096801F52B624FF0000108E00B464FEA830313444FF0000527
:201300001D6001F101010C29F4D34FEA80004EF6C431C0F201010844006840F6287100EB4C
:2013200001024FF0000108E008464FEA800010444FF00003036001F101013629F4D3606B9D
:201340006FF31C706063F0BC704730B585B0044620464FEA80004EF6A431C0F201010844DD
:2013600001680D6A20464FEA800040F6CC72C2F200021044006840F20402C0F2080200EAAA
:20138000020005EA00050D6205F0040048B34FF04C0014FB00F040F6EC71C2F200010844D6
:2013A000006958B14FF04C0014FB00F040F6EC71C2F2000108440069804712E04FF000003C
:2013C00002904FF0000001904FF00000009020464FF000034FF001024FF0000101F0ABFC1A
:2013E000002805F4002088B34FF04C0014FB00F040F6EC71C2F20001084400F1100000F161
:201400001000006878B14FF04C0014FB00F040F6EC71C2F20001084400F1100000F110000B
:201420000068804712E04FF0000002904FF0000001904FF00000009020464FF000034FF034
:2014400001024FF0040101F076FC002805B030BD00B585B001464FEA81014EF6A432C0F260
:201460000102114409684FF400320A624FF04C0110FB01F140F6EC72C2F20002114401F1A8
:20148000100101F10801096879B14FF04C0110FB01F040F6EC71C2F20001084400F1100088
:2014A00000F108000068804711E04FF0000102914FF0000101914FF0000100914FF000035B
:2014C0004FF001024FF0020101F035FC002805B000BD00B585B001464FEA81014EF6A432C6
:2014E000C0F20102114409684FF480320A624FF04C0110FB01F140F6EC72C2F200021144E8
:2015000001F1100101F10C01096879B14FF04C0110FB01F040F6EC71C2F20001084400F121
:20152000100000F10C000068804711E04FF0000102914FF0000101914FF0000100914FF0C9
:2015400000034FF001024FF0030101F0F4FB002805B000BD10B584B0044620464FEA800027
:201560004EF6A431C0F201010844016820464FEA800040F6AC72C2F2000210440A6A026096
:201580004FF0020008624FF04C0014FB00F040F6EC71C2F20001084400F1100000F104008C
:2015A000006878B14FF04C0014FB00F040F6EC71C2F20001084400F1100000F1040000681E
:2015C000804712E04FF0000002904FF0000001904FF00000009020464FF000034FF00102F8
:2015E0004FF0010101F0A7FB002820464FEA800040F6AC71C2F2000108444FF000010160DB
:2016000004B010BD10B584B0044620464FEA80004EF6A431C0F201010844016820464FEAC6
:20162000800040F6AC72C2F2000210440A6A02604FF4801008624FF04C0014FB00F040F6F9
:20164000EC71C2F20001084400F1100000F11400006878B14FF04C0014FB00F040F6EC7178
:20166000C2F20001084400F1100000F114000068804712E04FF0000002904FF000000190A1
:201680004FF00000009020464FF000034FF001024FF0050101F04FFB002820464FEA8000CA
:2016A00040F6AC71C2F2000108444FF00001016004B010BD30B585B0044620464FEA800031
:2016C0004EF6A431C0F2010108440068D0F8085BD0F8001B01F4403105EA0105C0F8085B05
:2016E00005F4803088B34FF04C0014FB00F040F6EC71C2F20001084400F1100000F13400C2
:20170000006878B14FF04C0014FB00F040F6EC71C2F20001084400F1100000F1340000688C
:20172000804712E04FF0000002904FF0000001904FF00000009020464FF000034FF0010296
:201740004FF00D0101F0F7FA002805F4003088B34FF04C0014FB00F040F6EC71C2F20001FC
:20176000084400F1100000F13800006878B14FF04C0014FB00F040F6EC71C2F20001084444
:2017800000F1100000F138000068804712E04FF0000002904FF0000001904FF0000000908E
:2017A00020464FF000034FF001024FF00E0101F0C2FA002805B030BD00B585B001464FEA10
:2017C00081014EF6A432C0F20102114409684FF001020A624FF04C0110FB01F140F6EC7227
:2017E000C2F20002114401F1100101F11801096879B14FF04C0110FB01F040F6EC71C2F266
:201800000001084400F1100000F118000068804711E04FF0000102914FF0000101914FF06D
:20182000000100914FF000034FF001024FF0060101F081FA002805B000BD30B585B00446E2
:2018400020464FEA80004EF6A431C0F2010108440068D0F8FC5AD0F8E01A01F4502105EAB3
:201860000105C0F8FC5A05F4002088B34FF04C0014FB00F040F6EC71C2F20001084400F1F1
:20188000100000F12800006878B14FF04C0014FB00F040F6EC71C2F20001084400F110006F
:2018A00000F128000068804712E04FF0000002904FF0000001904FF00000009020464FF0D9
:2018C00000034FF001024FF00A0101F034FA002805F4802088B34FF04C0014FB00F040F69E
:2018E000EC71C2F20001084400F1100000F12C00006878B14FF04C0014FB00F040F6EC71BE
:20190000C2F20001084400F1100000F12C000068804712E04FF0000002904FF000000190E6
:201920004FF00000009020464FF000034FF001024FF00B0101F0FFF9002805F4803088B3AE
:201940004FF04C0014FB00F040F6EC71C2F20001084400F1100000F13000006878B14FF077
:201960004C0014FB00F040F6EC71C2F20001084400F1100000F130000068804712E04FF006
:20198000000002904FF0000001904FF00000009020464FF000034FF001024FF00C0101F0EF
:2019A000CAF9002805B030BD2DE9F04C81B0064630464FEA80004EF6C431C0F20101084463
:2019C000D0F800A030464FEA80004EF6A431C0F2010108440468DAF8000000F07F0000F1B9
:2019E0000100276BA16A07EA0107C7F30F07102888BF102083464FF00005ACE04FF00100F8
:201A000000FA05F000EA0700002800F0A280DAF8000010F0005F77D0072D75D8052D24D18C
:201A20004FF04C0016FB00F040F6EC71C2F20001084400F1100000F11C00006878B14FF0A8
:201A40004C0016FB00F040F6EC71C2F20001084400F1100000F11C000068804705E0A06A79
:201A60006FF0200100EA0100A062062D24D14FF04C0016FB00F040F6EC71C2F200010844B1
:201A800000F1100000F12000006878B14FF04C0016FB00F040F6EC71C2F20001084400F192
:201AA000100000F120000068804705E0A06A6FF0400100EA0100A062072D45D14FF04C0085
:201AC00016FB00F040F6EC71C2F20001084400F1100000F12400006878B14FF04C0016FB2E
:201AE00000F040F6EC71C2F20001084400F1100000F124000068804726E0A06A6FF080012D
:201B000000EA0100A0621FE04FF04C0016FB00F040F6EC71C2F200010844006860B14FF001
:201B20004C0016FB00F040F6EC71C2F20001084401682846884707E04FF0010000FA05F107
:201B4000A06A20EA0100A0624FF0010000FA05F0206305F101055D45FFF450AF01B0BDE8D6
:201B6000F08C2DE9F044074638464FEA80004EF6C431C0F201010844016838464FEA800042
:201B80004EF6A432C0F2010210440568086800F07F0000F101002E6BA96A06EA01066FF3DF
:201BA0000F06202888BF202082464FF0100431E04FF0010000FA04F000EA060018B34FF0ED
:201BC0004C0017FB00F040F6EC71C2F20001084400F10400006870B14FF04C0017FB00F018
:201BE00040F6EC71C2F20001084400F1040001682046884707E04FF0010000FA04F1A86A96
:201C000020EA0100A8624FF0010000FA04F0286304F101045445CBD3BDE8F0842DE9F04462
:201C2000074638464FEA80004EF6C431C0F201010844016838464FEA80004EF6A432C0F27B
:201C4000010210440568086800F07F0000F10100EE6A696A06EA0106C6F30F06302888BF60
:201C6000302082464FF0200438E0A4F120004FF0010101FA00F000EA060028B34FF04C009A
:201C800017FB00F040F6EC71C2F20001084400F10800006870B14FF04C0017FB00F040F669
:201CA000EC71C2F20001084400F1080001682046884709E0A4F120004FF0010101FA00F164
:201CC000686A20EA01006862A4F120004FF0010101FA00F0E86204F10100C4B25445C4D396
:201CE000BDE8F0842DE9F044074638464FEA80004EF6C431C0F201010844016838464FEAA4
:201D000080004EF6A432C0F2010210440568086800F07F0000F10100EE6A696A06EA0106C0
:201D20006FF30F06402888BF402082464FF0300437E0A4F120004FF0010101FA00F000EA00
:201D4000060028B34FF04C0017FB00F040F6EC71C2F20001084400F10C00006870B14FF0BC
:201D60004C0017FB00F040F6EC71C2F20001084400F10C0001682046884709E0A4F1200048
:201D80004FF0010101FA00F1686A20EA01006862A4F120004FF0010101FA00F0E86204F14F
:201DA00001045445C5D3BDE8F0842DE9F04C81B0064630464FEA80004EF6C431C0F20101E9
:201DC0000844D0F800A030464FEA80004EF6A431C0F2010108440468DAF8000000F07F005A
:201DE00000F10100276BA16A07EA0107202888BF202083464FF00005AEE04FF0010000FAB7
:201E000005F000EA0700002800F0A480DAF8000010F0005F79D0072D77D8052D25D14FF03C
:201E20004C0016FB00F040F6EC71C2F20001084400F1100000F11C00006878B14FF04C0097
:201E400016FB00F040F6EC71C2F20001084400F1100000F11C000068804776E0A06A6FF0F1
:201E6000200100EA0100A0626FE0062D25D14FF04C0016FB00F040F6EC71C2F200010844BC
:201E800000F1100000F12000006878B14FF04C0016FB00F040F6EC71C2F20001084400F18E
:201EA000100000F12000006880474EE0A06A6FF0400100EA0100A06247E0072D45D14FF05D
:201EC0004C0016FB00F040F6EC71C2F20001084400F1100000F12400006878B14FF04C00EF
:201EE00016FB00F040F6EC71C2F20001084400F1100000F124000068804726E0A06A6FF099
:201F0000800100EA0100A0621FE04FF04C0016FB00F040F6EC71C2F200010844006860B1BB
:201F20004FF04C0016FB00F040F6EC71C2F20001084401682846884707E04FF0010000FABA
:201F400005F1A06A20EA0100A0624FF0010000FA05F0206305F101055D45FFF44EAF01B083
:201F6000BDE8F08C2DE9F044064630464FEA80004EF6C431C0F201010844016830464FEA2A
:201F800080004EF6A432C0F2010210440568086800F07F0000F10100EF6A696A07EA01073B
:201FA000402888BF402082464FF0200437E0A4F120004FF0010101FA00F000EA070028B323
:201FC0004FF04C0016FB00F040F6EC71C2F20001084400F10400006870B14FF04C0016FBC7
:201FE00000F040F6EC71C2F20001084400F1040001682046884709E0A4F120004FF00101EB
:2020000001FA00F1686A20EA01006862A4F120004FF0010101FA00F0E86204F1010454456F
:20202000C5D3BDE8F0842DE9F044064630464FEA80004EF6C431C0F2010108440168304612
:202040004FEA80004EF6A432C0F2010210440568086800F07F0000F101006F6FE96E07EA40
:202060000107602888BF602082464FF0400438E0A4F140004FF0010101FA00F000EA0700B4
:2020800028B34FF04C0016FB00F040F6EC71C2F20001084400F10800006870B14FF04C0038
:2020A00016FB00F040F6EC71C2F20001084400F1080001682046884709E0A4F140004FF0F7
:2020C000010101FA00F1E86E20EA0100E866A4F140004FF0010101FA00F0686704F101009D
:2020E000C4B25445C4D3BDE8F0842DE9F044064630464FEA80004EF6C431C0F20101084423
:20210000016830464FEA80004EF6A432C0F2010210440568086800F07F0000F101002F6F28
:20212000A96E07EA0107802828BF802082464FF0600437E0A4F160004FF0010101FA00F0BD
:2021400000EA070028B34FF04C0016FB00F040F6EC71C2F20001084400F10C00006870B10D
:202160004FF04C0016FB00F040F6EC71C2F20001084400F10C0001682046884709E0A4F126
:2021800060004FF0010101FA00F1A86E20EA0100A866A4F160004FF0010101FA00F02867D3
:2021A00004F101045445C5D3BDE8F0842DE9F04405460E4628464FEA80004EF6C431C0F2E0
:2021C00001010844046828464FEA80004EF6A431C0F201010844D0F800A04FF000072068CF
:2021E00010F0004F0CD12846FEF7EEFC10B14FF0010705E0284600F062FA08B14FF00107BF
:2022000027BB284600F030FA10B14FF001071DE02846FEF7D9FC10B14FF0010716E0206891
:2022200040F0007020604FF0000005E000F10100216811F0007F03D042F210718842F5D345
:2022400042F21071884201D34FF00107002F40F0C180206840F4805020602846FEF7BBFF1B
:202260004FF00000CAF828004FF00000CAF82400062D01D0072D07D14FF00000CAF86C0093
:202280004FF00000CAF868004FF0FF30CAF830004FF0FF30CAF82C00062D01D0072D07D109
:2022A0004FF0FF30CAF874004FF0FF30CAF8700040F20700C0F21B00CAF820004FF450203F
:2022C000CAF8FC0A4FF44030CAF8080B317F20686FF3CB2001F001014FEAC12140EA0100F0
:2022E0002060206840F480302060317F206D6FF3DF7001F001014FEAC17140EA0100206576
:20230000D4F8000C6FF3CF30C4F8000C317F606B6FF30C3001F001014FEA013140EA01001A
:202320006063307F01284CD1717FD4F8000C6FF3114001F003014FEA014140EA0100C4F813
:20234000000CB17FD4F8000C6FF3D44001F003014FEAC14140EA0100C4F8000C062D01D0CC
:20236000072D1AD1F17FD4F8000C6FF3975001F003014FEA815140EA0100C4F8000C96F82C
:202380002010D4F8000C6FF35A6001F003014FEA416140EA0100C4F8000C06F108012846E8
:2023A00000F02BFA012802D14FF0010712E006F12401284600F096FA01280BD14FF001077D
:2023C00008E006F10801284600F0A4F9012801D14FF00107002F54D12846FEF7B2FC3168DA
:2023E000814209D8062D02D24FF0400001E04FF080003168814202D94FF0010741E03068DC
:20240000A0F1010120686FF3060001F07F0140EA01002060F079022803D0206840F40030CB
:2024200020603079012823D1307FF0B9206840F0005020607179606B6FF31B6001F00F01E3
:202440004FEA016140EA01006063B17920686FF3CF3001F001014FEAC13140EA0100206017
:202460004FF0FF30CAF848000BE04FF0010708E020686FF35D702060B079012801D14FF030
:202480000107002F50D1206840F480202060F179284600F084F810B14FF0010744E0F0792F
:2024A000032824D02846FEF7D9FB10B14FF001073AE028464FEA80004EF6C431C0F2010190
:2024C00008440068416B41F000514163D0F8E01A6FF3DF71C0F8E01AD0F8E01A6FF3C71154
:2024E000C0F8E01A416B6FF35D7141631CE028464FEA80004EF6C431C0F2010108440068E6
:20250000416B41F000514163D0F8E01A6FF3DF71C0F8E01AD0F8E01A6FF3C711C0F8E01A15
:20252000416B6FF35D7141633846BDE8F08470B584B0054628464FEA80004EF6C431C0F2CE
:202540000101084406684FF000044FF0000002904FF0000001904FF00000009028464FF05F
:2025600000034FF001024FF0100100F0E4FB10B14FF0010410E0306810F0004F0CD12846D0
:20258000FEF722FB10B14FF0010405E0284600F096F808B14FF00104204604B070BD2DE9F9
:2025A000F04581B007468A4638464FEA80004EF6C431C0F201010844046825684FEAC5151C
:2025C0004FEAD5754FF000062DB93846FEF7FCFA08B14FF00106BEBB5046042834D80FF29D
:2025E0000808D8E800F000BF04111A312D0060686FF3C300606060686FF30C306060206874
:202600006FF3D75020601FE0606840F00800606060686FF30C30606016E060686FF3C300E9
:202620006060606840F48050606020686FF351402060D4F8000C6FF3CF30C4F8000C03E06F
:20264000206840F0004020604EB9BAF1030F06D02DB93846FEF702FB08B14FF0010630469D
:2026600001B0BDE8F085000010B401464FEA810108464EF6C431C0F20101084401684FF09A
:2026800000024FF00004086810F4801F14D00B686FF3DF730B6005E002F10102086810F41D
:2026A000801F03D042F210708242F5D342F21070824201D34FF00104204610BC704710B42B
:2026C00001464FEA810108464EF6C431C0F20101084401684FF000024FF00004086810F014
:2026E000004F14D10B6843F000430B6005E002F10102086810F4801F03D142F21070824218
:20270000F5D342F21070824201D34FF00104204610BC70472DE9F04482460D4650464FEA44
:2027200080004EF6C431C0F201010844046826684FEAC6164FEAD6764FF000072EB9504689
:20274000FEF742FA08B14FF00107002F52D1286838B1686828B1A86818B1E86808B1286961
:2027600010B94FF0010745E02868A0F1010160686FF3020001F0070140EA01006060A868E1
:20278000A0F1010160686FF3124001F007014FEA014140EA010060606868A0F101016068A0
:2027A0006FF3D54001F007014FEAC14140EA01006060E868A0F1010160686FF31F6001F006
:2027C000FF014FEA016140EA010060602869A0F1010160686FF3975001F003014FEA81513E
:2027E00040EA010060602EB95046FEF737FA08B14FF001073846BDE8F0842DE9F0448246A2
:202800000D4650464FEA80004EF6C431C0F201010844046826684FEAC6164FEAD6764FF00A
:2028200000072EB95046FEF7CFF908B14FF00107002F54D1286838B1686828B1A86818B108
:20284000E86808B1286910B94FF0010747E02868A0F10101206D6FF38F2001F03F014FEA7C
:20286000812140EA01002065A868A0F10101206D6FF3040001F01F0140EA010020656868DF
:20288000A0F10101206D6FF3491001F01F014FEA411140EA01002065E868A0F10101206DA1
:2028A0006FF35E5040F2FF3201EA02014FEA415140EA010020652869A0F10101206D6FF329
:2028C000144001F01F014FEA014140EA010020652EB95046FEF7C2F908B14FF001073846BD
:2028E000BDE8F0842DE9F04482460D4650464FEA80004EF6C431C0F20101084404682668D8
:202900004FEAC6164FEAD6764FF000072EB95046FEF75AF908B14FF00107002F5CD1286826
:2029200038B1686828B1A86818B1E86808B1286910B94FF0010748E02968D4F8040C6FF38B
:202940008E2001F01F014FEA812140EA0100C4F8040CA868A0F10101D4F8040C6FF3020003
:2029600001F0070140EA0100C4F8040C6868A0F10101D4F8040C6FF3471001F007014FEA3D
:20298000411140EA0100C4F8040CE868A0F10101D4F8040C6FF31D5040F2FF3201EA02010F
:2029A0004FEA015140EA0100C4F8040C2869A0F10101D4F8040C6FF3124001F007014FEAAF
:2029C000014140EA0100C4F8040C2EB95046FEF745F908B14FF001073846BDE8F084000077
:2029E00000000000F0B583B004460D4616461F4629462046FEF716F810B14FF0010021E0C7
:202A00004FF00F0000903B46324629462046FEF780FB40B94FF0000000903B46324629466A
:202A20002046FEF776FB18B929462046FDF7FAFF40B94FF0040000903B463246294620469D
:202A4000FEF767FB03B0F0BD2DE9F04486B004460D4616461F46DDF830A04FF0000005AB4D
:202A60000DF1130229462046FEF79CF9012802D14FF001002CE029462046FEF76EF8012843
:202A800002D14FF0010023E0059800684FEA00104FEA107030B1082804D0092802D04FF0F2
:202AA000020015E029462046FDF7BCFF10B14FF001000DE04FF0000002904FF00C00019000
:202AC000CDF800A03B46324629462046FEF7D2F906B0BDE8F084F0B583B004460D46164663
:202AE0001F464FF0000001AB0DF1030229462046FEF758F9012802D14FF001001CE02946C1
:202B00002046FEF72AF8012802D14FF0010013E0019800684FEA00104FEA107030B10828F5
:202B200004D0092802D04FF0020005E03B46324629462046FFF756FF03B0F0BD2DE9F04CCD
:202B400083B004468A46174620464FEA80004EF6A431C0F20101084406684FF0000501AB35
:202B60000DF103025FFA8AF001462046FEF71AF9012802D14FF001050AE0019800F1080B02
:202B800051462046FDF7E9FF012801D14FF00105002D40F0A58001980068019800684FEA5F
:202BA00000304FEA1070FDF773FF82469DF803102046FEF77BF8824505D99DF803102046D5
:202BC000FEF774F8824687F848A00198006838600198006810F4001F05D00198406820F082
:202BE0006040786006E0019840684FEAC0004FEA505078604FEAAA00C0B201464FF00000B1
:202C000052E04FEA800207F108031A44019C03464FEA830304F1080423441B6803F07F4321
:202C20004FEA1363DBB2137007F1080202F101024FEA80031A44019C03464FEA830304F129
:202C4000080423441B6803F47F034FEA1343DBB2137007F1080202F102024FEA80031A4453
:202C6000019C03464FEA830304F1080423441B6803F47F434FEA1323DBB2137007F108028A
:202C800002F103024FEA80031A44019C03464FEA830304F1080423441B6803F0FF03DBB210
:202CA000137000F10100C0B28842AAD34FEA8100C0B212E020F0030100F00302C2F1030207
:202CC000114401F03F01C9B207F10802024459440978117000F10100C0B25045EAD3B0683E
:202CE000284603B0BDE8F08C0000000000000000000000000000000010B44FF0000306285E
:202D000002D34FF0010313E0032902D94FF001030EE04FF04C0410FB04F040F6EC74C2F298
:202D2000000420440C464FEA8404214608440260184610BC70472DE9F04F83B005460C46FD
:202D40001646019328464FEA80004EF6C431C0F201010844D0F800A028464FEA80004EF650
:202D6000A431C0F2010108440768DAF800B04FEACB1B4FEADB7B4FF000098DF80390BBF1D3
:202D8000000F07D12846FDF71FFF18B14FF001098DF803909DF80380B8F1000F40F09D8283
:202DA0002046102800F28E820FF20408D8E810F04E004E0097009700EC00EC0035017E014F
:202DC0007E017E019B019B019B01C801C8011100E901EEB9B86ADDF8048040EA0800B86226
:202DE000786ADDF8308040EA08007862062D02D0072D40F06782F86EDDF8348040EA0800ED
:202E0000F866B86EDDF8388040EA0800B86659E2B86ADDF8048020EA0800B862786ADDF8B8
:202E2000308020EA08007862062D02D0072D40F04982F86EDDF8348020EA0800F866B86E3D
:202E4000DDF8388020EA0800B8663BE21EBB20464FEA80004EF6E431C0F20101014478686E
:202E6000096840EA0100786020464FEA80004EF62041C0F2010100EB010228464FEA800051
:202E800040F6CC71C2F2000101440868126840EA0200086016E220464FEA80004EF6E431D7
:202EA000C0F2010101447868096820EA0100786020464FEA80004EF62041C0F2010100EB82
:202EC000010228464FEA800040F6CC71C2F2000101440868126820EA02000860F2E14EBB21
:202EE000DAF8000040F40010CAF8000020464FEA80004EF6E431C0F2010101447868096838
:202F000040EA0100786020464FEA80004EF62041C0F2010100EB010228464FEA800040F6EB
:202F2000CC71C2F2000101440868126840EA02000860C7E1DAF800006FF35550CAF8000099
:202F400020464FEA80004EF6E431C0F2010101447868096820EA0100786020464FEA8000AD
:202F60004EF62041C0F2010100EB010228464FEA800040F6CC71C2F200010144086812688C
:202F800020EA020008609DE11EBB20464FEA80004EF6E431C0F201010144786B096840EA77
:202FA0000100786320464FEA80004EF62041C0F2010100EB010228464FEA800040F6CC7135
:202FC000C2F2000101440868126840EA0200086078E120464FEA80004EF6E431C0F20101F4
:202FE0000144786B096820EA0100786320464FEA80004EF62041C0F2010100EB010228467E
:203000004FEA800040F6CC71C2F2000101440868126820EA0200086054E11EBB20464FEA7F
:2030200080004EF6E431C0F2010101443868096840EA0100386020464FEA80004EF6204126
:20304000C0F2010100EB010228464FEA800040F6CC71C2F2000101440868126840EA020024
:2030600008602FE120464FEA80004EF6E431C0F2010101443868096820EA0100386020464D
:203080004FEA80004EF62041C0F2010100EB010228464FEA800040F6CC71C2F2000101449C
:2030A0000868126820EA020008600BE16EB920464FEA80004EF6E431C0F201010144B86A0C
:2030C000096840EA0100B862FCE020464FEA80004EF6E431C0F201010144B86A096820EA50
:2030E0000100B862EEE0DAF8340040F00050CAF83400DAF8E00A6FF3DF70CAF8E00A7EB91B
:2031000020464FEA80004EF6E431C0F201010144D7F8E00A096840EA0100C7F8E00AD1E08F
:2031200020464FEA80004EF6E431C0F201010144D7F8E00A096820EA0100C7F8E00AC1E09F
:203140007EB920464FEA80004EF6E431C0F201010144D7F8000B096840EA0100C7F8000B87
:20316000B0E020464FEA80004EF6E431C0F201010144D7F8000B096820EA0100C7F8000B2E
:20318000A0E0002E4DD1B86A40F0FF30B862786A40F0FF307862062D01D0072D07D1F86E37
:2031A00040F0FF30F866B86E40F0FF30B866786840F44C407860786B40F040407863DAF8F7
:2031C000340040F00050CAF83400DAF8E00A6FF3DF70CAF8E00AD7F8E00A40F45020C7F810
:2031E000E00ADAF8000040F08060CAF80000DAF8000040F40010CAF80000D7F8000B40F45B
:203200004030C7F8000B28464FEA800040F6CC71C2F20001084440F20701C0F21B01016070
:2032200050E0B86A00F00000B862786A00F000007862062D01D0072D07D1F86E00F0000020
:20324000F866B86E00F00000B86678686FF44C4100EA01007860786B20F040407863DAF829
:20326000340040F00050CAF83400DAF8E00A6FF3DF70CAF8E00AD7F8E00A6FF4502100EA14
:203280000100C7F8E00ADAF800006FF39A60CAF80000DAF800006FF35550CAF80000D7F82A
:2032A000000B6FF4403100EA0100C7F8000B28464FEA800040F6CC71C2F2000108444FF0A0
:2032C00000010160BBF1000F07D12846FDF7C6FC18B14FF001098DF803909DF8030003B060
:2032E000BDE8F08F10B403464FEA83034EF6A434C0F2010423441B684FF00004202912D2B1
:2033000042B94FF0010000FA01F1986A40EA0100986263E04FF0010000FA01F1986A20EAE4
:20332000010098625AE0402916D252B9A1F120004FF0010101FA00F1586A40EA0100586276
:203340004CE0A1F120004FF0010101FA00F1586A20EA0100586241E060291DD2062801D043
:20336000072816D152B9A1F140004FF0010101FA00F1D86E40EA0100D8662FE0A1F140009D
:203380004FF0010101FA00F1D86E20EA0100D86624E04FF0010421E080291DD2062801D091
:2033A000072816D152B9A1F160004FF0010101FA00F1986E40EA010098660FE0A1F16000BD
:2033C0004FF0010101FA00F1986E20EA0100986604E04FF0010401E04FF00104204610BC32
:2033E000704700000000000000B581B04FF00000FDF7ABFFBFF34F8F01B000BD00B581B06F
:203400004FF00000FEF724F8BFF34F8F01B000BD00B581B04FF00000FEF75BF8BFF34F8F61
:2034200001B000BD00B581B04FF00000FEF792F8BFF34F8F01B000BD00B581B04FF0000057
:20344000FEF7E0F8BFF34F8F01B000BD00B581B04FF00000FEF72EF9BFF34F8F01B000BD62
:2034600000B581B04FF00000FEF7A6F9BFF34F8F01B000BD00B581B04FF00000FEF7DDF9A5
:20348000BFF34F8F01B000BD00B581B04FF00000FEF78AFABFF34F8F01B000BD00B581B0AC
:2034A0004FF00000FEF75DFBBFF34F8F01B000BD00B581B04FF00000FEF7B0FBBFF34F8F2D
:2034C00001B000BD00B581B04FF00000FEF70AFCBFF34F8F01B000BD00B581B04FF001003A
:2034E000FDF733FFBFF34F8F01B000BD00B581B04FF00100FDF7ACFFBFF34F8F01B000BDE5
:2035000000B581B04FF00100FDF7E3FFBFF34F8F01B000BD00B581B04FF00100FEF71AF884
:20352000BFF34F8F01B000BD00B581B04FF00100FEF768F8BFF34F8F01B000BD00B581B02E
:203540004FF00100FEF7B6F8BFF34F8F01B000BD00B581B04FF00100FEF72EF9BFF34F8FB8
:2035600001B000BD00B581B04FF00100FEF765F9BFF34F8F01B000BD00B581B04FF0010040
:20358000FEF712FABFF34F8F01B000BD00B581B04FF00100FEF7E5FABFF34F8F01B000BD34
:2035A00000B581B04FF00100FEF738FBBFF34F8F01B000BD00B581B04FF00100FEF792FB17
:2035C000BFF34F8F01B000BD00B581B04FF00200FDF7BBFEBFF34F8F01B000BD00B581B035
:2035E0004FF00200FDF734FFBFF34F8F01B000BD00B581B04FF00200FDF76BFFBFF34F8F50
:2036000001B000BD00B581B04FF00200FDF7A2FFBFF34F8F01B000BD00B581B04FF002005B
:20362000FDF7F0FFBFF34F8F01B000BD00B581B04FF00200FEF73EF8BFF34F8F01B000BD59
:2036400000B581B04FF00200FEF7B6F8BFF34F8F01B000BD00B581B04FF00200FEF7EDF8A1
:20366000BFF34F8F01B000BD00B581B04FF00200FEF79AF9BFF34F8F01B000BD00B581B0B9
:203680004FF00200FEF76DFABFF34F8F01B000BD00B581B04FF00200FEF7C0FABFF34F8F29
:2036A00001B000BD00B581B04FF00200FEF71AFBBFF34F8F01B000BD00B581B04FF0030045
:2036C000FDF743FEBFF34F8F01B000BD00B581B04FF00300FDF7BCFEBFF34F8F01B000BDE3
:2036E00000B581B04FF00300FDF7F3FEBFF34F8F01B000BD00B581B04FF00300FDF72AFF7A
:20370000BFF34F8F01B000BD00B581B04FF00300FDF778FFBFF34F8F01B000BD00B581B034
:203720004FF00300FDF7C6FFBFF34F8F01B000BD00B581B04FF00300FEF73EF8BFF34F8FAD
:2037400001B000BD00B581B04FF00300FEF775F8BFF34F8F01B000BD00B581B04FF003004B
:20376000FEF722F9BFF34F8F01B000BD00B581B04FF00300FEF7F5F9BFF34F8F01B000BD32
:2037800000B581B04FF00300FEF748FABFF34F8F01B000BD00B581B04FF00300FEF7A2FA13
:2037A000BFF34F8F01B000BD00B581B04FF00400FDF7CBFDBFF34F8F01B000BD00B581B042
:2037C0004FF00400FDF744FEBFF34F8F01B000BD00B581B04FF00400FDF77BFEBFF34F8F4C
:2037E00001B000BD00B581B04FF00400FDF7B2FEBFF34F8F01B000BD00B581B04FF0040067
:20380000FDF700FFBFF34F8F01B000BD00B581B04FF00400FDF74EFFBFF34F8F01B000BD4F
:2038200000B581B04FF00400FDF7C6FFBFF34F8F01B000BD00B581B04FF00400FDF7FDFF8F
:20384000BFF34F8F01B000BD00B581B04FF00400FEF7AAF8BFF34F8F01B000BD00B581B0C6
:203860004FF00400FEF77DF9BFF34F8F01B000BD00B581B04FF00400FEF7D0F9BFF34F8F25
:2038800001B000BD00B581B04FF00400FEF72AFABFF34F8F01B000BD00B581B04FF0050050
:2038A000FDF753FDBFF34F8F01B000BD00B581B04FF00500FDF7CCFDBFF34F8F01B000BDE1
:2038C00000B581B04FF00500FDF703FEBFF34F8F01B000BD00B581B04FF00500FDF73AFE75
:2038E000BFF34F8F01B000BD00B581B04FF00500FDF788FEBFF34F8F01B000BD00B581B042
:203900004FF00500FDF7D6FEBFF34F8F01B000BD00B581B04FF00500FDF74EFFBFF34F8FA2
:2039200001B000BD00B581B04FF00500FDF785FFBFF34F8F01B000BD00B581B04FF005004F
:20394000FEF732F8BFF34F8F01B000BD00B581B04FF00500FEF705F9BFF34F8F01B000BD2F
:2039600000B581B04FF00500FEF758F9BFF34F8F01B000BD00B581B04FF00500FEF7B2F90F
:20398000BFF34F8F01B000BD00B581B04FF00600FDF7DBFCBFF34F8F01B000BD00B581B04F
:2039A0004FF00600FDF754FDBFF34F8F01B000BD00B581B04FF00600FDF78BFDBFF34F8F48
:2039C00001B000BD00B581B04FF00600FDF7C2FDBFF34F8F01B000BD00B581B04FF0060072
:2039E000FDF710FEBFF34F8F01B000BD00B581B04FF00600FDF75EFEBFF34F8F01B000BD4E
:203A000000B581B04FF00600FDF7D6FEBFF34F8F01B000BD00B581B04FF00600FDF70DFF8A
:203A2000BFF34F8F01B000BD00B581B04FF00600FEF7BBF9BFF34F8F01B000BD00B581B0D0
:203A40004FF00600FEF78EFABFF34F8F01B000BD00B581B04FF00600FEF7E5FABFF34F8F17
:203A600001B000BD00B581B04FF00600FEF73DFBBFF34F8F01B000BD00B581B04FF0070056
:203A8000FDF763FCBFF34F8F01B000BD00B581B04FF00700FDF7DCFCBFF34F8F01B000BDDF
:203AA00000B581B04FF00700FDF713FDBFF34F8F01B000BD00B581B04FF00700FDF74AFD71
:203AC000BFF34F8F01B000BD00B581B04FF00700FDF798FDBFF34F8F01B000BD00B581B04F
:203AE0004FF00700FDF7E6FDBFF34F8F01B000BD00B581B04FF00700FDF75EFEBFF34F8F9F
:203B000001B000BD00B581B04FF00700FDF795FEBFF34F8F01B000BD00B581B04FF007005A
:203B2000FEF743F9BFF34F8F01B000BD00B581B04FF00700FEF716FABFF34F8F01B000BD27
:203B400000B581B04FF00700FEF76DFABFF34F8F01B000BD00B581B04FF00700FEF7C5FAFF
:203B6000BFF34F8F01B000BD2DE9004144F21408C4F20608D8F8000010F4802F3DD044F214
:203B80001408C4F20608D8F8000010F0004F07D04FF0B64044F21408C4F20608C8F8000044
:203BA00044F21408C4F20608D8F8000040F4802044F21408C4F20608C8F8000044F2140823
:203BC000C4F20608D8F8000040F0004044F21408C4F20608C8F8000041F24C28C2F20008A8
:203BE000D8F8000038B141F24C28C2F20008D8F80000804701E000F00AFB44F21C08C4F22C
:203C00000608D8F8000010F4802F3FD044F21C08C4F20608D8F8000010F0004F07D04FF0B1
:203C2000B64044F21C08C4F20608C8F8000044F21C08C4F20608D8F8000040F4802044F2B8
:203C40001C08C4F20608C8F8000044F21C08C4F20608D8F8000040F0004044F21C08C4F24E
:203C60000608C8F8000041F24C20C2F2000000F10400006840B141F24C20C2F2000000F191
:203C800004000068804701E000F0F3FABFF34F8FBDE8008100004DF8048D44F21C08C4F297
:203CA0000608D8F8001011F0004F07D04FF0B64144F21C08C4F20608C8F8001044F21C0871
:203CC000C4F20608D8F800106FF3410100F001024FEA420241EA020144F21C08C4F20608E0
:203CE000C8F8001044F21C08C4F20608D8F8001041F0010144F21C08C4F20608C8F80010D5
:203D000044F21C08C4F20608D8F8001041F0004144F21C08C4F20608C8F800105DF8048B61
:203D200070472DE9004144F22808C4F20608D8F8001011F0004F07D04FF0B64144F22808A8
:203D4000C4F20608C8F8001044F22808C4F20608D8F8001041F4007144F22808C4F20608F5
:203D6000C8F8001044F22808C4F20608D8F800106FF3410100F001024FEA420241EA020127
:203D800044F22808C4F20608C8F8001044F22808C4F20608D8F8001041F0010144F2280886
:203DA000C4F20608C8F8001044F22808C4F20608D8F8001041F0004144F22808C4F20608C9
:203DC000C8F800104FF0050000F07FFD88BB4FF0B64044F22808C4F20608C8F8000044F2CB
:203DE0002808C4F20608D8F8001041F0007144F22808C4F20608C8F8001044F22808C4F237
:203E00000608D8F800106FF3492144F22808C4F20608C8F8001044F22808C4F20608D8F8F4
:203E2000001041F0004144F22808C4F20608C8F80010BDE800812DE9104181B044F21808F2
:203E4000C4F20608D8F8003013F0004F07D04FF0B64344F21808C4F20608C8F8003044F2FD
:203E60001808C4F20608D8F800306FF3820300F001044FEA840443EA040344F21808C4F281
:203E80000608C8F8003044F21808C4F20608D8F800306FF3000302F0010043EA000344F24C
:203EA0001808C4F20608C8F8003044F21808C4F20608D8F8003043F0020344F21808C4F2D0
:203EC0000608C8F8003044F21808C4F20608D8F8003043F0004344F21808C4F20608C8F87A
:203EE000003044F21408C4F20608D8F8000010F0004F07D04FF0B64044F21408C4F206083B
:203F0000C8F8000044F21408C4F20608D8F800306FF3410301F001014FEA410143EA010386
:203F200044F21408C4F20608C8F8003044F21408C4F20608D8F8001041F0010144F2140800
:203F4000C4F20608C8F8001044F21408C4F20608D8F8001041F0004144F21408C4F206084F
:203F6000C8F800104FF0040000F0AFFC01B0BDE810812DE9104181B04FF0000401283BD19C
:203F80004FF0030000F0A1FC08B14FF00104002C40F0AD8044F20C08C4F20608D8F80000EE
:203FA00010F0004F07D04FF0B64044F20C08C4F20608C8F8000044F20C08C4F20608D8F8FA
:203FC00000006FF4E02100EA010040F4803044F20C08C4F20608C8F8000044F20C08C4F2E0
:203FE0000608D8F8000040F0004044F20C08C4F20608C8F800007AE002283AD14FF00400D3
:2040000000F063FC08B14FF00104002C6FD144F20C08C4F20608D8F8000010F0004F07D0E4
:204020004FF0B64044F20C08C4F20608C8F8000044F20C08C4F20608D8F800006FF4E0213B
:2040400000EA010040F4003044F20C08C4F20608C8F8000044F20C08C4F20608D8F8000065
:2040600040F0004044F20C08C4F20608C8F800003DE0032839D14FF0050000F026FC08B1A1
:204080004FF001049CBB44F20C08C4F20608D8F8000010F0004F07D04FF0B64044F20C0802
:2040A000C4F20608C8F8000044F20C08C4F20608D8F800006FF4E02100EA010040F44030AB
:2040C00044F20C08C4F20608C8F8000044F20C08C4F20608D8F8000040F0004044F20C087A
:2040E000C4F20608C8F8000001E04FF00104204601B0BDE8108100004DF8048D44F20001BD
:20410000C4F2060144F22C08C4F20608D8F8002012F0004F02D04FF0B642CA62427844F24E
:204120002C08C4F20608D8F800106FF3124102F007024FEA024241EA020144F22C08C4F22C
:204140000608C8F80010027844F22C08C4F20608D8F800106FF3010102F0030241EA020170
:2041600044F22C08C4F20608C8F80010426844F22C08C4F20608D8F800106FF30F2102F005
:20418000FF024FEA022241EA020144F22C08C4F20608C8F80010427A44F22C08C4F20608AB
:2041A000D8F800106FF3041102F001024FEA021241EA020144F22C08C4F20608C8F800103A
:2041C000017A44F22C08C4F20608D8F800006FF3451001F001014FEA411140EA010044F2D0
:2041E0002C08C4F20608C8F8000044F22C08C4F20608D8F8000040F0004044F22C08C4F279
:204200000608C8F800005DF8048B704700004DF8048D44F21408C4F20608D8F8000010F079
:20422000004F07D04FF0B64044F21408C4F20608C8F8000044F21408C4F20608D8F8000067
:204240006FF3492044F21408C4F20608C8F8000044F21408C4F20608D8F8000040F0004067
:2042600044F21408C4F20608C8F800005DF8048B70474DF8048D44F21C08C4F20608D8F809
:20428000000010F0004F07D04FF0B64044F21C08C4F20608C8F8000044F21C08C4F20608C7
:2042A000D8F800006FF3492044F21C08C4F20608C8F8000044F21C08C4F20608D8F8000097
:2042C00040F0004044F21C08C4F20608C8F800005DF8048B7047000000004DF8048D4FEAE6
:2042E00090024FEA820240F69013C2F200031A4413680246543A31D2283217D214320AD2C8
:20430000121D66D0121D64D0121D62D0121D60D0121D5ED00AE1121E5BD0121F59D0121FE7
:2043200057D0121F55D0121F53D0FFE0143A0AD2121D4ED0121D4CD0121D4AD0121D48D07B
:20434000121D46D0F2E0121E43D0121F41D0121F3FD0121F3DD0121F3BD0E7E0283A17D2F5
:2043600014320AD2121D34D0121D32D0121D30D0121D2ED0121D2CD0D8E0121E29D0121F1E
:2043800027D0121F25D0121F23D0121F21D0CDE00C3A0AD2921C00F29A8064D0521C2ED091
:2043A000521D16D0121D14D0C0E02C3A08D2121D0FD010320DD014320BD0121D09D0B5E0CA
:2043C000121E06D0121F04D0121F02D0121F40F0AD80186810F0004F02D04FF0B6401860F3
:2043E0001A686FF30B2201F00F014FEA012142EA01021A60196841F00041196096E044F28F
:204400000C08C4F20608D8F8000010F0004F07D04FF0B64044F20C08C4F20608C8F80000CB
:2044200044F20C08C4F20608D8F800206FF4706002EA00024FEA012040EA020044F20C088D
:20444000C4F20608C8F8000044F20C08C4F20608D8F8001041F0004144F20C08C4F206086A
:20446000C8F8001062E044F20C08C4F20608D8F8000010F0004F07D04FF0B64044F20C08A7
:20448000C4F20608C8F8000044F20C08C4F20608D8F800206FF0F00002EA00024FEA011013
:2044A00040EA020044F20C08C4F20608C8F8000044F20C08C4F20608D8F8001041F00041A2
:2044C00044F20C08C4F20608C8F800102EE044F20C08C4F20608D8F8000010F0004F07D0EC
:2044E0004FF0B64044F20C08C4F20608C8F8000044F20C08C4F20608D8F8002022F00F0298
:2045000041EA020044F20C08C4F20608C8F8000044F20C08C4F20608D8F8001041F0004140
:2045200044F20C08C4F20608C8F800105DF8048B70472DE910014FEA90024FEA820240F61D
:204540009013C2F200031A4412684FF000030446543C3AD2283418D214340BD2241D6ED017
:20456000241D6CD0241D6AD0241D68D0241D00F05581A2E1241E62D0241F60D0241F5ED0E8
:20458000241F5CD0241F5AD097E1143C0FD2241D00F0B080241D00F0AD80241D00F0AA807C
:2045A000241D00F0A780241D00F0A48085E1241E00F0A080241F00F09D80241F00F09A80F9
:2045C000241F3CD0241F3AD077E1283C17D214340AD2241D33D0241D31D0241D2FD0241D6F
:2045E0002DD0241D2BD068E1241E28D0241F26D0241F24D0241F22D0241F20D05DE1343C79
:204600000DD2103400F0BA80143400F00781241D00F00481083412D0241D10D04DE1241E28
:2046200000F0FC80241F00F0F980241F00F0F680241F00F0F380241F00F0F0803DE11068DA
:2046400010F0004F02D04FF0B64010600846052849D80FF20808D8E800F000BF3B040F1A10
:20466000253014686FF3061401F007014FEA011144EA0104146038E014686FF3061401F001
:2046800007014FEA011144EA010414602DE014686FF3061401F007014FEA011144EA0104A4
:2046A000146022E014686FF3061401F007014FEA011144EA0104146017E014686FF30614B2
:2046C00001F007014FEA011144EA010414600CE014686FF3061401F007014FEA011144EA99
:2046E0000104146001E04FF00103116841F000411160E4E0106810F0004F02D04FF0B6402F
:2047000010600C46241E27D0E41E30D303D0A41E0CD316D02BE014686FF3061401F0070143
:204720004FEA011144EA0104146022E014686FF3061401F007014FEA011144EA01041460A2
:2047400017E014686FF3061401F007014FEA011144EA010414600CE014686FF3061401F0AA
:2047600007014FEA011144EA0104146001E04FF00103116841F000411160A0E0106810F0C7
:20478000004F02D04FF0B6401060084606283ED80FF20408D8E800F0303B3B040F1A25000C
:2047A00014686FF3061401F007014FEA011144EA010414602DE014686FF3061401F0070118
:2047C0004FEA011144EA0104146022E014686FF3061401F007014FEA011144EA0104146002
:2047E00017E014686FF3061401F007014FEA011144EA010414600CE014686FF3061401F00A
:2048000007014FEA011144EA0104146001E04FF00103116841F00041116050E0106810F076
:20482000004F02D04FF0B6401060084604283DD80FF20408D8E800F02F030E19240014686D
:204840006FF3061401F007014FEA011144EA010414602DE014686FF3061401F007014FEABA
:20486000011144EA0104146022E014686FF3061401F007014FEA011144EA0104146017E0A3
:2048800014686FF3061401F007014FEA011144EA010414600CE014686FF3061401F0070158
:2048A0004FEA011144EA0104146001E04FF00103116841F00041116001E04FF00103184604
:2048C000BDE810017047000000004DF8048D4FF000014FF000020346052B74D80FF2040842
:2048E000D8E803F07103050406070EE022E036E04AE05EE048F2A060C0F20100814202D982
:204900004FF0010261E001F101014DF20408C4F20708D8F8000010F0040FEBD055E048F203
:20492000A060C0F20100814202D94FF001024CE001F1010144F21C08C4F20608D8F80000D6
:2049400010F4803FEBD040E044F64030C0F24C00814202D94FF0010237E001F1010149F2EB
:204960000008C4F20708D8F8000010F4007FEBD02BE048F2A060C0F20100814202D94FF087
:20498000010222E001F1010144F21408C4F20608D8F8000010F4803FEBD016E048F2A0608A
:2049A000C0F20100814202D94FF001020DE001F1010144F22808C4F20608D8F8000010F485
:2049C000803FEBD001E04FF0010210465DF8048B704700002DE9304143F21C08C4F20708A4
:2049E000D8F8005005F0030543F21808C4F20708D8F8000005EA000543F21C08C4F207089E
:204A0000C8F800504FF000042FE04FF0010000FA04F000EA050030B320464FEA800041F2E2
:204A20005421C2F200010844006850B120464FEA800041F25421C2F20001084400688047A0
:204A400011E04FF0010000FA04F143F21808C4F20708D8F8000020EA010043F21808C4F236
:204A60000708C8F8000004F10104022CCDD3BFF34F8FBDE8308130B581B0054628464FEAB1
:204A800080004EF67841C0F2010108440068846804F44034C16804EA0104C4604FF4003026
:204AA00000EA0400F8B128464FEA40004FEA800041F25C21C2F200010844006860B1284627
:204AC0004FEA40004FEA800041F25C21C2F2000108440068804706E028464FF001024FF0EF
:204AE000000100F02BF84FF4803000EA040018B341F25C20C2F2000000F1040128464FEAF6
:204B000040004FEA80000844006870B141F25C20C2F2000000F1040128464FEA40004FEA4E
:204B2000800008440068804706E028464FF001024FF0010100F002F801B030BD30B40346EE
:204B40004FEA83034EF68444C0F2010423441C6803464FEA830318464EF67843C0F20103CD
:204B600018440368A06810F0004F05D09D6825F07F4545F0B6459D606AB94FEA810108460B
:204B80004EF66C41C0F2010108449968006841EA000199600CE04FEA810108464EF66C41B0
:204BA000C0F2010108449968006821EA00019960A16841F00041A16030BC704700B581B082
:204BC0004FF00000FFF757FFBFF34F8F01B000BD00B581B04FF00100FFF74DFFBFF34F8F54
:204BE00001B000BD00B581B04FF00200FFF743FFBFF34F8F01B000BD2DE9104181B04FF013
:204C00000104BFF34F8F4EF60C58CEF20008D8F8000000F4E06040F20001C0F2FA5140EA31
:204C2000010040F004004EF60C58CEF20008C8F80000BFF34F8F00E000BF002CFCD101B036
:204C4000BDE810814DF8048D002800F09980427A42F21008C4F20308D8F800106FF300010B
:204C600002F0010241EA020142F21008C4F20308C8F80010027A42F21008C4F20308D8F8DB
:204C800000106FF3820102F001024FEA820241EA020142F21008C4F20308C8F8001042F22E
:204CA0001008C4F20308D8F8001011F0010F15D1426842F20C08C4F20308D8F800106FF34F
:204CC0000F014FF6FF7302EA030241EA020142F20C08C4F20308C8F8001006E0416842F252
:204CE0000C08C4F20308C8F80010C17A71B942F21008C4F20308D8F8001041F0C00142F297
:204D00001008C4F20308C8F800100FE042F21008C4F20308D8F800106FF3871141F0800162
:204D200042F21008C4F20308C8F80010827A42F21008C4F20308D8F800106FF3051102F043
:204D400003024FEA021241EA020142F21008C4F20308C8F8001042F21008C4F20308D8F819
:204D6000001041F0020142F21008C4F20308C8F80010006842F20808C4F20308C8F80000E5
:204D80005DF8048B70472DE930014FF00004012A13D142F21008C4F20308D8F8005045F07D
:204DA000020542F21008C4F20308C8F8005042F20808C4F20308C8F8003042F21008C4F2D8
:204DC0000308D8F800506FF3410542F21008C4F20308C8F8005024E004EB000204F10103F5
:204DE00003441B784FEA0323127843EA020204F1020303441B784FEA034343EA020204F146
:204E0000030303441B784FEA036343EA020542F20808C4F20308C8F8005004F10404A1F13B
:204E200004010429D8D20CE004EB0002127842F20808C4F2030888F80020A1F1010104F101
:204E400001040029F0D842F21008C4F20308D8F800004FEA80604FEA907008B1012807D173
:204E600042F20808C4F20308D8F8000080B208E042F20808C4F20308D8F800004FEA1040E5
:204E800080B2BDE8300170472DE9304148F21C08C4F20008D8F8005048F20C08C4F2000884
:204EA000D8F8000005EA00054FF000044BE020464FEA80004EF69041C0F201010844006824
:204EC00000EA0500E8B34FEA044048F28001C8F2000140EA010048F21408C4F20008C8F856
:204EE000000020464FEA40004FEA800041F27421C2F200010844006860B120464FEA4000F9
:204F00004FEA800041F27421C2F2000108440068804716E020464FEA80004EF69041C0F204
:204F20000101014448F20C08C4F20008D8F80000096820EA010048F20C08C4F20008C8F806
:204F4000000004F10104102CB1D3BDE830812DE9004148F22008C4F20008D8F80020014693
:204F60004FEA81014EF69043C0F201031944096801EA0201B1B34FEA006148F20002C0F201
:204F8000800241EA020140EA010148F21408C4F20008C8F8001041F27421C2F2000101F1E2
:204FA000040201464FEA41014FEA81011144096869B141F27421C2F2000101F104014FEAE1
:204FC00040004FEA80000844006880470AE04FEA401048F20021C4F20001014488696FF340
:204FE00041008861BDE8008100B581B04FF00000FFF7ADFFBFF34F8F01B000BD00B581B0B6
:205000004FF00100FFF7A3FFBFF34F8F01B000BD00B581B04FF00200FFF799FFBFF34F8F75
:2050200001B000BD00B581B04FF00300FFF78FFFBFF34F8F01B000BD00B581B04FF004002F
:20504000FFF785FFBFF34F8F01B000BD00B581B04FF00500FFF77BFFBFF34F8F01B000BD40
:2050600000B581B04FF00600FFF771FFBFF34F8F01B000BD00B581B04FF00700FFF767FF19
:20508000BFF34F8F01B000BD00B581B04FF00800FFF75DFFBFF34F8F01B000BD00B581B0AF
:2050A0004FF00900FFF753FFBFF34F8F01B000BD00B581B04FF00A00FFF749FFBFF34F8F65
:2050C00001B000BD00B581B04FF00B00FFF73FFFBFF34F8F01B000BD00B581B04FF00C00CF
:2050E000FFF735FFBFF34F8F01B000BD00B581B04FF00D00FFF72BFFBFF34F8F01B000BD38
:2051000000B581B04FF00E00FFF721FFBFF34F8F01B000BD00B581B04FF00F00FFF717FF08
:20512000BFF34F8F01B000BD00B581B0FFF7ACFEBFF34F8F01B000BD2DE9104181B041F222
:205140000004C4F206044FF0000000F017F8A06800F0100068B141F2F428C2F20008D8F851
:20516000000030B141F2F428C2F20008D8F800008047BFF34F8F01B0BDE8108141F2000200
:20518000C4F20602916841F080719160704700B581B0FFF7D1FF01B000BD2DE9F04581B0F8
:2051A000064630464FEA80004EF6E051C0F201010844056830464FEA80004EF6CC51C0F250
:2051C00001010844D0F800A0D5F890704FF000043FE04FF0010000FA04F000EA070070B3A8
:2051E00041F2F828C2F20008D8F8000050B141F2F828C2F20008D8F80020E0B20146304681
:2052000090471CE020464FEA80000AF1100108444FF0B641016020464FEA800005F1100187
:20522000014408686FF31340086020464FEA800005F110010144086840F4004008604FF0A6
:20524000010000FA04F000EA0700C5F8900004F10104202CBDD3BFF34F8F01B0BDE8F085F0
:2052600000B581B04FF00000FFF797FF01B000BD00B581B04FF00100FFF78FFF01B000BDF7
:2052800000B581B04FF00200FFF787FF01B000BD00B581B04FF00300FFF77FFF01B000BDF3
:2052A00000B581B04FF00400FFF777FF01B000BD30B403464FEA83034EF6E054C0F20104D0
:2052C00023441B6804464FEA840420464EF6CC54C0F20104204400680C464FEA840403F185
:2052E00010052C44246814F4004F08D00C464FEA840400F1100020444FF0B64404600C4607
:205300004FEA8404204603F11004204404686FF30A2402F007024FEA022244EA020404600E
:205320004FEA8101084603F110010844016841F40041016030BC704770B5044620464FEA22
:2053400080004EF66061C0F201010844056820464FEA80004EF65861C0F2010108440068D7
:20536000C66DC16906EA0106C6654FF0010000EA060020B320464FEAC001A1EB00004FEA86
:2053800040004FEA800041F2FC21C2F200010844006880B120464FEAC001A1EB00004FEA05
:2053A00040004FEA800041F2FC21C2F2000108440068804703E0E8696FF30000E8614FF056
:2053C000020000EA060040B341F2FC20C2F2000000F1040120464FEAC002A2EB00004FEAC8
:2053E00040004FEA80000844006890B141F2FC20C2F2000000F1040120464FEAC002A2EBD8
:2054000000004FEA40004FEA800008440068804703E0E8696FF34100E8614FF0040000EA92
:20542000060040B341F2FC20C2F2000000F1080120464FEAC002A2EB00004FEA40004FEAD6
:2054400080000844006890B141F2FC20C2F2000000F1080120464FEAC002A2EB00004FEAB3
:2054600040004FEA800008440068804703E0E8696FF38200E8614FF0080000EA060040B32D
:2054800041F2FC20C2F2000000F10C0120464FEAC002A2EB00004FEA40004FEA800008449F
:2054A000006890B141F2FC20C2F2000000F10C0120464FEAC002A2EB00004FEA40004FEAA2
:2054C000800008440068804703E0E8696FF3C300E8614FF0100000EA060040B341F2FC20AE
:2054E000C2F2000000F1100120464FEAC002A2EB00004FEA40004FEA80000844006890B1E1
:2055000041F2FC20C2F2000000F1100120464FEAC002A2EB00004FEA40004FEA800008441A
:205520000068804703E0E8696FF30410E8614FF0200000EA060040B341F2FC20C2F2000004
:2055400000F1140120464FEAC002A2EB00004FEA40004FEA80000844006890B141F2FC20E1
:20556000C2F2000000F1140120464FEAC002A2EB00004FEA40004FEA8000084400688047D6
:2055800003E0E8696FF34510E8614FF4800000EA060040B341F2FC20C2F2000000F1180124
:2055A00020464FEAC002A2EB00004FEA40004FEA80000844006890B141F2FC20C2F20000D3
:2055C00000F1180120464FEAC002A2EB00004FEA40004FEA800008440068804703E0E869F2
:2055E0006FF39650E8614FF4000000EA060040B341F2FC20C2F2000000F11C0120464FEA44
:20560000C002A2EB00004FEA40004FEA80000844006890B141F2FC20C2F2000000F11C0103
:2056200020464FEAC002A2EB00004FEA40004FEA800008440068804703E0E8696FF3D75012
:20564000E8614FF0807000EA060040B341F2FC20C2F2000000F1200120464FEAC002A2EBEC
:2056600000004FEA40004FEA80000844006890B141F2FC20C2F2000000F1200120464FEA4F
:20568000C002A2EB00004FEA40004FEA800008440068804703E0E8696FF31860E8614FF078
:2056A000007000EA060040B341F2FC20C2F2000000F1240120464FEAC002A2EB00004FEA57
:2056C00040004FEA80000844006890B141F2FC20C2F2000000F1240120464FEAC002A2EBD5
:2056E00000004FEA40004FEA800008440068804703E0E8696FF35960E8614FF0806000EA5C
:20570000060040B341F2FC20C2F2000000F1280120464FEAC002A2EB00004FEA40004FEAD3
:2057200080000844006890B141F2FC20C2F2000000F1280120464FEAC002A2EB00004FEAB0
:2057400040004FEA800008440068804703E0E8696FF39A60E8614FF0006000EA060040B37A
:2057600041F2FC20C2F2000000F12C0120464FEAC002A2EB00004FEA40004FEA800008449C
:20578000006890B141F2FC20C2F2000000F12C0120464FEAC002A2EB00004FEA40004FEA9F
:2057A000800008440068804703E0E8696FF3DB60E8614FF0804000EA060040B341F2FC20A3
:2057C000C2F2000000F1300120464FEAC002A2EB00004FEA40004FEA80000844006890B1DE
:2057E00041F2FC20C2F2000000F1300120464FEAC002A2EB00004FEA40004FEA8000084418
:205800000068804703E0E8696FF39E70E8614FF0004000EA060040B341F2FC20C2F2000007
:2058200000F1340120464FEAC002A2EB00004FEA40004FEA80000844006890B141F2FC20DE
:20584000C2F2000000F1340120464FEAC002A2EB00004FEA40004FEA8000084400688047D3
:2058600003E0E8696FF3DF70E861BFF34F8F70BD00B581B04FF00000FFF75EFD01B000BD59
:2058800000B581B04FF00100FFF756FD01B000BD2DE9F044054628464FEA80004EF6BC610E
:2058A000C0F201010844076828464FEA80004EF6B461C0F201010844D0F800A04FF000044E
:2058C000EFE02146284600F003F9064628464FEA800020444FEA800041F2EC31C2F20001A3
:2058E0000844006806EA000620464FEA800108444FEA80000AF108010844C6604FF0100014
:2059000000EA060058B328464FEA800020444FEA80004FEA800041F26C31C2F200010844BE
:20592000006878B128464FEA800020444FEA80004FEA800041F26C31C2F2000108440068A0
:2059400080470CE020464FEA800108444FEA800007F108010144C8686FF30000C8604FF030
:20596000200000EA060078B341F26C30C2F2000000F1040029464FEA810121444FEA81012A
:205980004FEA81010844006888B141F26C30C2F2000000F1040029464FEA810121444FEA1F
:2059A00081014FEA81010844006880470CE020464FEA800108444FEA800007F108010144D8
:2059C000C8686FF34100C8604FF0400000EA060078B341F26C30C2F2000000F10800294647
:2059E0004FEA810121444FEA81014FEA81010844006888B141F26C30C2F2000000F10800A8
:205A000029464FEA810121444FEA81014FEA81010844006880470CE020464FEA80010844AE
:205A20004FEA800007F108010144C8686FF38200C8604FF0800000EA060078B341F26C3082
:205A4000C2F2000000F10C0128464FEA800020444FEA80004FEA80000844006888B141F277
:205A60006C30C2F2000000F10C0029464FEA810121444FEA81014FEA810108440068804759
:205A80000CE020464FEA800108444FEA800007F108010144C8686FF3C300C86004F101003C
:205AA000C4B2042CFFF40DAFBFF34F8FBDE8F08400B581B04FF00000FFF7EAFE01B000BD77
:205AC00000B581B04FF00100FFF7E2FE01B000BD02464FEA820210464EF6B462C0F20102F2
:205AE000104403680A464FEA820002444FEA8202104603F108010844C268104670470028DB
:205B00000FDB4FEA50114FEA81014EF20012CEF20002114400F01F004FF0010202FA00F0A0
:205B20000860704700B581B0002813DB4FEA50114FEA81014EF28012CEF20002114400F01C
:205B40001F004FF0010202FA00F00860BFF34F8FBFF36F8F01B000BD00280BDB4EF2004252
:205B6000CEF2000210444FEA011101F0FF01C9B201700EE000F00F00A0F104004EF61852B7
:205B8000CEF2000210444FEA011101F0FF01C9B2017070472DE9104181B04FF00004A0F1A4
:205BA0000101B1F1807F02D34FF001041DE0A0F101004EF21408CEF20008C8F800004FF077
:205BC0000F014FF0FF30FFF7C7FF4FF000004EF21808CEF20008C8F800004FF007004EF2DE
:205BE0001008CEF20008C8F80000204601B0BDE8108100002DE9F04405464FF000044FF0A1
:205C0000000028464FEA80004EF6E061C0F201010844076828464FEA80004EF6D861C0F213
:205C200001010844D0F800A04FF6FF76B86B06EA00064FF0000444E04FF0010000FA04F046
:205C400000EA0600D8B320464FEA80000AF13C010844006810F0100F31D020464FEA80007F
:205C600007F13C01084400686FF0200100EA010021464FEA810107F13C021144086005EBCB
:205C8000051020444FEA800041F20C41C2F200010844006860B105EB051020444FEA8000B6
:205CA00041F20C41C2F2000108440068804706E0E0B2014628464FF0010200F023FA04F1C3
:205CC0000104072CB8D9BFF34F8FBDE8F08400B581B04FF0000101464FEA81014EF6E062A4
:205CE000C0F2010211440A684FF03001D2F8903001EA03014FF0300303EA010343B3D2F81C
:205D000090106FF0300301EA0301C2F8901041F20C41C2F2000101F1400200EB00114FEA6A
:205D200081011144096869B141F20C41C2F2000101F1400100EB00104FEA80000844006831
:205D4000804705E04FF001024FF0100100F0DAF9BFF34F8F01B000BD70B504464FF0000096
:205D600020464FEA80004EF6E061C0F20101084405684FF6FF76A86B06EA00064FF480503C
:205D800000EA060038B3A86B6FF4805100EA0100A86341F20C40C2F2000000F1300104EBA7
:205DA00004104FEA80000844006868B141F20C40C2F2000000F1300104EB04104FEA800038
:205DC00008440068804706E020464FF001024FF00C0100F097F94FF4005000EA060038B380
:205DE000A86B6FF4005100EA0100A86341F20C40C2F2000000F1340104EB04104FEA8000D1
:205E00000844006868B141F20C40C2F2000000F1340104EB04104FEA800008440068804725
:205E200006E020464FF001024FF00D0100F06AF94FF4804000EA060038B3A86B6FF480411F
:205E400000EA0100A86341F20C40C2F2000000F1380104EB04104FEA80000844006868B166
:205E600041F20C40C2F2000000F1380104EB04104FEA800008440068804706E020464FF003
:205E800001024FF00E0100F03DF94FF4004000EA060038B3A86B6FF4004100EA0100A86380
:205EA00041F20C40C2F2000000F13C0104EB04104FEA80000844006868B141F20C40C2F2C5
:205EC000000000F13C0104EB04104FEA800008440068804706E020464FF001024FF00F0180
:205EE00000F010F9BFF34F8F70BD70B504464FF0000020464FEA80004EF6E061C0F20101E6
:205F0000084405684FF6FF76A86B06EA00064FF4807000EA060038B3A86B6FF4807100EAA6
:205F20000100A86341F20C40C2F2000000F1200104EB04104FEA80000844006868B141F254
:205F40000C40C2F2000000F1200104EB04104FEA800008440068804706E020464FF001026A
:205F60004FF0080100F0CEF84FF4007000EA060038B3A86B6FF4007100EA0100A86341F285
:205F80000C40C2F2000000F1240104EB04104FEA80000844006868B141F20C40C2F200002F
:205FA00000F1240104EB04104FEA800008440068804706E020464FF001024FF0090100F0CD
:205FC000A1F84FF4806000EA060038B3A86B6FF4806100EA0100A86341F20C40C2F20000AA
:205FE00000F1280104EB04104FEA80000844006868B141F20C40C2F2000000F1280104EBC2
:2060000004104FEA800008440068804706E020464FF001024FF00A0100F074F84FF4006061
:2060200000EA060038B3A86B6FF4006100EA0100A86341F20C40C2F2000000F12C0104EB78
:2060400004104FEA80000844006868B141F20C40C2F2000000F12C0104EB04104FEA800099
:2060600008440068804706E020464FF001024FF00B0100F047F8BFF34F8F70BD00B581B0FA
:206080004FF00000FFF7B6FD01B000BD00B581B04FF00000FFF71BFE01B000BD00B581B022
:2060A0004FF00000FFF758FE01B000BD00B581B04FF00000FFF719FF01B000BD00B581B060
:2060C0004FF00100FFF796FD01B000BD00B581B04FF00100FFF7FBFD01B000BD00B581B021
:2060E0004FF00100FFF738FE01B000BD00B581B04FF00100FFF7F9FE01B000BD0000000045
:20610000000000002DE9700103464FEA830318464EF6D863C0F2010318440368002A14BF99
:20612000002001200446112900F2AE810FF20408D8E801F00914233241505F6E7D88939EB5
:20614000A9B4BFCAD5E2D96B6FF3041104F001044FEA041441EA0401D96395E103F13C008B
:2061600000F1040529686FF3041104F001034FEA031341EA0301296086E103F13C0000F196
:20618000080529686FF3041104F001034FEA031341EA0301296077E103F13C0000F10C0561
:2061A00029686FF3041104F001034FEA031341EA0301296068E103F13C0000F110052968C8
:2061C0006FF3041104F001034FEA031341EA0301296059E103F13C0000F1140529686FF3E2
:2061E000041104F001034FEA031341EA030129604AE103F13C0000F1180529686FF304111A
:2062000004F001034FEA031341EA030129603BE103F13C0000F11C0529686FF3041104F025
:2062200001034FEA031341EA030129602CE1596B6FF3104104F001044FEA044441EA040125
:20624000596321E1596B6FF3514104F001044FEA444441EA0401596316E1596B6FF3924132
:2062600004F001044FEA844441EA040159630BE1596B6FF3D34104F001044FEAC44441EAAD
:206280000401596300E1596B6FF3145104F001044FEA045441EA04015963F5E0596B6FF360
:2062A000555104F001044FEA445441EA04015963EAE0596B6FF3965104F001044FEA8454A1
:2062C00041EA04015963DFE0596B6FF3D75104F001044FEAC45441EA04015963D4E0D3F810
:2062E0008C106FF30C3104F001044FEA043441EA0401C3F88C10C7E0D96B6FF3041104F01C
:2063000001054FEA051541EA0501D96303F13C0000F1040631686FF3041104F001054FEA49
:20632000051541EA0501316003F13C0000F1080631686FF3041104F001054FEA051541EACA
:206340000501316003F13C0000F10C0631686FF3041104F001054FEA051541EA0501316054
:2063600003F13C0000F1100631686FF3041104F001054FEA051541EA0501316003F13C0097
:2063800000F1140631686FF3041104F001054FEA051541EA0501316003F13C0000F1180694
:2063A00031686FF3041104F001054FEA051541EA0501316003F13C0000F11C0631686FF380
:2063C000041104F001054FEA051541EA05013160596B6FF3104104F001054FEA054541EA7A
:2063E00005015963596B6FF3514104F001054FEA454541EA05015963596B6FF3924104F08C
:2064000001054FEA854541EA05015963596B6FF3D34104F001054FEAC54541EA0501596322
:20642000596B6FF3145104F001054FEA055541EA05015963596B6FF3555104F001054FEA58
:20644000455541EA05015963596B6FF3965104F001054FEA855541EA05015963596B6FF388
:20646000D75104F001054FEAC55541EA05015963D3F88C106FF30C3104F001044FEA04344A
:2064800041EA0401C3F88C10BDE8700170470000000000002DE9104181B04DF21008C4F203
:2064A0000708D8F8004040F66428C2F20008D8F8000004EA000440F20000C9F273404DF29E
:2064C0000008C4F20708C8F800004DF21008C4F20708C8F800404DF20008C4F20708D8F837
:2064E000000040F000404DF20008C4F20708C8F800004FF0400000EA0400A0B141F2944893
:20650000C2F20008D8F8000038B141F29448C2F20008D8F80000804705E04FF001014FF03F
:20652000000000F024F84FF0800000EA0400B0B141F29440C2F2000000F10400006840B138
:2065400041F29440C2F2000000F104000068804705E04FF001014FF0010000F008F8BFF354
:206560004F8F01B0BDE810810000000000004DF8048D40F20002C9F273424DF20008C4F2DF
:206580000708C8F8002041BB02464FEA820211464EF63C72C0F2010211444DF21008C4F2AB
:2065A0000708D8F80020096842EA01024DF21008C4F20708C8F800204FEA80004EF63071A2
:2065C000C0F20101014440F66422C2F200021068096840EA0100106027E002464FEA8202C0
:2065E00011464EF63C72C0F2010211444DF21008C4F20708D8F80020096822EA01024DF27D
:206600001008C4F20708C8F800204FEA80004EF63071C0F20101014440F66422C2F20002B4
:206620001068096820EA010010604DF20008C4F20708D8F8000040F000404DF20008C4F2AD
:206640000708C8F800005DF8048B7047202802D34FF0010210E069B102464FEA820210460C
:206660004CF20002C4F207021044096801604FF0000201E04FF0010210467047202802D367
:206680004FF001020CE002464FEA820210464CF20002C4F207021044006808604FF000020D
:2066A000104670472DE9104181B049F21808C4F20708D8F8000010F0004F09D040F20000EB
:2066C000C9F6670049F21808C4F20708C8F8000049F20008C4F20708D8F8004041F2AC4875
:2066E000C2F20008D8F8000004EA00044FF4807000EA040030B34FF0FF3049F21008C4F2A1
:206700000708C8F8000041F29C40C2F2000000F10400006840B141F29C40C2F2000000F1E5
:206720000400006880470DE049F20408C4F20708D8F800006FF3041049F20408C4F20708DB
:20674000C8F800004FF0800000EA0400E0B141F29C48C2F20008D8F8000038B141F29C4898
:20676000C2F20008D8F8000080470DE049F20408C4F20708D8F800006FF3C30049F2040891
:20678000C4F20708C8F800004FF4006000EA040060B349F20008C4F20708D8F8000040F4C4
:2067A000006049F20008C4F20708C8F8000041F29C40C2F2000000F10800006840B141F269
:2067C0009C40C2F2000000F10800006880470DE049F20408C4F20708D8F800006FF3451081
:2067E00049F20408C4F20708C8F800004FF4005000EA040060B349F20008C4F20708D8F861
:20680000000040F4005049F20008C4F20708C8F8000041F29C40C2F2000000F10C00006804
:2068200040B141F29C40C2F2000000F10C00006880470DE049F20408C4F20708D8F80000AF
:206840006FF3861049F20408C4F20708C8F8000049F21808C4F20708D8F8000040F0004014
:2068600049F21808C4F20708C8F80000BFF34F8F01B0BDE8108100000000000000000000C1
:2068800000000000000000B581B0FFF70BFF01B000BD00B581B0FFF705FF01B000BD000056
:2068A0002DE9104181B048F24008C4F20408D8F8004041F2CC48C2F20008D8F8000004EA2B
:2068C000000448F24008C4F20408C8F800404FF0807000EA0400F0B141F2B040C2F20000DB
:2068E00000F10400006840B141F2B040C2F2000000F10400006880470DE048F20408C4F266
:206900000408D8F800006FF3186048F20408C4F20408C8F800004FF0007000EA0400F0B1BB
:2069200041F2B040C2F2000000F10800006840B141F2B040C2F2000000F10800006880472F
:206940000DE048F20408C4F20408D8F800006FF3596048F20408C4F20408C8F800004FF050
:20696000806000EA0400F0B141F2B040C2F2000000F10C00006840B141F2B040C2F20000A4
:2069800000F10C00006880470DE048F20408C4F20408D8F800006FF39A6048F20408C4F2AE
:2069A0000408C8F800004FF0006000EA0400F0B141F2B040C2F2000000F11000006840B1AC
:2069C00041F2B040C2F2000000F11000006880470DE048F20408C4F20408D8F800006FF389
:2069E000DB6048F20408C4F20408C8F800004FF0805000EA0400F0B141F2B040C2F200001F
:206A000000F11400006840B141F2B040C2F2000000F11400006880470DE048F20408C4F224
:206A20000408D8F800006FF31C7048F20408C4F20408C8F800004FF0005000EA0400F0B1A6
:206A400041F2B040C2F2000000F11800006840B141F2B040C2F2000000F1180000688047EE
:206A60000DE048F20408C4F20408D8F800006FF35D7048F20408C4F20408C8F800004FF417
:206A8000803000EA0400E0B141F2B048C2F20008D8F8000038B141F2B048C2F20008D8F870
:206AA000000080470DE048F20408C4F20408D8F800006FF3104048F20408C4F20408C8F8D0
:206AC0000000BFF34F8F01B0BDE8108100B581B0FFF7E6FE01B000BD00B581B0FFF7E0FE57
:206AE00001B000BD00000000000000002DE900414FF001004FF20C08C4F20708C8F80000B7
:206B000041F2D048C2F20008D8F8000030B141F2D048C2F20008D8F800008047BFF34F8F8F
:206B2000BDE800812DE9104181B04FF0000429E04FF0010000FA04F04FF21C08C4F20708F3
:206B4000D8F8001000EA0100D0B14FF21C08C4F20708C8F8000020464FEA800041F2D44198
:206B6000C2F200010844006850B120464FEA800041F2D441C2F2000108440168E0B2884779
:206B800004F10104112CD3D3BFF34F8F01B0BDE8108100B581B0FFF7A9FF01B000BD00B5FA
:206BA00081B0FFF7BFFF01B000BD00B581B001464FEA81014FF21802C0F2010211440968C4
:206BC00002464FEA82024FF20803C0F201031A441268136A4FF0010202EA0302D2B100EBB8
:206BE00080024FEA820241F21853C2F200031A4412685AB100EB80004FEA800041F218515E
:206C0000C2F2000108440068804703E0C8696FF30000C861BFF34F8F01B000BD00B581B0C1
:206C200001464FEA81014FF21802C0F201021144096802464FEA82024FF20803C0F2010375
:206C40001A441268136A4A6A02F001024FF0020202EA0302F2B141F21852C2F2000202F119
:206C6000040300EB80024FEA82021A4412686AB141F21851C2F2000101F1040100EB80003D
:206C80004FEA800008440068804703E0C8696FF34100C861BFF34F8F01B000BD00B581B0FC
:206CA00001464FEA81014FF21802C0F201021144096802464FEA82024FF20803C0F20103F5
:206CC0001A441268136A4FF0100202EA0302F2B141F21852C2F2000202F1100300EB8002B4
:206CE0004FEA82021A4412686AB141F21851C2F2000101F1100100EB80004FEA8000084420
:206D00000068804703E0C8696FF30410C861BFF34F8F01B000BD00B581B001464FEA8101AB
:206D20004FF21802C0F201021144096802464FEA82024FF20803C0F201031A441268136A21
:206D4000CA6A02F001024FF0040202EA0302F2B141F21852C2F2000202F1080300EB800273
:206D60004FEA82021A4412686AB141F21851C2F2000101F1080100EB80004FEA80000844A7
:206D80000068804703E0C8696FF38200C861BFF34F8F01B000BD00B581B001464FEA8101BD
:206DA0004FF21802C0F201021144096802464FEA82024FF20803C0F201031A441268136AA1
:206DC0008A6A02F001024FF0080202EA0302F2B141F21852C2F2000202F10C0300EB80022B
:206DE0004FEA82021A4412686AB141F21851C2F2000101F10C0100EB80004FEA8000084423
:206E00000068804703E0C8696FF3C300C861BFF34F8F01B000BD00B581B04FF00000FFF7C8
:206E2000C4FE01B000BD00B581B04FF00000FFF7F5FE01B000BD00B581B04FF00000FFF78B
:206E40002DFF01B000BD00B581B04FF00000FFF762FF01B000BD00B581B04FF00000FFF793
:206E60009AFF01B000BD00B581B04FF00100FFF79CFE01B000BD00B581B04FF00100FFF7CB
:206E8000CDFE01B000BD00B581B04FF00100FFF705FF01B000BD00B581B04FF00100FFF70F
:206EA0003AFF01B000BD00B581B04FF00100FFF772FF01B000BD00B581B04FF00200FFF713
:206EC00074FE01B000BD00B581B04FF00200FFF7A5FE01B000BD00B581B04FF00200FFF787
:206EE000DDFE01B000BD00B581B04FF00200FFF712FF01B000BD00B581B04FF00200FFF790
:206F00004AFF01B000BD00B581B04FF00300FFF74CFE01B000BD00B581B04FF00300FFF7C6
:206F20007DFE01B000BD00B581B04FF00300FFF7B5FE01B000BD00B581B04FF00300FFF70B
:206F4000EAFE01B000BD00B581B04FF00300FFF722FF01B000BD10B402464FEA820210460F
:206F60004FF21802C0F2010210440268002957D0087813686FF3555300F001044FEA445428
:206F800043EA04031360C868D3686FF30F034FF6FF7400EA040043EA0003D3604868A0F121
:206FA000010013686FF3144300F01F044FEA044443EA04031360087A13686FF3861300F079
:206FC00001044FEA841443EA04031360487A13686FF3C71300F001044FEAC41443EA040381
:206FE0001360887A13686FF3092300F003044FEA042443EA04031360086913696FF30103C1
:2070000000F0030043EA00031361486911696FF3114100F003034FEA034341EA03011161E4
:2070200010BC704701464FEA810108464FF21801C0F2010108440268916841F0010191609C
:20704000704701464FEA810108464FF21801C0F201010844026891686FF300019160704761
:2070600010B402464FEA820210464FF21802C0F2010210440468A2686FF3114201F003036B
:207080004FEA034342EA0302A26010BC704702464FEA820210464FF20802C0F2010210440C
:2070A00002681166704701464FEA810108464FF20801C0F2010108440168086E70470246C0
:2070C0004FEA820210464FF20802C0F20102104402684FF0010000FA01F0926900EA0200CD
:2070E00020FA01F1C8B270472DE9104181B04EF20808C4F20708D8F8004041F28858C2F2CF
:207100000008D8F8000004EA00044EF20808C4F20708C8F800404FF0040000EA0400E0B1CE
:2071200041F26858C2F20008D8F8000038B141F26858C2F20008D8F8000080470DE04EF274
:207140001C08C4F20708D8F800006FF382004EF21C08C4F20708C8F800004FF0200000EA60
:207160000400F0B141F26850C2F2000000F10400006840B141F26850C2F2000000F10400E9
:20718000006880470DE04EF21C08C4F20708D8F800006FF345104EF21C08C4F20708C8F83A
:2071A00000004FF0400000EA0400F0B141F26850C2F2000000F10800006840B141F26850E5
:2071C000C2F2000000F10800006880470DE04EF21C08C4F20708D8F800006FF386104EF2B5
:2071E0001C08C4F20708C8F800004FF4007000EA0400F0B141F26850C2F2000000F10C0008
:20720000006840B141F26850C2F2000000F10C00006880470DE04EF21C08C4F20708D8F864
:2072200000006FF349204EF21C08C4F20708C8F800004FF4806000EA0400F0B141F26850FD
:20724000C2F2000000F11000006840B141F26850C2F2000000F11000006880470DE04EF224
:207260001C08C4F20708D8F800006FF38A204EF21C08C4F20708C8F800004FF4805000EA63
:20728000040060B341F26850C2F2000000F11400006840B141F26850C2F2000000F1140036
:2072A000006880470DE04EF21C08C4F20708D8F800006FF30C304EF21C08C4F20708C8F832
:2072C00000004EF20808C4F20708D8F8000040F480504EF20808C4F20708C8F800004FF4AD
:2072E000005000EA040060B341F26850C2F2000000F11800006840B141F26850C2F200009D
:2073000000F11800006880470DE04EF21C08C4F20708D8F800006FF34D304EF21C08C4F256
:207320000708C8F800004EF20808C4F20708D8F8000040F400504EF20808C4F20708C8F840
:2073400000004FF4004000EA0400F0B141F26850C2F2000000F11C00006840B141F268502B
:20736000C2F2000000F11C00006880470DE04EF21C08C4F20708D8F800006FF3CF304EF296
:207380001C08C4F20708C8F80000BFF34F8F01B0BDE8108110B54FF0000452E020464FEAF4
:2073A000800040F22401C4F20401084400684FEA00404FEAD07021464FEA810140F224021B
:2073C000C4F20402114409684FEA81414FEAD17100EA010021464FEA810140F22402C4F29A
:2073E000040201EB020319686FF3CF3100F001024FEAC23241EA0201196000B320464FEA9A
:20740000800041F28C51C2F200010844006850B120464FEA800041F28C51C2F20001084442
:20742000006880470BE020464FEA800040F22401C4F20401014408686FF34D30086004F110
:207440000104042CAAD3BFF34F8F10BD00B581B0FFF7A0FF01B000BD084403464FEA8303E0
:20746000184641F28C51C2F2000108440260704710B402464FEA820240F22403C4F20403A5
:2074800002EB03040B7822686FF38A2203F001034FEA832342EA030222600A78002A55D182
:2074A00002464FEA820240F21403C4F204031A444B68136002464FEA820240F22403C4F229
:2074C000040302EB03040B7A22686FF3CB2203F001034FEAC32342EA0302226002464FEA09
:2074E000820240F22403C4F2040313444C7A1A686FF3010204F0030442EA04021A600246FF
:207500004FEA820240F22403C4F2040302EB03044B7B22686FF3861203F001034FEA831394
:2075200042EA030222604FEA800040F22402C4F204020244097B10686FF3850001F00F01A1
:207540004FEA810140EA010010607CE002464FEA820240F21403C4F204031A444B681360EA
:2075600002464FEA820240F22403C4F2040302EB03040B7A22686FF3CB2203F001034FEA6E
:20758000C32342EA0302226002464FEA820240F22403C4F2040313444C7A1A686FF3010233
:2075A00004F0030442EA04021A6002464FEA820240F22403C4F2040302EB03048B7A226886
:2075C0006FF3092203F003034FEA032342EA0302226002464FEA820240F22403C4F20403F8
:2075E00002EB0304CB7A22686FF3C71203F001034FEAC31342EA0302226002464FEA8202CF
:2076000040F22403C4F2040302EB03044B7B22686FF3861203F001034FEA831342EA03021F
:2076200022604FEA800040F22402C4F204020244097B10686FF3850001F00F014FEA810116
:2076400040EA0100106010BC704701464FEA8101084640F22401C4F2040100EB0102116843
:2076600041F480411160704701464FEA8101084640F22401C4F2040100EB010211686FF3C1
:207680008E311160704710B402464FEA8202104640F22402C4F2040200EB020422686FF3F3
:2076A0004D3201F001034FEA433342EA0302226010BC704701464FEA910001464FEA81015E
:2076C000084640F66821C2F2000108440168086810F0004F02D04FF0B64008600A686FF331
:2076E00055520A600A6842F400120A600A6842F000420A60704701464FEA910001464FEABD
:207700008101084640F66821C2F2000108440168086810F0004F02D04FF0B64008600A68D0
:207720006FF3010242F001020A600A6842F400120A600A6842F000420A60704701464FEA9A
:20774000910001464FEA8101084640F66821C2F2000108440168086810F0004F02D04FF04F
:20776000B64008600A686FF301020A600A686FF355520A600A6842F000420A60704700007E
:2077800070B5044620464FEA80004FF2B001C0F201010844056820464FEA80004FF2A801F3
:2077A000C0F2010108440068066906F03F06C16806EA010606614FF0010000EA0600D0B17F
:2077C000C4EBC4004FEA800041F29C51C2F200010844006858B1C4EBC4004FEA800041F28C
:2077E0009C51C2F2000108440068804703E0E8686FF30000E8604FF0020000EA0600F0B1BD
:2078000041F29C50C2F2000000F10401C4EBC4004FEA80000844006868B141F29C50C2F2D3
:20782000000000F10401C4EBC4004FEA800008440068804703E0E8686FF34100E8604FF04E
:20784000040000EA0600F0B141F29C50C2F2000000F10801C4EBC4004FEA800008440068E6
:2078600068B141F29C50C2F2000000F10801C4EBC4004FEA800008440068804703E0E86848
:207880006FF38200E8604FF0080000EA0600F0B141F29C50C2F2000000F10C01C4EBC400A0
:2078A0004FEA80000844006868B141F29C50C2F2000000F10C01C4EBC4004FEA80000844F9
:2078C0000068804703E0E8686FF3C300E8604FF0100000EA0600F0B141F29C50C2F2000026
:2078E00000F11001C4EBC4004FEA80000844006868B141F29C50C2F2000000F11001C4EB09
:20790000C4004FEA800008440068804703E0E8686FF30410E8604FF0200000EA0600F0B18E
:2079200041F29C50C2F2000000F11401C4EBC4004FEA80000844006868B141F29C50C2F2A2
:20794000000000F11401C4EBC4004FEA800008440068804703E0E8686FF34510E860BFF396
:207960004F8F70BD10B501464FEA81014FF2B002C0F201021144096802464FEA82024FF281
:20798000A803C0F201031A44146840F23F12236902EA03024FF4807303EA020333B34FF25D
:2079A0008802C0F2010202F118021268226141F29C52C2F2000202F11803C0EBC0024FEAF3
:2079C00082021A4412686AB141F29C51C2F2000101F11801C0EBC0004FEA80000844006878
:2079E000804703E0C8686FF30820C860BFF34F8F10BD00B581B04FF00000FFF7C1FE01B013
:207A000000BD00B581B04FF00000FFF7ABFF01B000BD00B581B04FF00100FFF7B1FE01B0FA
:207A200000BD00B581B04FF00100FFF79BFF01B000BD000000000000000000000000000065
:207A40002DE9F04406464FF000044FF000054FF0000030464FEA80004FF2C801C0F20101DD
:207A60000844D0F800A030464FEA80004FF2B801C0F201010844076840F2FF35786905EA84
:207A800000054FF000044CE04FF0010000FA04F000EA0500002842D020464FEA80000AF101
:207AA00018010844006810F0100F38D020464FEA800007F11801084400686FF0200100EA84
:207AC000010021464FEA810107F11802114408604FF00B0016FB00F020444FEA800041F219
:207AE000D451C2F200010844006870B14FF00B0016FB00F020444FEA800041F2D451C2F263
:207B0000000108440068804709E020464FEA80000AF11801014408686FF30410086004F145
:207B20000104072CB0D9BFF34F8FBDE8F08410B54FF0000201464FEA81014FF2C802C0F216
:207B400001021144096802464FEA82024FF2B803C0F201031A441368DA6E6FF0100402EA25
:207B60000402DA6641F2D452C2F2000202F128034FF00B0210FB02F24FEA82021A441268B2
:207B80007AB141F2D451C2F2000101F128014FF00B0210FB02F04FEA800008440068804715
:207BA00003E0886E6FF386108866BFF34F8F10BD10B54FF0000201464FEA81014FF2C80296
:207BC000C0F201021144096802464FEA82024FF2B803C0F201031A4413685A696FF4007400
:207BE00002EA04025A6141F2D452C2F2000202F124034FF00B0210FB02F24FEA82021A4449
:207C000012687AB141F2D451C2F2000101F124014FF00B0210FB02F04FEA800008440068E5
:207C2000804703E008696FF349200861BFF34F8F10BD10B54FF0000201464FEA81014FF24F
:207C4000C802C0F201021144096802464FEA82024FF2B803C0F201031A4413685A696FF429
:207C6000807402EA04025A6141F2D452C2F2000202F120034FF00B0210FB02F24FEA820236
:207C80001A4412687AB141F2D451C2F2000101F120014FF00B0210FB02F04FEA8000084473
:207CA0000068804703E008696FF308200861BFF34F8F10BD00B581B04FF00000FFF7C0FE18
:207CC00001B000BD00B581B04FF00000FFF72FFF01B000BD00B581B04FF00000FFF768FFFD
:207CE00001B000BD00B581B04FF00000FFF7A1FF01B000BD00B581B04FF00100FFF7A0FE33
:207D000001B000BD00B581B04FF00100FFF70FFF01B000BD00B581B04FF00100FFF748FFFA
:207D200001B000BD00B581B04FF00100FFF781FF01B000BD00B581B04FF00200FFF780FE30
:207D400001B000BD00B581B04FF00200FFF7EFFE01B000BD00B581B04FF00200FFF728FFF9
:207D600001B000BD00B581B04FF00200FFF761FF01B000BD00B581B04FF00300FFF760FE2E
:207D800001B000BD00B581B04FF00300FFF7CFFE01B000BD00B581B04FF00300FFF708FFF7
:207DA00001B000BD00B581B04FF00300FFF741FF01B000BD00000000000000000000000089
:207DC0000000000000000000000000002DE9104181B04FF00F0444F25408C4F20308D8F896
:207DE000000004EA000444F25C08C4F20308D8F8000004EA000444F25808C4F20308C8F85D
:207E0000004004F00100E0B141F28468C2F20008D8F8000038B141F28468C2F20008D8F85D
:207E2000000080470DE044F25C08C4F20308D8F8000020F0010044F25C08C4F20308C8F837
:207E400000004FEA540000F00100F0B141F28460C2F2000000F10400006840B141F28460D3
:207E6000C2F2000000F10400006880470DE044F25C08C4F20308D8F8000020F0020044F2CA
:207E80005C08C4F20308C8F800004FEA940000F00100F0B141F28460C2F2000000F10800DA
:207EA000006840B141F28460C2F2000000F10800006880470DE044F25C08C4F20308D8F85E
:207EC000000020F0040044F25C08C4F20308C8F800004FEAD40000F00100F0B141F28460BD
:207EE000C2F2000000F10C00006840B141F28460C2F2000000F10C00006880470DE044F25E
:207F00005C08C4F20308D8F8000020F0080044F25C08C4F20308C8F80000BFF34F8F01B0F8
:207F2000BDE8108100000000000030B581B0054642F20004C4F2050472B607B41A481B490A
:207F40001B4A0160026007BC62B6E56042F20002C4F205024FF000014FF0000007E0B1F5DA
:207F6000801F02D34FF0010005E001F10101936813F0807FF3D001B030BD00000000000016
:207F80002DE9004141F29468C2F20008D8F8000030B141F29468C2F20008D8F8000080476C
:207FA000BFF34F8FBDE8008114200540C4A1D9B00F3B1E1A00B583B04FF071008DF8040001
:207FC00001A800F101004FF00101017001A800F102004FF0FF01017001A800F103004FF02C
:207FE0000101017001F032F8012806D101A84FF0040101F0A8FE01F03EF803B000BD4DF893
:20800000048D4FF0000047F6F478C0F20208D8F800104AF65522CAF65522914201D14FF079
:2080200001005DF8048B70472DE9104181B04FF48028D8F800104FF00418D8F800404FF493
:2080400080204EF60858CEF20008C8F80000084680F30888084680F30988BFF34F8FA0473A
:20806000FEE700B581B04FF004014FF06400FCF760FA4FF000014FF06400FCF72EF94FF0C5
:208080006400FFF717FB4FF06400FFF734FB4FF004014FF0B400FCF74CFA4FF004014FF0B9
:2080A000C000FCF746FA4FF0B400FFF724FB4FF0C000FFF720FB4FF002024FF000014FF0F3
:2080C0000400FDF7F5F84FF002024FF001014FF00400FDF7EDF84FF002024FF002014FF057
:2080E0000400FDF7E5F84FF004024FF005014FF00100FDF7DDF84FF23C11C0F201014FF097
:208100000000FEF728FF4FF001014FF00000FEF7A7FF4FF00000FEF785FF01B000BD00B54D
:2081200081B04FF06400FFF7C5FA4FF00000FEF788FF4FF06400FFF701FB01B000BD00B543
:2081400081B04FF004014FF0B000FCF7F2F94FF000014FF0B000FCF7C0F84FF0B000FFF71E
:20816000CAFA4FF0D000FFF7C6FA4FF003024FF00D014FF00000FDF79BF84FF003024FF09C
:208180000C014FF00000FDF793F801B000BD00B581B04FF0B000FFF78DFA4FF0D000FFF74F
:2081A00089FA4FF0B000FFF7C9FA4FF0D000FFF7C5FA01B000BD2DE9004141F29868C2F224
:2081C0000008D8F800003C2808D241F29861C2F20001086800F10100086007E04FF00000B8
:2081E00041F29868C2F20008C8F8000041F29868C2F20008D8F800104FF01400B1FBF0F022
:208200004FF0140808FB00F0A1EB000008B900F020FBBDE800812DE9004100F0F1FC41F22B
:208220009C68C2F20008D8F80000B0F5FA6F08D241F29C61C2F20001086800F10100086017
:2082400007E04FF0000041F29C68C2F20008C8F80000BDE8008100B581B047F20010C0F23E
:208260000200FDF797FC10B14FF0010001E04FF0000001B000BD2DE900414FF000004EF210
:208280001408CEF20008C8F800004FF000004EF21808CEF20008C8F800004FF000004EF294
:2082A0001008CEF20008C8F800004FF000014FF0FF30FDF751FCBDE800812DE900414FF073
:2082C000000042F20808C4F20508D8F8001040F27132C0F2070201EA020140F24102C0F212
:2082E0000402914237D04AF2C411CBF2D90142F21408C4F20508C8F8001043F60F31C1F6E3
:208300001E2142F21408C4F20508C8F8001040F24101C0F2040142F20808C4F20508C8F849
:20832000001047F20071C0F2010142F20C08C4F20508C8F8001004E0B0F5801F12D200F1F7
:20834000010042F20808C4F20508D8F8001011F0807FF1D006E047F20070C0F20100FFF73C
:20836000E4FD002800F075FABDE8008100B581B04FF6FF70C0F20100FFF7D7FD002800F040
:2083800068FA01B000BD10B54FF000044FF000014FF08500FBF7A1FF4FF000014FF086006A
:2083A000FBF79BFF4FF001014FF08700FBF795FF4FF000024FF001014FF00100FBF73BFDB8
:2083C00018B14FF00104204636E040F64830C2F20000FBF791FE4FF00100FBF7A2FC4FF022
:2083E0000300FBF7C6FD0028F9D14FF0A000FFF7A5F94FF004014FF0A000FCF79AF84FF079
:2084000001014FF0A000FBF768FF4FF0A000FFF772F94FF004014FF03000FCF78AF8012891
:2084200003D14FF00104204606E04FF000014FF03000FBF752FF204610BD00B581B04FF08E
:208440000100FBF728FC4FF00100FBF792FD88B94FF001014FF08500FBF73FFF4FF001018D
:208460004FF08600FBF739FF4FF003014FF08700FBF733FF4FF000014FF03000FCF759F8ED
:20848000002801B000BD00B581B04FF004014FF00800FCF74EF84FF000014FF00800FBF723
:2084A0001CFF4FF00800FFF726F94FF0B500FDF726FB4FF22C11C0F201014FF00000FEF7D6
:2084C000D7FF48F2B712C0F201024FF000014FF00000FEF7C1FF4FF001014FF00000FFF764
:2084E000D2F84FF00000FFF7B0F801B000BD00B581B04FF00000FFF7B7F84FF000014FF01E
:208500000000FFF7C0F84FF00800FFF717F94FF0B500FDF707FB01B000BD00B581B0FFF72C
:20852000A0FD01B000BD00B581B0FFF7F8FD01B000BD00B581B04FF09400FFF7BBF84FF050
:208540009400FFF7FBF801B000BD00B581B0FFF7B4FEFFF718FFFFF77EFEFFF794FF00F0AA
:20856000B0F9FFF7ECFD00F062F9FFF7D6FF02F0D5FA00F0F6FC06F0F9F800F000FDFFF7F0
:2085800019FD01B000BD00B581B0FFF700FE4FF0C800FFF7D3F8FFF7CCFF00F070FAFFF7A4
:2085A0006AFEFFF74AFFFFF7E1FEFFF7A0FFFFF7BAFF01B000BD2DE9104181B04FF00004B2
:2085C0004FF0000041F20078C2F2000888F800004FF0C800FFF78FF8FFF7B7FF40F6841873
:2085E000C2F20008D8F8000045F2AA51C5F2AA51884217D0FFF703FD012813D105E001F081
:2086000083FF042801D14FF0010441F20078C2F2000898F800001428F1D91CB9FFF7B3FF1C
:20862000FFF702FD00F010FCFCE72DE9004182B04FF0000000904FF00000019001A96846E6
:2086400000F02AF9009841F2A068C2F20008C8F8000041F2A068C2F20008D8F80010086871
:20866000009A1044086041F2A068C2F20008D8F800104868009A1044486041F2A068C2F298
:208680000008D8F800108868009A1044886041F2A068C2F20008D8F80010C868009A104437
:2086A000C86002B0BDE800812DE9104181B0044672B641F2A068C2F20008D8F8000002687F
:2086C00041F2A861C2F2000120469047044662B6204601B0BDE810812DE9F04585B00446F3
:2086E0004FF00005174602F00F0010B14FF0010550E04FEA11104FEA0010064601F00F0AA9
:2087000072B6AEB141F2A068C2F20008D8F80000D0F808C041F2A868C2F20008D8F8043078
:20872000224631463846E047012801D14FF001057DBB3744BAF1000F2BD04FF0000010E0DE
:20874000504507D26946014400EB0602224412780A7004E0694601444FF0FF020A7000F1D7
:2087600001001028ECD341F2A068C2F20008D8F80000846841F2A868C2F20008D8F804304B
:208780006A4638464FF01001A047012801D14FF0010562B6284605B0BDE8F0854FF000029E
:2087A000002811D3B0F5001F0ED201EB0003A3F10103002B08D301EB0003A3F10103B3F54D
:2087C000001F01D24FF00102B0F1807F12D3B0F1817F0FD201EB0003A3F10103B3F1807F34
:2087E00008D301EB0003A3F10103B3F1817F01D24FF00102B0F1007F17D347F6FF73C0F2F3
:208800000023984211D801EB0003A3F10103B3F1007F0AD30844A0F1010047F6FF71C0F2AE
:208820000021884201D84FF00102104670474DF8048D4FF0000040F20008C4F20208D8F846
:20884000001011F0010F01D04FF001005DF8048B70472DE9104181B0EFF310800446002CCB
:2088600000D172B64BF2D610CAF2C40042F21408C4F20508C8F8000040F67B40C1F60D6074
:2088800042F21408C4F20508C8F80000002C00D162B601B0BDE810814DF8048D4FF2541886
:2088A000C0F20108D8F8002002604FF25418C0F20108D8F8040008604FF001005DF8048BE3
:2088C00070472DE9304192B04FF000044FF0000504AA4FF25C15C0F201050BCD0BC20BCDFC
:2088E0000BC20BCD0BC20BCD0BC295E8030082E803004FF03000FEF7DDFE4FF03000FEF7D1
:20890000FAFE40F60408C2F20008B8F8000040F2011188420CD140F60608C2F20008B8F816
:2089200000004FF6FE61884202D140F2737518E040F60408C2F20008B8F8000040F20221E1
:2089400088420CD140F60608C2F20008B8F800004FF6FD51884202D140F2747501E040F262
:20896000737504A94FF00100F9F720FC10B14FF0010480E02B464FF000024FF000014FF080
:208980000100FAF7A8F8012801D14FF0010440F2DF734FF000024FF002014FF00100FAF7CE
:2089A0009AF8012801D14FF0010448F6B322C0F201024FF000014FF00100FAF79DF94FF0D8
:2089C000000002904FF0000001904FF0000000904FF000034FF001024FF010014FF0010052
:2089E000FAF7A9F94FF0000002904FF0000001904FF0000000904FF000034FF000024FF0B2
:208A00000A014FF00100FAF796F94FF0000002904FF0000001904FF0000000904FF00003D9
:208A20004FF000024FF00B014FF00100FAF783F94FF000024FF000014FF00100FAF752FCFD
:208A4000012801D14FF001044FF000024FF002014FF00100FAF746FC012801D14FF00104A2
:208A60004CB94FF001014FF04B00FDF775F84FF04B00FDF744F8204612B0BDE8308100B5D8
:208A800081B04FF00100F9F752FD4FF000014FF04B00FDF761F84FF04B00FDF743F84FF017
:208AA0003000FEF707FE4FF03000FEF747FE01B000BD2DE9004184B008B1022809D141F2FA
:208AC000B462C2F2000201464FF00100FAF736F80028684600F00FF8684601F01FF94FF061
:208AE000010041F2B068C2F2000888F8000004B0BDE80081FEE72DE9004141F2B468C2F2D5
:208B0000000898F84810016041F2B468C2F20008D8F80410C160026841F2B461C2F200018D
:208B200001F1080100F1040005F05BFFBDE800812DE9304184B004464FF002024FF0000544
:208B40004FF000008DF80800082902D94FF0080000E008468DF809004FF000008DF80A006C
:208B60004FF000008DF80B004FF000008DF80C004FF000008DF80D0040F60408C2F2000887
:208B8000B8F8000040F2011188420CD140F60608C2F20008B8F800004FF6FE61884202D149
:208BA00040F27B7523E040F60408C2F20008B8F8000040F2022188420CD140F60608C2F2EE
:208BC0000008B8F800004FF6FD51884202D140F27C750CE040F27B7509E000942B4602AAE2
:208BE0004FF001014FF00100F9F72EFF0246022AF3D0012A01D1FFF77DFF04B0BDE8308127
:208C00004DF8048D41F20271C2F20001088800F1010080B2088041F20471C2F200010888FA
:208C200000F1010080B2088041F20671C2F20001088800F1010080B208804FF0010041F27A
:208C40000B78C2F2000888F8000041F20078C2F2000898F80000142809D841F20071C2F2E9
:208C60000001087800F10100C0B2087007E04FF0640041F20078C2F2000888F8000041F2F3
:208C80000278C2F20008B8F8000000F0010038B94FF0010041F20978C2F2000888F80000DC
:208CA00041F20278C2F20008B8F800104FF0050091FBF0F000EB8000A1EB000038B94FF0B4
:208CC000010041F20878C2F2000888F8000041F20278C2F20008B8F8000000F101014FF059
:208CE0000A0091FBF0F04FF00A0808FB00F0A1EB000038B94FF0010041F20A78C2F200088C
:208D000088F8000041F20278C2F20008B8F8000000F102014FF0640091FBF0F04FF064080C
:208D200008FB00F0A1EB000038B94FF0010041F20C78C2F2000888F8000041F20278C2F22F
:208D40000008B8F80000662807D34FF0000041F20278C2F20008A8F8000041F20478C2F248
:208D60000008B8F800004FF6FF6188420ED341F20478C2F20008B8F800004FEA201080B235
:208D800041F20478C2F20008A8F8000041F20678C2F20008B8F800104FF4FA7091FBF0F082
:208DA0004FF4FA7808FB00F0A1EB000038B94FF0010041F20D78C2F2000888F8000041F227
:208DC0000678C2F20008B8F80000B0F5FA7F07D34FF0000041F20678C2F20008A8F8000065
:208DE0005DF8048B70474DF8048D41F20478C2F20008B8F800005DF8048B70474DF8048D76
:208E000041F20478C2F20008B8F80010B1F57E4F0FD341F20478C2F20008B8F800004FEA7E
:208E2000201080B241F20478C2F20008A8F8000007E041F20472C2F200021188014488B267
:208E400010805DF8048B70472DE9004141F20B78C2F2000898F8000068B100F0C7FD05F0CC
:208E600062FB05F0EFF94FF0000041F20B78C2F2000888F8000041F20978C2F2000898F887
:208E8000000038B14FF0000041F20978C2F2000888F8000041F20878C2F2000898F80000BB
:208EA00070B101F098FE08B101F06EFC01F03BFD4FF0000041F20878C2F2000888F800009F
:208EC00041F20A78C2F2000898F8000098B14FF0030002F08CFB08B102F034FB01F086FE3E
:208EE00008B101F0F1FC4FF0000041F20A78C2F2000888F8000041F20C78C2F2000898F8A8
:208F00000000D8B103F0D9FF012805D14FF0000003F0C8FF03F071FC03F0E5FF012805D1CF
:208F20004FF0000003F0D4FF03F01DFD4FF0000041F20C78C2F2000888F8000041F20D7835
:208F4000C2F2000898F8000048B105F0EAFC4FF0000041F20D78C2F2000888F80000BDE819
:208F6000008100B581B04FF09400FEF7C4FB4FF29410C0F20100FBF765FE01B000BD30B5C3
:208F800081B04FF000044FF000004FF6FF7340F65440C2F200004FF001024FF07801FBF7FD
:208FA000F2FE4DF6E911884201D14FF001044FF000054FF0000040F65431C2F200014FF46E
:208FC000807000F014F805464FF6FF7340F65430C2F200004FF001024FF48071FBF7D3FEFC
:208FE000854201D14FF00104204601B030BD70B44FF6FF724FF0000323E003EB01042478E2
:209000004FEA0424A4B24FF0000515E084EA020606F400463EB14FEA420241F2210682EA78
:20902000060292B202E04FEA420292B24FEA4404A4B205F10105ADB2082DE7D303F1010328
:209040009BB28342D9D3104670BC704700B583B001A94FF00100FDF711FB01984AF6CC2181
:20906000CAF6CC21884202D14FF0010001E04FF0000003B000BD00B583B04FF0000001901E
:2090800001A94FF00100FDF7E1FA012802D14FF0010001E04FF0000003B000BD2DE9F00144
:2090A00040F20002C1F6FE726FF060454FF0005340F2FF76C2F2000640F60004C2F200046C
:2090C00040F68F17C2F2000740F69010C2F200004FF6FF71C2F2010105E04FF0000CC2F81A
:2090E00000C002F10402AA42F7D304E04FF000021A6003F10403B342F8D34EF20808C4F2A1
:209100000708D8F8002012F4806F0DD104E04FF00002226004F10404BC42F8D304E04FF0ED
:209120000002026000F104008842F8D3BDE8F00170474DF8048D032822D238B94FF47A71E0
:2091400041F21478C2F20008C8F80010012808D141F21471C2F2000101F104014FF47A722F
:209160000A6002280CD141F21470C2F2000000F1080041F21078C2F2000898F800100160A2
:209180005DF8048B70474DF8048D032818D228B941F21478C2F20008C8F80010012806D11D
:2091A00041F21472C2F2000202F104021160022806D141F21470C2F2000000F10800016010
:2091C0005DF8048B704703280BD201464FEA8101084641F21471C2F2000108444FF00001A3
:2091E00001607047032802D34FF0000031E001464FEA810141F21472C2F2000211440968D0
:2092000011B94FF0000024E001464FEA810141F21472C2F200021144096801290CD14FEACA
:20922000800041F21471C2F2000108444FF0000101604FF0FF300CE04FEA800041F2147189
:20924000C2F2000101440868A0F1010008604FF001007047032802D34FF0000023E001462A
:209260004FEA810141F21472C2F200021144096800290CD94FEA800041F21471C2F20001CA
:2092800008444FF0000101604FF001000BE04FEA800041F21471C2F2000108444FF0000104
:2092A00001604FF0000070472DE9104181B04FF0000041F22678C2F2000888F800004FF034
:2092C000000041F22578C2F2000888F800004FF0000041F22478C2F2000888F800004FF0F9
:2092E000000041F22378C2F2000888F800004FF0000041F22278C2F2000888F800004FF0DD
:20930000000041F22178C2F2000888F800004FF0000041F22078C2F2000888F800004FF0C0
:20932000000405E02046FFF74EFF04F10100C4B2032CF7D301B0BDE810812DE9704181B057
:20934000082907D8037803F00F039BB21C464FF0010304E000F101031C784FF00203072CA7
:2093600037D8B4B341F22878C2F20008A8F800404FF000040CE041F23875C2F200052544D7
:2093800004EB0306064436782E7004F10104A4B2A1F10105AC42EEDBA1EB030080B241F2AC
:2093A0002A78C2F20008A8F8000041F22C78C2F20008D8F80440134641F22878C2F2000820
:2093C000B8F8001041F23870C2F200004FF00002A04701B0BDE870812DE93041027802F0DC
:2093E0000F0292B24FEA022292B2144600F10102127844EA020294B2082C02D24FF0FF30B1
:2094000057E040F6FF72944206D34FF0020000F0A3F96FF001004CE041F22878C2F20008D7
:20942000A8F800404FF000020CE041F23873C2F20003134402F1020505442D781D7002F1CB
:20944000010292B2A1F102039A42EEDBA1F1020080B241F22A78C2F20008A8F800004FF053
:20946000000000F079F94FF0000041F22178C2F2000888F800004FF0010041F22578C2F27F
:20948000000888F800004FF00000FFF752FE4FF0000041F22078C2F2000888F8000041F246
:2094A0002C78C2F20008D8F80010204688474FF00100BDE830812DE9F0410646A1F101007B
:2094C000C0B20546307800F00F00C0B207464FF000044FF00000FFF7BDFE002802DC4FF0F1
:2094E000FF30B4E041F22072C2F20002107800F10100C0B2107041F22078C2F2000898F8AB
:2095000000000F2807D94FF0000041F22078C2F2000888F8000041F22078C2F2000898F8D7
:209520000000B84217D041F22C78C2F20008D8F8044041F22A78C2F20008B8F8001041F21F
:209540003870C2F200004FF001034FF00402A0476FF001007BE04FF0000013E041F22A787E
:20956000C2F20008B8F80010014441F23872C2F20002114400F10102324412780A7000F1E3
:20958000010080B2A842E9D341F22A72C2F200021088284480B2108041F22A78C2F2000816
:2095A000B8F8000041F22878C2F20008B8F8001088421FD34FF0000041F22578C2F2000825
:2095C00088F8000041F22C78C2F20008D8F8044041F22878C2F20008B8F8001041F238703A
:2095E000C2F200004FF001034FF00002A0474FF000002CE0002C1CD941F22172C2F2000264
:20960000107800F10100C0B2107041F22178C2F2000898F80000A0420BD34FF0000000F0D7
:209620009BF84FF0000041F22178C2F2000888F800004FF0010041F22578C2F2000888F804
:2096400000004FF00000FFF774FD4FF00100BDE8F0812DE9704181B004461546207800F0E9
:209660000F00C0B206464FF00100FFF7F3FD002802DC4FF0FF306CE0022D02D14FF0FF30C7
:2096800067E04FF0000041F22478C2F2000888F80000032E0BD341F22C78C2F20008D8F8C7
:2096A00008204FF0050090476FF0010051E0022E0BD141F22C78C2F20008D8F808204FF000
:2096C000080090476FF0020043E0012E0ED14FF0010041F22478C2F2000888F800004FF08F
:2096E0000100FFF726FD4FF0010032E004F10100007842F23778C2F2000888F8000004F17C
:20970000020000787F280CD804F10200007800F10100C0B241F21078C2F2000888F800007A
:2097200007E04FF07F0041F21078C2F2000888F800004FF0000041F22378C2F2000888F844
:2097400000004FF001014FF00200FFF71CFD4FF0000001B0BDE870812DE9004182B04FF228
:20976000A018C0F20108D8F800104FF2A018C0F20108D8F804200091019200F00F0040F09B
:209780003000C0B28DF80000684600F101004FF000010170684600F102004FF000010170FF
:2097A00068464FF0080100F0FBFA02B0BDE800812DE9704183B04FF2B018C0F20108D8F868
:2097C00000204FF2B018C0F20108D8F80430009201934FF00802B9B3082935D2CBB203F01E
:2097E0000F03DBB28DF800304FF001044FF000030AE003EB04056E46354403EB00063678DF
:209800002E7003F101039BB28B42F2D301EB040081B24FF0000011E04FF2A813C0F20103CE
:2098200003441B78994206D84FF2A811C0F201010844027804E000F1010080B20828EBD32B
:209840001146684600F0ACFA03B0BDE870812DE9004182B04FF2B818C0F20108D8F80020DF
:209860004FF2B818C0F20108D8F8043000920193082902D3B1F5805F02D34FF0000033E040
:209880004FEA2122D2B202F00F0242F01002D2B28DF800206A4602F1010201F0FF01C9B246
:2098A00011704FF000020AE0694601F10201114402EB00031B780B7002F101018AB2062AA4
:2098C000F2D368464FF0080100F06AFA4FF0010041F22478C2F2000888F800004FF00100EE
:2098E000FFF727FC4FF0060002B0BDE800812DE9104183B00C464FF2C018C0F20108D8F8A2
:2099000000104FF2C018C0F20108D8F804300091019302F00F0141F02001C9B28DF80010D6
:209920004FF000010AE06A4602F101020A4401EB00031B78137001F1010189B2A1420CD214
:209940000729F0D309E0684600F1010008444FF00002027001F1010081B20729F3D36846C2
:209960004FF0080100F01CFA072C02D94FF0070000E0204603B0BDE810812DE9104181B07E
:209980000C46082C2FD3B4F5805F2CD24FF000010BE042F23C72C2F200020A4401EB0003B9
:2099A0001B78137001F1010189B2A142F1D34FF0000141F22278C2F2000888F800102146FB
:2099C000FFF745FFC0B2014642F23A78C2F20008A8F80010A4EB010080B242F23878C2F2E8
:2099E0000008A8F8000001B0BDE810812DE9104181B04FF00000FFF7F5FB002816DAFFF70D
:209A000053FC41F22C78C2F20008D8F8044041F22A78C2F20008B8F8001041F23870C2F270
:209A200000004FF001034FF00302A0474FF00100FFF7D8FB00280ADAFFF736FC41F22C78A4
:209A4000C2F20008D8F808104FF0020088474FF00200FFF7C7FB002880F2858041F22271F4
:209A6000C2F20001087800F10100C0B2087041F22278C2F2000898F800000F2807D94FF066
:209A8000000041F22278C2F2000888F8000041F22278C2F2000898F8002042F23878C2F2EC
:209AA0000008B8F8001042F23A78C2F20008B8F8000042F23C73C2F200031844FFF717FF8A
:209AC000C0B2014642F23A72C2F200021088084480B2108042F23872C2F200021088A0EBDA
:209AE000010080B2108042F23878C2F20008B8F80000002835D942F23778C2F2000898F8EE
:209B00000000002828D941F22371C2F20001087800F10100C0B2087041F22378C2F20008BA
:209B200098F8000042F23778C2F2000898F80010884204D24FF00200FFF7FBFA13E04FF058
:209B4000010041F22478C2F2000888F800004FF00100FFF7EEFA06E04FF00200FFF7E9FADB
:209B600001E0FFF7A1FB01B0BDE810812DE9F0410D46164610B94FF0010401E04FF0020462
:209B800028784FEA2010C0B20146491E06D33CD0891EC0F0818000F09F80BDE041F22678E2
:209BA000C2F2000898F80000022801D1012C08D041F22678C2F2000898F80000002840F0E3
:209BC000AB80FFF771FB41F22678C2F2000898F80000022813D141F22C78C2F20008D8F86A
:209BE0000470234641F22A78C2F20008B8F8001041F23870C2F200004FF00602B8472246FA
:209C000031462846FFF799FB86E041F22678C2F2000898F80000022807D041F22678C2F2CC
:209C2000000898F80000002876D1FFF73DFB41F22678C2F2000898F80000022814D141F290
:209C40002C78C2F20008D8F8044041F22A78C2F20008B8F8001041F23870C2F200004FF071
:209C600001034FF00602A04731462846FFF7B4FB002808DD4FF0020041F22678C2F200084D
:209C800088F8000048E04FF0000041F22678C2F2000888F800003FE041F22678C2F2000824
:209CA00098F80000022837D141F22578C2F2000898F8000080B331462846FFF7FCFB002899
:209CC0002ADCFFF7F1FA4FF0000041F22678C2F2000888F800001FE041F22678C2F20008C5
:209CE00098F80000012817D141F22478C2F2000898F8000080B1224631462846FFF7A9FC8F
:209D0000002809DAFFF7D0FA4FF0000041F22678C2F2000888F80000BDE8F08100B581B030
:209D2000C16840F2DF72914202D14FF0010301E04FF0000301780A4600F104011846FFF758
:209D400015FF01B000BD2DE9004189B1B1F5805F0ED2072902D8FFF72BFD09E04FF0010238
:209D600041F22678C2F2000888F80020FFF705FEBDE8008107B4009818B1019808B102988F
:209D800010B94FF0FF3009E041F22C72C2F2000200A80BC882E80B004FF0000003B0704783
:209DA00000B581B0FEF7C4FE01B000BD10B504464FF0010000F0B3FB4FF001014FF001002A
:209DC00001F039FCE07900F14000C0B2E07104F1070000F102004FF00001017004F1070074
:209DE00000F103004FF03201017004F1070000F104004FF00701017004F1070000F10500F1
:209E00004FF0D00101704FF00600A0804FF0000010BD10B504464FF0020000F080FB4FF056
:209E2000000000F0EEFEE07900F14000C0B2E07104F1070000F102004FF00001017004F164
:209E4000070000F103004FF03201017004F1070000F104004FF00701017004F1070000F18E
:209E600005004FF0D00101704FF00600A0804FF0000010BD10B504464FF0040000F04FFB5F
:209E80004FF0000000F0BDFEE07900F14000C0B2E07104F1070000F102004FF000010170EB
:209EA00004F1070000F103004FF03201017004F1070000F104004FF00701017004F107002A
:209EC00000F105004FF0D00101704FF00600A0804FF0000010BD10B504464FF001014FF00B
:209EE000010001F0A8FB4FF00200A080E07900F14000C0B2E0714FF0000010BD10B5044604
:209F00004FF0000004F1070000F1030001F0EAFC38B9E17901F14001C9B2E1714FF00B01A5
:209F2000A18010BD10B504464FF0000004F1070000F1030001F0F2FC38B9E17901F1400198
:209F4000C9B2E1714FF00E01A18010BD10B504464FF0000004F1070000F1030001F0FAFCD3
:209F600038B9E17901F14001C9B2E1714FF00501A18010BD10B504464FF0000004F1070019
:209F800000F1030001F0FFFC38B9E17901F14001C9B2E1714FF00F01A18010BD10B504464A
:209FA0004FF0000004F1070000F1030001F007FD38B9E17901F14001C9B2E1714FF00401EE
:209FC000A18010BD10B504464FF0000004F1070000F1030001F075FD38B9E17901F1400174
:209FE000C9B2E1714FF00601A18010BD4FF0000200F1070101F102010978032906D0022983
:20A0000004D0012902D04FF0310207E04FF002018180C17901F14001C9B2C17110467047AD
:20A020004FF0000200F1070101F102010978032906D0022904D0012902D04FF0310207E01A
:20A040004FF002018180C17901F14001C9B2C1711046704710B504464FF0000000F0D1FD8A
:20A06000E07900F14000C0B2E0714FF00200A0804FF0000010BDC17901F14001C9B2C1710C
:20A080004FF0020181804FF000007047C17901F14001C9B2C1714FF0020181804FF00000EB
:20A0A00070474FF000014FF0000111E00A464FEA8203A3EB02024FEA820240F6CC43C2F222
:20A0C00000031A441278904204D001F10101C9B20629EBD3062901D34FF0FF01084670474C
:20A0E00070B50E464FF0FF044FF0000506F10701002960D0FFF7D5FF044606F1070000F106
:20A10000010000784FEAE01000F00100C0B20146FF2C4ED0012913D121464FEA8100A0EBF0
:20A1200001014FEA8101084640F6CC41C2F200010844007920B14FF0010000F048FE03E02D
:20A140004FF0000000F043FE21464FEA8100A0EB01014FEA8101084640F6CC41C2F20001E0
:20A1600008444088B188884202D94FF0130522E021464FEA8100A0EB01014FEA81010846DD
:20A1800040F6CC41C2F200010844806898B121464FEA8100A0EB01014FEA8101084640F65D
:20A1A000CC41C2F200010844816830468847054601E04FF01105284670BD00B581B04FF022
:20A1C000000100F1070242B18288022A05D3C27901461046FFF784FF0146084601B000BD2F
:20A1E00010B44FF000034FF0000309E01C464FEA04140C442468A04204D003F10103DBB264
:20A200009342F3D3934201D34FF0FF03184610BC70472DE9F04C81B08B4614464FF0FF05E7
:20A220004FF000074FF000014FF00006BBF804A01A462146FFF7D4FF054600F065F9074686
:20A2400000F078F90146FF2D0BD140F68450C2F20000844202D14FF031064DE04FF01206FD
:20A260004AE028464FEA00102044C088504506D828464FEA001020440089504502D24FF092
:20A28000130639E028464FEA00102044007900EA0700B8B940F65450C2F20000844202D16F
:20A2A0004FF07E0628E040F63450C2F20000844205D040F61450C2F2000084421CD14FF08A
:20A2C000220619E028464FEA001020444079012804D1012902D04FF033060DE028464FEA83
:20A2E00000102044C06838B128464FEA00102044C168584688470646304601B0BDE8F08C94
:20A3000000B581B04FF000034FF0000100F107028AB100F1070101F10101097801F07F03BF
:20A3200040F65452C2F20002014618464FF00303FFF76FFF0146084601B000BD00B581B054
:20A340004FF000034FF0000100F107028AB100F1070101F10101097801F07F0340F6E452F9
:20A36000C2F20002014618464FF00103FFF751FF0146084601B000BD4FF000014FF0000176
:20A3800000F1070169B100F1070101F1010109784FEA012100F1070000F10200007841EA53
:20A3A00000014FF031010846704700B581B04FF000034FF0000100F107028AB100F1070190
:20A3C00001F10101097801F07F0340F63452C2F20002014618464FF00203FFF71AFF0146E4
:20A3E000084601B000BD00B581B04FF000034FF0000100F107028AB100F1070101F1010117
:20A40000097801F07F0340F6F452C2F20002014618464FF00103FFF7FCFE0146084601B0F8
:20A4200000BD00B581B04FF000034FF0000100F107028AB100F1070101F10101097801F063
:20A440007F0340F61452C2F20002014618464FF00203FFF7DEFE0146084601B000BD00006A
:20A46000000030B44FF000044FF000040FE023464FEA83052B444FEA83030B441B88834274
:20A4800002D14FF0000006E004F101039CB29442EDD34FF0010030BC7047884202D04FF029
:20A4A000010001E04FF00000704700000000F0B581B006460D4617464FF000004FF0000470
:20A4C00000F038F801464FF0000018E002464FEA82031A444FEA82022A44128896420BD101
:20A4E00079B94FEA800108444FEA80002844C07838B14FF0010404E000F10100C0B2B84258
:20A50000E4D3204601B0F0BD4DF8048D40F60468C2F2000898F800005DF8048B70474DF81C
:20A52000048D40F60468C2F2000888F800005DF8048B70474DF8048D43F24A78C2F2000888
:20A5400098F800005DF8048B70474DF8048D43F24A78C2F2000888F800005DF8048B70472C
:20A5600000004DF8048D43F25078C2F20008D8F800005DF8048B70474DF8048D43F250780E
:20A58000C2F20008C8F800005DF8048B70474DF8048D43F25478C2F20008D8F800005DF8EC
:20A5A000048B70474DF8048D43F25478C2F20008C8F800005DF8048B70474DF8048D43F25C
:20A5C0005878C2F2000898F800005DF8048B70474DF8048D43F25878C2F2000888F80000AD
:20A5E0005DF8048B70474DF8048D43F25C78C2F20008D8F800005DF8048B70474DF8048DE4
:20A6000043F25C78C2F20008C8F800005DF8048B70474DF8048D43F26078C2F2000898F8EB
:20A6200000005DF8048B70474DF8048D43F26078C2F2000888F800005DF8048B70474DF880
:20A64000048D43F26178C2F2000898F800005DF8048B70474DF8048D43F26178C2F20008D4
:20A6600088F800005DF8048B70474DF8048D40F60568C2F2000898F800005DF8048B70475F
:20A680004DF8048D40F60568C2F2000888F800005DF8048B70474DF8048D43F26278C2F2D1
:20A6A000000898F800005DF8048B70474DF8048D43F26278C2F2000888F800005DF8048B62
:20A6C00070474DF8048D43F26478C2F20008B8F800005DF8048B70474DF8048D43F26478EE
:20A6E000C2F20008A8F800005DF8048B70472DE9104181B0FFF7B9FF0446012C0FD14FF087
:20A70000FF334FF001024FF4E6114FF45030FAF73AFB43F24C78C2F20008A8F80000022C1F
:20A720000FD14FF0FF334FF001024FF400614FF00050FAF728FB43F24C78C2F20008A8F8EA
:20A7400000007CB94FF0FF334FF001024FF4C0314FF48020FAF717FB43F24C78C2F2000842
:20A76000A8F8000043F24C78C2F20008B8F8000001B0BDE810814FF000028088884201D207
:20A780004FF01302104670472DE9F0414FF00C074FF000044FF0000543F26C76C2F2000667
:20A7A0004FF000046FE020464FEA8001A1EB00004FEA800040F60861C2F20001084400788A
:20A7C000F17988425CD120464FEA8001A1EB00004FEA800040F60861C2F20001084441884A
:20A7E0003046FFF7C8FF054606F1070000F1010000784FEAE01000F00100C0B2002D44D1A5
:20A80000012816D120464FEA8001A1EB00004FEA800040F60861C2F200010844007940B1B9
:20A820004FF0010043F26678C2F2000888F8000007E04FF0000043F26678C2F2000888F814
:20A84000000020464FEA8001A1EB00004FEA800040F60861C2F2000108448068A8B120464C
:20A860004FEA8001A1EB00004FEA800040F60861C2F200010844816830468847054604E0DC
:20A8800004F10100C4B2BC428DD3BC4201D34FF0110555B943F26678C2F2000898F800203A
:20A8A000B188304600F06DFA03E02946304600F044FA4FF0000043F26778C2F2000888F80D
:20A8C00000002846BDE8F0812DE930414FF0000443F67C75C2F200052846FFF76EFC04462F
:20A8E000112C03D0122C01D0312C01D14FF0FF0454B943F26978C2F2000898F80020A98808
:20A90000284600F03EFA03E02146284600F015FA4FF0000043F26878C2F2000888F800005A
:20A920002046BDE8308100B581B043F23C70C2F2000000F03EFD43F23C70C2F2000000F12F
:20A94000040002F01CFA43F23C70C2F2000000F1060002F0F3FD43F23C70C2F2000000F1F7
:20A96000080002F03DFA43F23C70C2F2000000F10A0001F029FD43F23C70C2F2000000F179
:20A980000C0002F05EFA01B000BD4DF8048D4FF0000143F23C78C2F20008A8F800105DF833
:20A9A000048B70472DE9F04105460C4616461F464FF0000000F073F926B14FF0000000F00B
:20A9C00020F960E0012F2FD14FF0000043F26C78C2F20008C8F8000043F26C78C2F2000845
:20A9E000A8F804404FF0010043F26C78C2F2000888F806004FF000000BE043F27371C2F2E1
:20AA00000001014400EB050212780A7000F1010080B2A042F1D34FF0010043F26778C2F228
:20AA2000000888F800002EE04FF0000043F67C78C2F20008C8F8000043F67C78C2F20008AF
:20AA4000A8F804404FF0000043F67C78C2F2000888F806004FF000000BE043F68371C2F259
:20AA60000001014400EB050212780A7000F1010080B2A042F1D34FF0010043F26878C2F2C7
:20AA8000000888F80000BDE8F08100B581B04FF0000000F0B6F801B000BD2DE9004182B05E
:20AAA0004FF050008DF80000684600F101004FF002010170684600F102004FF000010170DD
:20AAC000684600F103004FF032010170684600F104004FF007010170684600F105004FF0B3
:20AAE000D001017040F68418C2F20008D8F8000045F2AA51C5F2AA5188420CD14FF00200EA
:20AB0000FFF70DFD4FF0000000F07BF868464FF00601FFF718F902B0BDE800812DE9004169
:20AB200084B04FF0000043F26778C2F2000888F800004FF0000043F26878C2F2000888F8C2
:20AB400000004FF0000043F26678C2F2000888F800004FF0000043F26978C2F2000888F8D6
:20AB600000004FF0000043F23C78C2F20008A8F804004FF0000043F23C78C2F20008A8F8C9
:20AB800006004FF0000043F23C78C2F20008A8F808004FF0000043F23C78C2F20008A8F89F
:20ABA0000A0001F016F9FFF778FF4AF68B10C0F2010001904AF6A510C0F2010002904AF685
:20ABC0008B20C0F20100039001A807C8FFF7D2F804B0BDE800814DF8048D43F26778C2F2D4
:20ABE000000898F800005DF8048B70474DF8048D43F26878C2F2000898F800005DF8048B07
:20AC000070474DF8048D0146062945D80FF20408D8E801F0040D161F28313A004FF47A7050
:20AC200043F23C78C2F20008A8F8000034E04FF0040043F23C78C2F2000888F802002BE046
:20AC40004FF0100043F23C78C2F20008A8F8040022E04FF4B47043F23C78C2F20008A8F8AE
:20AC6000060019E04FF4B47043F23C78C2F20008A8F8080010E04FF4FA6043F23C78C2F2F7
:20AC80000008A8F80A0007E04FF4B47043F23C78C2F20008A8F80C005DF8048B70474DF883
:20ACA000048D0146062945D80FF20408D8E801F0040D161F28313A004FF0000043F23C78B1
:20ACC000C2F20008A8F8000034E04FF0000043F23C78C2F2000888F802002BE04FF0000054
:20ACE00043F23C78C2F20008A8F8040022E04FF0000043F23C78C2F20008A8F8060019E086
:20AD00004FF0000043F23C78C2F20008A8F8080010E04FF0000043F23C78C2F20008A8F833
:20AD20000A0007E04FF0000043F23C78C2F20008A8F80C005DF8048B704730B581B0044697
:20AD40000D46782D03D04FF00000FFF75AFFFF2D15D004F1070000F10200057004F1070029
:20AD600000F10100E17901704FF07F00E0714FF00300A080A18804F10700FEF7E4FF01B0F7
:20AD800030BD70B504460D4616464FF00000FFF738FF26B9294604F10700FEF7D4FF70BDFD
:20ADA0004DF8048D40F60668C2F2000898F800005DF8048B70474DF8048D40F60668C2F204
:20ADC000000888F800005DF8048B704700004DF8048D43F26978C2F2000888F800005DF8D3
:20ADE000048B704799281AD84FF0000103464FF0010211E003F00F0002FB00F0C0B20844F1
:20AE0000C1B24FEA820002444FEA4202D0B2C2B24FEA2310C0B20346002BEBD801E04FF016
:20AE2000FF0108467047884202D04FF0010001E04FF0000070472DE9F04B84B083464FF0CD
:20AE400001004FF000054FF000044FF000064FF000070BF1070000F1010000784FEA002019
:20AE600080B206460BF1070000F10200007846EA000086B24FF0000410E020464FEA80012B
:20AE800008444FEA80004FF2C811C0F2010108440088864204D004F10100C4B2002CECD01B
:20AEA000012C65D020464FEA800108444FEA80004FF2C811C0F201010844D0F80C80D0F8D5
:20AEC0001090CDF80880CDF80C9020464FEA800108444FEA80004FF2C811C0F201010844E5
:20AEE000B0F80480ADF806804FF000004FF0000736E0029838440078133804D00F380CD090
:20AF000011381ED029E0BDF80610BBF80400FFF78AFF10B34FF013051FE0FFF7F5FA21468B
:20AF20004FEA810211444FEA81014FF2C812C0F201021144897801EA000070B94FF02205A5
:20AF40000BE04FF2C811C0F2010130464FF00102FFF7ADFA08B14FF0330507F10100C7B241
:20AF6000039800F0FF00874204D2002DC1D001E04FF03105284604B0BDE8F08B70B50546E2
:20AF80004FF001004FF000004FF000044FF0000605F1070000F1010000784FEA002080B2B8
:20AFA000064605F1070000F10200007846EA000086B22846FFF73FFFC0BB4FF0000433E002
:20AFC00021464FEA810211444FEA81014FF2C812C0F20102114409888E4222D120464FEA26
:20AFE000800108444FEA80004FF2C811C0F201010844816805F1070000F1030088472146A1
:20B000004FEA810211444FEA81014FF2C812C0F201021144C988A980E97901F14001C9B2B5
:20B02000E97104F10101CCB2002CC9D070BD70B584B004464FF000004FF0000008E001A99C
:20B04000014400EB040212780A7000F10100C0B20C28F4D32078FFF7C5FE064604F10100C4
:20B060000078FFF7BFFE054604F102000078FFF7B9FE632E05D80C2D03D815B11F2800D8D7
:20B0800010B94FF0310007E001A94FF0020002F02CFC08B14FF0720004B070BD2DE9F04BEF
:20B0A00084B007464FF001004FF000064FF0000407F1070000F10100007800F07F00C0B2FD
:20B0C00083464FF000044FE020464FEA800108444FEA80004FF2E011C0F201010844D0F816
:20B0E0000C80D0F81090CDF80880CDF80C9020464FEA800108444FEA80004FF2E011C0F2A5
:20B1000001010844B0F80480ADF806804FF000054FF000051EE002982844007812380AD062
:20B12000401E14D1BDF80610B888FFF7B6F970B14FF013060BE04FF2E011C0F20101584634
:20B140004FF00102FFF78DF908B14FF0120605F10100C5B2039800F0FF00854201D2002E61
:20B16000D9D004F10100C4B2002CADD0304604B0BDE8F08B30B581B004464FF000052046BD
:20B18000FFF78CFF054604F1070000F10100007800F07F00C0B22DB9001E03D14FF0000085
:20B1A000FFF72FFD3DB9E07900F14000C0B2E0714FF00200A080284601B030BD2DE9F04B6C
:20B1C00082B083464FF003004FF000054FF000044FF000064FF00007FFF796F907460BF152
:20B1E000070000F10100007800F07F00C0B24FF0000410E021464FEA810211444FEA810197
:20B200004FF2F812C0F2010211440988884204D004F10101CCB2032CECD3032C4DD0204695
:20B220004FEA800108444FEA80004FF2F811C0F201010844D0F80C80D0F81090CDF8008004
:20B24000CDF804904FF000062FE020464FEA800108444FEA80004FF2F811C0F201010844D2
:20B260008188009830440078133802D06B3808D018E0BBF80400FFF710F998B14FF013055B
:20B2800010E020464FEA800108444FEA80004FF2F811C0F201010844807800EA070008B9A5
:20B2A0004FF07E0506F10100C6B2019800F0FF00864204D2002DC8D001E04FF012052846CC
:20B2C00002B0BDE8F08B30B581B004464FF000052046FFF773FF054604F1070000F10100F1
:20B2E000007800F07F00C0B295B9401E10D303D0801E04D30AD00BE000F032F808E000F067
:20B3000040F84FF0010000F06BF801E000F045F81DBBE07900F14000C0B2E07104F1070033
:20B3200000F102004FF00001017004F1070000F103004FF03201017004F1070000F10400A5
:20B340004FF00701017004F1070000F105004FF0D00101704FF00600A080284601B030BD51
:20B3600010B5FFF7D1F804464FF00100FFF7D7F8022C05D14FF001014FF0030000F05BF92F
:20B3800010BD00B581B04FF00200FFF7C8F84FF00000FFF736FC01B000BD00B581B04FF009
:20B3A0000400FFF7BCF84FF00000FFF72AFC01B000BD00B581B0018881B10188A1F1010158
:20B3C00089B20180008848B9FFF79EF8012805D0FFF7C6FF4FF0000000F09CFD01B000BDAD
:20B3E0004DF8048D44F28C78C2F2000888F800005DF8048B70472DE9F04B84B083464FF0D9
:20B4000001004FF000054FF000040BF1070000F10100007800F07F00C0B207464FF00004C6
:20B4200089E020464FEA800108444FEA80004FF23C21C0F201010844D0F80C80D0F8109024
:20B44000CDF80880CDF80C9020464FEA800108444FEA80004FF23C21C0F201010844B0F8D3
:20B460000480ADF806804FF0000620464FEA800108444FEA80004FF23C21C0F20101084415
:20B4800000788DF805004FF000064AE0029830440078123810D0401E04D00F3819D01138E0
:20B4A00030D03BE0BDF80610BBF80400FEF7F5FFA0B34FF0130531E04FF23C21C0F20101F9
:20B4C00038464FF00102FEF7CCFF38B34FF0120524E09DF80580B84514D14FF00000FFF776
:20B4E00013F821464FEA810211444FEA81014FF23C22C0F201021144897801EA000008B9B8
:20B500004FF022054FF23C21C0F2010138464FF00102FEF7CCFF08B14FF0330506F10100CB
:20B52000C6B2039800F0FF00864201D2002DADD004F10100C4B2002C3FF473AF284604B0B5
:20B54000BDE8F08B2DE900414FF0000044F28D78C2F2000888F802004FF0FF3040F684187C
:20B56000C2F20008C8F80000F9F746FBBDE800812DE9304104464FF0000004F1070000F1FB
:20B580000100007800F07F00C0B205462046FFF732FF08BB2946491E1ED303D0891E0AD398
:20B5A00012D019E04FF0010144F28D78C2F2000888F8001010E04FF0010144F28D78C2F2C8
:20B5C000000888F8011007E04FF0010144F28D78C2F2000888F8021038B94FF00201A180CD
:20B5E000E17901F14001C9B2E171BDE830814DF8048D4FF000010246521E18D303D0921E5F
:20B6000008D30ED013E044F28D78C2F2000898F800100CE044F28D78C2F2000898F8011063
:20B6200005E044F28D78C2F2000898F8021008465DF8048B70474DF8048D0246521E18D32A
:20B6400003D0921E08D30ED013E044F28D78C2F2000888F800100CE044F28D78C2F2000851
:20B6600088F8011005E044F28D78C2F2000888F802105DF8048B70474FEA002101F0FF21C5
:20B680004FEA102000F0FF1040EA01004FEA30407047884202D04FF0010001E04FF00000BB
:20B6A0007047F0B581B005460C4616464FF00000FEF72AFF02464FF000014FF000001AE0E6
:20B6C00003464FEA83073B444FEA830323441B889D420DD103464FEA83052B444FEA830321
:20B6E00023449B7803EA02023AB94FF0010104E000F10100C0B2B042E2D3B04201D14FF0B9
:20B700000101084601B0F0BD2DE9F04B82B007464FF00A004FF000044FF000004FF000059C
:20B720004FF0000607F1070000F1010000784FEA002080B2054607F1070000F1020000781B
:20B7400045EA000085B24FF0000010E001464FEA810211444FEA81014FF25422C0F20102D5
:20B76000114409888D4204D000F10100C0B20A28ECD30A2857D001464FEA810211444FEA01
:20B7800081014FF25422C0F201021144D1F80C80D1F81090CDF80080CDF804904FEA800150
:20B7A00008444FEA80004FF25421C0F201010844B0F804B04FF000062DE00098304400789C
:20B7C000133804D00F380AD0113815D020E05946B888FFF75EFFD8B14FF0130418E04FF2B1
:20B7E0005421C0F2010128464FF00A02FFF759FF70B14FF022040BE04FF25421C0F201013E
:20B8000028464FF00A02FEF752FE08B14FF0330406F10100C6B2019800F0FF00864204D265
:20B82000002CCAD001E04FF03104204602B0BDE8F08B70B505464FF00A004FF000004FF07E
:20B8400000044FF0000605F1070000F1010000784FEA002080B2064605F1070000F1020071
:20B86000007846EA000086B22846FFF74DFFC0BB4FF0000433E021464FEA810211444FEAB6
:20B8800081014FF25422C0F20102114409888E4222D120464FEA800108444FEA80004FF2AB
:20B8A0005421C0F201010844816805F1070000F10300884721464FEA810211444FEA810137
:20B8C0004FF25422C0F201021144C988A980E97901F14001C9B2E97104F10101CCB20A2C18
:20B8E000C9D370BD10B5044621464FF0040002F0C2F801464FF0000007E000EB04024FF07D
:20B90000FF03137000F10100C0B20728F5D311B94FF0000001E04FF0220010BD10B5044620
:20B9200021464FF0040002F0A6F801464FF0000007E000EB04024FF0FF03137000F10100B9
:20B94000C0B20F28F5D311B94FF0000001E04FF0220010BD10B440F25452C0F204024FF0CB
:20B96000000109E001EB0003144602F1010224781C7001F10101C9B20F29F3D34FF00001C9
:20B98000084610BC704710B5044621464FF0040002F071F801464FF0000007E000EB040264
:20B9A0004FF0FF03137000F10100C0B21528F5D311B94FF0000001E04FF0220010BD10B47E
:20B9C00040F24052C0F204024FF0000109E001EB0003144602F1010224781C7001F1010167
:20B9E000C9B21429F3D34FF00001084610BC70472DE93041044643F6F478C0F20208D8F8B6
:20BA000000104FF000050846FFF736FE01464FEA116000F0FF00C0B2207004F101004FEA49
:20BA2000114202F0FF02D2B2027004F102004FEA112202F0FF02D2B2027004F1030001F095
:20BA4000FF01C9B201702846BDE8308110B5044621464FF0040002F00EF801464FF00000FF
:20BA600007E000EB04024FF0FF03137000F10100C0B21828F5D311B94FF0000001E04FF095
:20BA8000220010BD00B581B001464FF0020001F0F2FF014611B94FF0000101E04FF02201D3
:20BAA000084601B000BD10B50446FEF72DFD0146042901D14FF003014FF0000221701046EB
:20BAC00010BD2DE93041044643F6EF78C0F20208D8F800104FF000050846FFF7CDFD0146F3
:20BAE0004FEA116000F0FF00C0B2207004F101004FEA114202F0FF02D2B2027004F1020049
:20BB00004FEA112202F0FF02D2B2027004F1030001F0FF01C9B201702846BDE830812DE921
:20BB2000004182B04FF24838C0F20108D8F8001000914FF24C38C0F20108D8F800100191B3
:20BB4000012806D169464FF0030001F0CEFE014605E001A94FF0030001F0C7FE01460846D4
:20BB600002B0BDE800812DE9704183B0054644F29D78C2F2000898F8000001280DD14FF0CB
:20BB8000000407E001A820444FF00001017004F10100C4B2042CF5D33CE044F29C78C2F27E
:20BBA000000898F8000010BB4FF0000414E044F29E70C2F2000004EB000600F0D3F83070A3
:20BBC00001A8204444F29E71C2F2000121440978017004F10100C4B2042CE8D34FF0010070
:20BBE00044F29C78C2F2000888F8000012E04FF000040BE001A8204444F29E71C2F2000198
:20BC000021440978017004F10100C4B2042CF1D300F0F2FB4FF00600A880E87900F1400091
:20BC2000C0B2E87101A905F1070000F102004FF0040202F0D6FE03B0BDE870812DE90041F4
:20BC400082B044F29E78C2F2000898F800108DF8041001A901F1010144F29E72C2F20002D7
:20BC600002F1010212780A7001A901F1020144F29E72C2F2000202F1020212780A7001A98A
:20BC800001F1030144F29E72C2F2000202F1030212780A70024601A84FF000034FF004013F
:20BCA00000F067FB02B0BDE800812DE9104185B004464FF0000044F29C78C2F2000888F8AF
:20BCC00000006846FFF7BAFF02A9684600F063F804F1070000F10200014601A84FF004023F
:20BCE00002F07FFE03A901A800F055F802980399884232D144F2A278C2F2000898F80000A4
:20BD000040B144F2A271C2F200010878A0F10100C0B208704FF0000044F2A378C2F20008EC
:20BD200088F800004FF00000FFF7F9FE4FF0010044F29D78C2F2000888F800004FF0010050
:20BD4000FEF703FC4FF00200A080E07900F14000C0B2E0714FF0000001E000F04DFB05B034
:20BD6000BDE8108110B54FF00000FDF73CF802F032FE02F022FE01464FF0FF0091FBF0F03C
:20BD8000C0EB0020A1EB0000C0B204462046FDF735F8204610BDD8B1D1B14FF0000203780F
:20BDA0004FEA036342EA030200F101031B784FEA034342EA030200F102031B784FEA032393
:20BDC00042EA030200F10300007842EA00020A6070472DE9004182B04FF000000AE044F28F
:20BDE0009E71C2F2000101444FF000020A7000F10100C0B20428F2D34FF0000044F29C78A1
:20BE0000C2F2000888F8000040F60408C2F20008B8F8000040F2022188422CD140F60608D8
:20BE2000C2F20008B8F800004FF6FD51884222D14FF0C50040F69868C2F2000888F80000D0
:20BE400040F69860C2F2000000F101004FF04D01017040F69860C2F2000000F102004FF0FC
:20BE60008701017040F69860C2F2000000F103004FF0730101704FF0000044F29D78C2F291
:20BE8000000888F8000001A94FF0030001F0F3FD40B99DF8040044F2A378C2F2000888F82E
:20BEA000000007E04FF0000044F2A378C2F2000888F8000044F2A378C2F2000898F8000032
:20BEC000012814D14FF0030044F2A278C2F2000888F800004FF0010044F2A478C2F2000838
:20BEE00088F800004FF00500FEF78BFE0FE04FF0000044F2A478C2F2000888F800004FF005
:20BF0000000044F2A278C2F2000888F8000002B0BDE800814DF8048D44F29D78C2F20008E0
:20BF200088F800005DF8048B70472DE9F04B84B083464FF002004FF000054FF000040BF1D4
:20BF4000070000F1010007784FF0000410E020464FEA800108444FEA80004FF25031C0F29D
:20BF6000010108440088874204D004F10100C4B2022CECD3022C00F0838020464FEA8001B4
:20BF800008444FEA80004FF25031C0F201010844D0F80C80D0F81090CDF80880CDF80C9070
:20BFA00020464FEA800108444FEA80004FF25031C0F201010844B0F80480ADF806804FF004
:20BFC000000620464FEA800108444FEA80004FF25031C0F20101084400788DF805004FF033
:20BFE000000645E0029830440078133806D00F380ED0801E26D013382ED036E0BDF806108C
:20C00000BBF80400FEF749FA78B34FF013052CE09DF80580B84528D14FF00000FEF774FAF1
:20C0200021464FEA810211444FEA81014FF25032C0F201021144897801EA0000A8B94FF074
:20C04000220512E044F29C78C2F2000898F8000058B94FF0240508E044F2A478C2F20008C2
:20C0600098F8000008B14FF0370506F10100C6B2039800F0FF00864204D2002DB2D001E0D4
:20C080004FF01205284604B0BDE8F08B70B504464FF0000504F1070000F101000678204683
:20C0A000FFF743FF05466DB93046401E02D0401E04D007E02046FFF756FD03E02046FFF72A
:20C0C000F4FD0546284670BD2DE9100140F69868C2F2000898F80020037882EA0302D2B250
:20C0E0000A7001F1010200F1010340F69864C2F2000404F1010424781B7884EA0303DBB2C8
:20C10000137001F1020200F1020340F69864C2F2000404F1020424781B7884EA0303DBB29B
:20C12000137001F1030100F1030040F69862C2F2000202F103021278007882EA0000C0B2D4
:20C1400008704FF00100BDE81001704700F0AA314FEA510100F055304FEA400040EA01004B
:20C1600000F0CC314FEA910100F033304FEA800040EA010000F0F0314FEA111100F00F3035
:20C180004FEA001040EA010000F0FF214FEA112100F0FF104FEA002040EA01004FEA304084
:20C1A000704710B50C464FF000024FF0000301784FEA016142EA010200F1010109784FEA3E
:20C1C000014142EA010200F1020109784FEA012142EA010200F10300007842EA00021046FF
:20C1E000FFF7B4FF03464FEA136000F0FF00C0B2207004F101004FEA134101F0FF01C9B2C1
:20C20000017004F102004FEA132101F0FF01C9B2017004F1030003F0FF01C9B201704FF056
:20C22000010010BD2DE9100140F69868C2F2000898F80020037882EA0302D2B20A7001F18B
:20C24000010200F1010340F69864C2F2000404F1010424781B7884EA0303DBB2137001F15D
:20C26000020200F1020340F69864C2F2000404F1020424781B7884EA0303DBB2137001F13A
:20C28000030100F1030040F69862C2F2000202F103021278007882EA0000C0B208704FF031
:20C2A0000100BDE81001704770B44FF000034FF000064FF000044FF000044FF0000504781F
:20C2C0004FEA046443EA040300F1010424784FEA044443EA040300F1020424784FEA04244E
:20C2E00043EA040300F10300007843EA000308784FEA006046EA000601F1010000784FEA7B
:20C30000004046EA000601F1020000784FEA002046EA000601F10300007846EA000606EB18
:20C32000030000464FF0000104460D46204600F0FF344FEA146000F0FF00C0B2107002F1CD
:20C3400001004FEA144101F0FF01C9B2017002F102004FEA142101F0FF01C9B2017002F13E
:20C36000030004F0FF01C9B201704FF0010070BC704730B581B00446154644F29471C2F20D
:20C3800000012046FFF7A0FE44F29071C2F200012046FFF706FF44F29871C2F2000144F22B
:20C3A0009070C2F20000FFF73DFF2A4644F29871C2F2000144F29470C2F20000FFF774FFDC
:20C3C0004FF0010001B030BD4DF8048D018881B10188012908D14FF0000044F2A478C2F21D
:20C3E000000888F8000004E00188A1F1010189B201805DF8048B70472DE9004144F2A278B6
:20C40000C2F2000898F80000FF2808D244F2A271C2F20001087800F10100C0B2087044F23F
:20C42000A278C2F2000898F80000032821D34FF0010044F2A478C2F2000888F8000044F273
:20C44000A378C2F2000898F8000058B94FF00100FFF765FB4FF0010044F2A378C2F2000881
:20C4600088F800004FF00500FEF7CBFB4FF0360001E04FF03500BDE800812DE9F04B84B0C8
:20C4800083464FF002004FF000054FF000044FF000000BF1070000F10100007800F07F00F0
:20C4A000C0B207464FF0000410E020464FEA800108444FEA80004FF28031C0F20101084473
:20C4C0000088874204D004F10100C4B2022CECD3022C68D020464FEA800108444FEA800053
:20C4E0004FF28031C0F201010844D0F80C80D0F81090CDF80880CDF80C9020464FEA8001C0
:20C5000008444FEA80004FF28031C0F201010844B0F80480ADF806804FF0000620464FEAE9
:20C52000800108444FEA80004FF28031C0F20101084400788DF805004FF000062BE0029897
:20C5400030440078133802D00F380AD020E0BDF80610BBF80400FDF7A0FFC8B14FF01305CC
:20C5600016E09DF80580B84512D1FDF7CDFF21464FEA810211444FEA81014FF28032C0F233
:20C5800001021144897801EA000008B94FF0220506F10100C6B2039800F0FF00864204D298
:20C5A000002DCCD001E04FF01205284604B0BDE8F08B10B504464FF000002046FFF75DFF33
:20C5C00004F1070101F10101097801F07F01C9B20A4604F1070101F10201097810BB521EFF
:20C5E00001D310D01EE0A1F10101022908D8E17901F14001C9B2E1714FF00201A18011E03C
:20C600004FF031000EE0A1F10101022908D8E17901F14001C9B2E1714FF00201A18001E07F
:20C620004FF0310010BD4DF8048D03465B1E18D324D05B1E30D101290AD1012A08D14FF084
:20C64000010044F2A578C2F2000888F8000023E04FF0000044F2A578C2F2000888F8000079
:20C660001AE040F69C68C2F2000888F8011040F69C68C2F2000888F802200DE040F69C6082
:20C68000C2F2000000F10300417040F69C60C2F2000000F1030082705DF8048B70470128B1
:20C6A00002D04FF0010001E04FF000007047884202D04FF0010001E04FF0000070472DE9C8
:20C6C000704181B004460D461646FDF7E4FF06EA050111B94FF0010016E0B4F57F4F09D161
:20C6E00044F2A578C2F2000898F8001011B94FF0010009E040F202218C4203D110B94FF099
:20C70000010001E04FF0000001B0BDE87081F0B581B04FF000024FF000034FF000044FF0D6
:20C7200000054FF000014FF000064FF004024FF00403114612E000F1070707F1030701EBAE
:20C74000070CA2EB01074FEAC7079CF800C00CFA07F744EA0704A1F10101C9B20029EAD89F
:20C7600002EB0301C9B214E000F1070707F1030701EB070C02EB0307A7EB01074FEAC707C1
:20C780009CF800C00CFA07F745EA0705A1F10101C9B29142E8D82946204601F09CF90328DE
:20C7A00002D14FF0010613E0012808D1B4F5503F02D1B5F5E61F02D04FF0010608E038B9C0
:20C7C000B4F5802F02D1B5F5C03F01D04FF00106304601B0F0BD2DE900414FF0010144F2CC
:20C7E000A678C2F2000888F800104FF00400FEF708FA4FF07800BDE8008110B582B04FF082
:20C8000071008DF8040001A800F101004FF00101017001A800F102004FF00201017001A8D9
:20C8200000F103004FF002010170FDF71EFF044601A84FF00401FDF786FA4FF00000FEF761
:20C84000E0F920464FF001024FF00101FFF7EBFE022C07D1FBF7E9FE4FF001014FF00000D8
:20C8600001F067F84FF00400FEF719FA02B010BDC17901F14001C9B2C17100F1070000F19B
:20C8800004004FF0000101704FF000007047F0B585B004464FF2AC30C0F201006D460668D8
:20C8A0002E6046686E608668AE60C068E8604FF000054FF000000BE06E46064447F6F077F2
:20C8C000C0F2020707443F78377000F10100C0B21028F1D3012A00D00ABB684600F1040031
:20C8E0004FEA116202F0FF02D2B20270684600F105004FEA114202F0FF02D2B202706846DC
:20C9000000F106004FEA112202F0FF02D2B20270684600F1070001F0FF01C9B201701846EA
:20C92000FBF7C2FE08B14FF00105224668464FF01001FBF7D1FE08B14FF00105284605B0FF
:20C94000F0BD2DE900414FF0010144F2A778C2F2000888F800104FF00600FEF752F94FF02D
:20C960007800BDE8008110B582B04FF071008DF80000684600F101004FF0010101706846ED
:20C9800000F102004FF0FF010170684600F103004FF001010170FDF768FE044684BB45F286
:20C9A000AA51C5F2AA5147F6F070C0F202004FF418334FF00002FFF76AFF20464FF00002A4
:20C9C0004FF00001FFF72FFE4FF07F008DF805000DF1050000F101004FF0310101700DF1D7
:20C9E000050000F102004FF0780101700DF105004FF00301FDF7A7F9FBF7C5FDFBF714FB87
:20CA0000012C14D145F2AA51C5F2AA5147F6F070C0F202004FF418334FF00102FFF737FFD3
:20CA200020464FF000024FF00001FFF7FCFD68464FF00401FDF787F94FF00000FEF7E1F8AD
:20CA40004FF00600FEF72BF902B010BDF0B581B004464FF000014FF000054FF000024FF0D5
:20CA600000034FF000004FF000054FF004014FF00405084611E004F1070606F1030600EB78
:20CA80000607A1EB00064FEAC6063F7807FA06F642EA0602A0F10100C0B20028EBD801EB2F
:20CAA0000500C0B213E004F1070606F1030600EB060701EB0506A6EB00064FEAC6063F78C8
:20CAC00007FA06F643EA0603A0F10100C0B28842E9D8B2F5802F0ED1B3F5C03F0BD14FF09D
:20CAE0000000FEF768F94FF4C0314FF4802001F01BF8054613E0B2F5503F0ED1B3F5E61FC5
:20CB00000BD14FF00100FEF756F94FF4E6114FF4503001F009F8054601E04FF03105782D80
:20CB200004D14FF00200FEF76CF80CE05DB9E07900F14000C0B2E07104F1070000F1040046
:20CB40004FF000010170284601B0F0BD2DE9F04B84B007464FF004004FF000044FF00005BC
:20CB60004FF000064FF0000B07F1070000F1010090F800808DF805804FF000098DF80490C2
:20CB8000B888042802D24FF01304A5E007F1070000F1020000784FEA002080B2064607F141
:20CBA000070000F10300007846EA000086B24FF0000510E028464FEA800108444FEA800039
:20CBC0004FF2BC31C0F2010108440088864204D005F10100C5B2042DECD3042D7AD22846BA
:20CBE0004FEA800108444FEA80004FF2BC31C0F201010844D0F80C80D0F81090CDF808803F
:20CC0000CDF80C9028464FEA800108444FEA80004FF2BC31C0F201010844B0F80480ADF887
:20CC20000680FDF771FC8DF804004FF0000B49E0029858440078123814D0401E1AD00F38A6
:20CC400021D00F3834D0801E38D14FF2BC31C0F2010130464FF00402FDF729FC70B34FF0D9
:20CC600033042BE09DF80500FFF719FD30B34FF0120423E0BDF80610B888FFF718FDE8B1E2
:20CC80004FF013041AE028464FEA800108444FEA80004FF2BC31C0F20101084482789DF85A
:20CCA00004103046FFF70BFD40B14FF0220405E03846FFF72CFD08B14FF031040BF10100EA
:20CCC0005FFA80FB039800F0FF00834504D2002CAED001E04FF03104204604B0BDE8F08B1F
:20CCE0002DE9304104464FF000014FF0000504F1070000F1020000784FEA002080B20546A2
:20CD000004F1070000F10300007845EA000085B22046FFF71BFF014671BB284640F2022892
:20CD2000B0EB080009D0401E0FD04FF6FD48B0EB080012D0401E18D01EE02046FFF74BFD43
:20CD400001464FF00400A08016E02046FFF790FD01464FF00500A0800EE02046FFF776FEE1
:20CD600001464FF00500A08006E02046FFF7E9FD01464FF00400A0800846BDE8308100B5DD
:20CD800081B0018851B10188012902D100F008F804E00188A1F1010189B2018001B000BD36
:20CDA00000B583B04FF00200FDF72BFF4FF07F008DF805000DF1050000F101004FF031017E
:20CDC00001700DF1050000F102004FF0780101700DF105004FF00301FCF7B5FF03B000BD66
:20CDE00000B581B0018851B10188012902D100F008F804E00188A1F1010189B2018001B0DE
:20CE000000BD00B583B04FF00400FDF7FAFE4FF07F008DF805000DF1050000F101004FF0C2
:20CE2000310101700DF1050000F102004FF0780101700DF105004FF00301FCF784FF03B0C1
:20CE400000BD00B581B0018851B10188012902D100F008F804E00188A1F1010189B2018071
:20CE600001B000BD00B583B04FF00600FDF7C9FE4FF07F008DF805000DF1050000F101001F
:20CE80004FF0310101700DF1050000F102004FF0780101700DF105004FF00301FCF753FF06
:20CEA00003B000BD4DF8048D44F2A678C2F2000888F800005DF8048B70474DF8048D44F2F5
:20CEC000A678C2F2000898F800005DF8048B70474DF8048D44F2A778C2F2000888F80000E6
:20CEE0005DF8048B70474DF8048D44F2A778C2F2000898F800005DF8048B7047F0B581B0AF
:20CF0000069D4FF000044FF000041C604FF000042C600C4613E000F1070606F1020604EB6C
:20CF20000607A1EB04064FEAC6063F7807FA06F71E6846EA07061E60A4F10104E4B2002CF7
:20CF4000E9D801EB0204E4B215E000F1070606F1020604EB060701EB0206A6EB04064FEAD2
:20CF6000C6063F7807FA06F72E6846EA07062E60A4F10104E4B28C42E7D82968186800F011
:20CF8000AAFD01B0F0BD114401F10301884202D04FF0010001E04FF00000704700B581B0A8
:20CFA000FDF70BFB10B14FF0010001E04FF0000001B000BD00B585B003AB009302ABFFF71A
:20CFC0009DFF0346032B02D14FF0010327E0012B0AD10298B0F5503F03D10398B0F5E61F33
:20CFE00002D04FF001031AE053B90298B0F5802F03D10398B0F5C03F02D04FF001030EE012
:20D00000022B0AD10298B0F1005F03D10398B0F5006F02D04FF0010301E04FF00003184655
:20D0200005B000BDF0B587B004464FF000064FF000074FF0000003A8009002AB2046FFF74A
:20D040005DFF05465DB94FF4C0314FF4802000F0CEFD06464FF00000FDF712FB07E0039932
:20D06000029800F0C4FD06462846FDF709FB04F1070000F10300014604A84FF0040201F09A
:20D08000B0FC04F1070000F10700014605A84FF0040201F0A6FC002E57D10298FDF76CFADA
:20D0A000022D08D025B94FF4802000F0EEFF02E0029800F0EAFF039802990844A0F1010062
:20D0C000FDF770FA4FF00100FDF782FAFDF749FAFDF794FA4FF00100FDF7A6FA4FF0000076
:20D0E000FDF7B8FA4FF00000FDF7E0FAE07900F14000C0B2E07104F1070000F101004FF003
:20D100002001017004F1070000F102004FF00801017004F1070000F103004FF00201017032
:20D1200004F1070000F1020000784FEA002004F1070101F10301097841EA000080B2FDF76A
:20D14000CBFA4FF00400A08001E04FF00107384607B0F0BD2DE9F04B84B005464FF001008D
:20D160004FF000044FF000064FF000098DF807904FF000074FF000098DF806904FF0000BD0
:20D18000A888052802D24FF0130493E005F1070000F1010090F800808DF8078005F1070095
:20D1A00000F10200007800F0F0004FEA2010C0B2834605F1070000F10200007800F00F0019
:20D1C000C0B28DF806009DF80780B8F1000F07D19DF80680B8F1040F02D1BBF1040F02D06B
:20D1E0004FF0310466E04FF0000661E030464FEA800108444FEA80004FF21C41C0F2010168
:20D200000844D0F80C80D0F81090CDF80880CDF80C904FF0000741E0029838440078133818
:20D2200008D00F3832D00F380ED0801E16D03D3822D030E05A469DF80610A888FFF7A3FE9B
:20D2400048B34FF0130426E05A469DF806102846FFF7B0FEF8B14FF031041CE04FF21C4163
:20D26000C0F201019DF807004FF00102FDF71FF988B14FF033040EE05A469DF806102846BA
:20D28000FFF7D0FE38B14FF0700404E0FFF786FE08B14FF0220407F10100C7B2039800F0B5
:20D2A000FF00874201D2002CB6D006F10100C6B2002E9BD0204604B0BDE8F08B00B581B0F8
:20D2C0004FF00001FFF746FF0146084601B000BD10B54FF00004FDF770F908B94FF0010466
:20D2E000204610BD4FF00003084402F10101884201D94FF001031846704770B506460D46B8
:20D300004FF00004FDF79BF90146B54203D08D4201D04FF00104204670BD4FF00002A1F1E7
:20D320000201884201D94FF00102104670472DE9F04D82B004468B464FF0FF064FF00007CD
:20D340004FF00000FDF77BF98246FDF762F90546FDF726FD8DF8070004F1070000F1020032
:20D36000A188A1F1020189B20F4604F1070101F101010978514510D14FF00006E07900F1E7
:20D380004000C0B2E07104F1070000F1010080F800A04FF00200A08033E03A4601465846AB
:20D3A00000F07FFC06460EB1782E2AD104F1070000F1010005702846FDF74CF907EB0B004F
:20D3C000FDF71CF9FF2D03D205F10100C5B201E04FF000052846FDF727F99DF80780B8F169
:20D3E000020F06D2782E04D14FF00300FDF709FC07E04FF00200A080E07900F14000C0B24A
:20D40000E071304602B0BDE8F08D2DE9F04B86B007464FF001004FF000044FF000054FF097
:20D42000000607F1070000F1010090F800808DF80780FDF7D8F80390FDF7A9F80290FDF76F
:20D44000E8F88DF80600FDF73CF98346B888032802D24FF0130459E04FF0000554E02846BB
:20D460004FEA800108444FEA80004FF23841C0F201010844D0F80C80D0F81090CDF8108022
:20D48000CDF814904FF0000634E0049830440078133806D011380FD04D3813D0801E1DD006
:20D4A00025E05946B888A0F1020080B2FFF735FFE8B14FF013041AE0FFF70AFFB8B14FF009
:20D4C000240414E0029A0399B888A0F1020080B2FFF708FF58B14FF0710408E09DF80710A5
:20D4E0009DF80600FFF709FF08B14FF0730406F10100C6B2059800F0FF00864201D2002C61
:20D50000C3D005F10100C5B2002DA8D0204606B0BDE8F08B30B581B005464FF00004284617
:20D52000FFF773FF0446FDF75EF824B901462846FFF7FDFE0446204601B030BD00B581B038
:20D54000018851B10188012902D100F008F804E00188A1F1010189B2018001B000BD00B5EA
:20D5600083B04FF00300FDF74CFB4FF07F008DF805000DF1050000F101004FF036010170D7
:20D580000DF1050000F102004FF0780101700DF105004FF00301FCF7D6FB03B000BD30B50D
:20D5A00081B004460D46FDF708F8024605F10100844200D112B94FF0010201E04FF00002A4
:20D5C000104601B030BD884202D04FF0010001E04FF00000704730B581B004460D464FF0B2
:20D5E0000000FCF7F5FF4FF00100FDF75FF84FF00000FDF703F8E07900F14000C0B2E0713E
:20D6000004F1070000F101004FEA252101F0FF01C9B2017004F1070000F1020005F0FF01DC
:20D62000C9B201704FF00300A0804FF0000001B030BD2DE9F04B84B083464FF001004FF0F2
:20D6400000054FF00004FCF7CEFF0190FCF79FFF00904FF000045DE020464FEA8001084424
:20D660004FEA80004FF25041C0F201010844D0F80C80D0F81090CDF80880CDF80C9020464F
:20D680004FEA800108444FEA80004FF25041C0F20101084487884FF000064FF000062FE051
:20D6A00002983044007813381FD0113815D05B3823D1FCF729FF21464FEA810211444FEA29
:20D6C00081014FF25042C0F201021144897801EA000090B94FF07F050FE000990198FFF7DC
:20D6E0005EFF50B14FF0240507E03946BBF80400FFF769FF08B14FF0130506F10100C6B269
:20D70000039800F0FF00864201D2002DC8D004F10100C4B2002C9FD0284604B0BDE8F08BD6
:20D720002DE9704181B00546FCF7E1FF06462846FFF77FFF044644F2EC78C2F2000898F875
:20D740000000012807D14FF0000044F2EC78C2F2000888F80000FCF788FF4FF000024FF0B9
:20D760000101FEF760FF24B931462846FFF733FF0446204601B0BDE870812DE9F04B84B0ED
:20D7800083464FF002004FF000054FF000044FF000000BF1070000F10100007800F07F00DD
:20D7A000C0B207464FF0000410E020464FEA800108444FEA80004FF26841C0F20101084468
:20D7C0000088874204D004F10100C4B2022CECD3022C68D020464FEA800108444FEA800040
:20D7E0004FF26841C0F201010844D0F80C80D0F81090CDF80880CDF80C9020464FEA8001B5
:20D8000008444FEA80004FF26841C0F201010844B0F80480ADF806804FF0000620464FEADE
:20D82000800108444FEA80004FF26841C0F20101084400788DF805004FF000062BE002988C
:20D8400030440078133802D00F380AD020E0BDF80610BBF80400FCF720FEC8B14FF013053B
:20D8600016E09DF80580B84512D1FCF74DFE21464FEA810211444FEA81014FF26842C0F2AA
:20D8800001021144897801EA000008B94FF0220506F10100C6B2039800F0FF00864204D285
:20D8A000002DCCD001E04FF01205284604B0BDE8F08B10B504464FF000002046FFF75DFF20
:20D8C00004F1070101F10101097801F07F01C9B208B9491E491E38B9E17901F14001C9B262
:20D8E000E1714FF00201A18010BD10B44FF0000210E003464FEA03134FF29444C0F2010449
:20D900002344DB68134402EB010424781C7002F10102D2B203464FEA03134FF29444C0F20F
:20D92000010423445B799A42E3D34FF0000010BC70472DE9704191B004460E464FF0000569
:20D9400072B64FF000000CE0694601444FF29448C0F20108D8F80020024412780A7000F17D
:20D9600001004028F0D362B620464FEA00104FF29441C0F2010108440068FAF795FE08B1F9
:20D980004FF001054EBB4FF000021AE020464FEA00104FF29441C0F201010844007910446C
:20D9A0006946014420464FEA00104FF29443C0F201031844C06810440078087002F101003A
:20D9C000C2B220464FEA00104FF29441C0F20101084440798242D9D330E04FF000032BE088
:20D9E0004FF000021AE018464FEA00104FF29441C0F2010108440079104469460144184610
:20DA00004FEA00104FF29446C0F201063044C06810440078087002F10100C2B218464FEA0A
:20DA200000104FF29441C0F20101084440798242D9D303F10100C3B2042BD1D320464FEABB
:20DA400000104FF29441C0F20101084402684FF29440C0F2010000F13000007900F11000D3
:20DA600001466846FAF738FE08B14FF00105284611B0BDE8708170B4042828D04FF000023E
:20DA80001AE002EB010304464FEA04144FF29445C0F20105254404464FEA04144FF294460F
:20DAA000C0F20106344424792D682C44144424781C7002F10102D2B203464FEA03134FF2C0
:20DAC0009444C0F2010423445B799A42D9D34FF0000070BC704770B44FF000024FF0030328
:20DAE0004FF000044FF0000219E014464FEA84052C444FEAC40440F6C065C2F200052C4498
:20DB00006568A84208D301EB0005A5F10105E668B54201D8237804E002F10102D2B2032AA2
:20DB2000E3D3184670BC70472DE9F04107460E464FF0000431463846FFF7CDFF0546B7F515
:20DB4000802F0CD1B6F5C03F09D14FF4E6164FF0010044F2EC78C2F2000888F80000032D30
:20DB600040D028464FEA800108444FEAC00040F6C061C2F20001084490F82400A0B3284663
:20DB80004FEA800108444FEAC00040F6C061C2F200010844006980B128464FEA8001084420
:20DBA0004FEAC00040F6C061C2F2000108440269314638469047044601E04FF072040CB140
:20DBC000782C11D128464FEA800108444FEAC00040F6C061C2F2000108444FF0010180F841
:20DBE000251001E04FF031042046BDE8F08170B505460E464FF0000431462846FFF76BFFD3
:20DC0000024610464FEA800108444FEAC00040F6C061C2F20001084490F8240080B11046DC
:20DC20004FEA800108444FEAC00040F6C061C2F20001084490F8250010B94FF024042EE0A2
:20DC4000032A1DD010464FEA800108444FEAC00040F6C061C2F200010844406980B11046CD
:20DC60004FEA800108444FEAC00040F6C061C2F200010844426931462846904704460EE0AE
:20DC800010464FEA800108444FEAC00040F6C061C2F200010844406908B14FF0720420465A
:20DCA00070BD2DE9704181B004460E4615464FF0000029462046FFF70EFF034644F2EC784C
:20DCC000C2F2000898F80000012807D0B4F5001F04D2B4F5802F01D34FF0010318464FEA54
:20DCE000800108444FEAC00040F6C061C2F20001084490F8240080B118464FEA80010844C5
:20DD00004FEAC00040F6C061C2F20001084490F8250010B94FF0240021E0032B1DD018465F
:20DD20004FEA800108444FEAC00040F6C061C2F200010844C06980B118464FEA80010844CE
:20DD40004FEAC00040F6C061C2F200010844C3692A4631462046984701E04FF0720001B0D7
:20DD6000BDE8708130B44FF0000303461C464FF0000309E0204604F101040D4601F101016A
:20DD80002D78057003F101039342F3D34FF0000030BC704700B583B04FF071018DF80010C6
:20DDA000694601F101014FF001020A70694601F102014FF0FF020A70694601F103014FF0C2
:20DDC00000020A70694601F104014FF000020A7068464FF00501FBF7B6FF4FF00200FCF798
:20DDE0005EFF4FF00000FCF70CFF03B000BD00B581B003464DF69552C0F20102184600F0BD
:20DE00004FF84FF0780001B000BD00B581B000F087F84FF0000001B000BD00B583B0FCF7B9
:20DE2000F8FB014611B94FF0FF0102E0A1F10101C9B24FF076028DF806200DF1060202F153
:20DE4000010211700DF106004FF00201FBF77BFF4FF00300FCF723FF4FF00000FCF7D1FE34
:20DE600003B000BD30B581B00C46154600F00DF94DF61B62C0F201022146284600F083F8C4
:20DE80004FF0780001B030BD00B581B0FAF786FC10B14FF0000001E04FF0010001B000BD45
:20DEA0002DE9704181B004460D46164605EB0400A04202D24FF0FF002FE000F04CFC10B181
:20DEC0004FF0FF0029E0C4F30C0080B1C4F30C0240F63871C2F2000188681044886040F64C
:20DEE0003871C2F2000148686FF30C00486040F63878C2F20008C8F8044040F63878C2F2BE
:20DF00000008C8F8085040F63878C2F20008C8F80C6000F008FC4FF0000001B0BDE8708199
:20DF20002DE9304104460D464FF0000040F63878C2F2000888F8000005EB0400A04202D2B2
:20DF40004FF0FF001DE029462046FFF79DFF10B14FF0FF0015E04FF0010040F63878C2F251
:20DF6000000888F8000040F63878C2F20008C8F8044040F63878C2F20008C8F808504FF07A
:20DF80000000BDE830812DE9304104464FF0000040F63878C2F2000898F80030012B30D18C
:20DFA00040F63878C2F20008D8F80830002B28D940F63878C2F20008D8F80800844205D96D
:20DFC00040F63878C2F20008D8F8084013460A46214640F63878C2F20008D8F8040000F011
:20DFE0005FF870B940F63875C2F20005AB68A3EB0403AB6040F63875C2F200056B6823447C
:20E000006B60BDE8308100004DF8048D4FF0000045F2F478C2F2000898F808180A4602F178
:20E02000010202F0010240F6044303FB02F244F2F473C2F200031A4492F8022C02BB01F160
:20E04000010101F00101C9B245F2F478C2F2000888F8081845F2F478C2F2000898F8081842
:20E0600040F6044211FB02F144F2F472C2F2000211444FF0000201F54068A8F8002001E0FE
:20E080004FF0FF005DF8048B70474DF8048D45F2F478C2F20008C8F80C085DF8048B704703
:20E0A0002DE9F0410C461F464FF0000145F2F478C2F2000898F8083845F2F478C2F2000894
:20E0C00098F8083840F6044513FB05F344F2F475C2F200052B4493F8023CABB945F2F47854
:20E0E000C2F2000898F8083840F6044513FB05F344F2F475C2F200052B444FF0000503F50C
:20E100004068A8F8005014E045F2F478C2F2000898F8083840F6044513FB05F344F2F47520
:20E12000C2F200052B4493F8023C012B01D04FF0FF01002940F0828016464FF0000571E066
:20E1400045F2F478C2F2000898F8082840F6044312FB03F244F2F473C2F200031A4402F578
:20E160004068B8F80020B2F5006F02D3FFF74CFF0146002958D145F2F478C2F2000898F873
:20E18000082840F6044312FB03F244F2F473C2F200031A4402F54068B8F8003045F2F478FC
:20E1A000C2F2000898F8082840F6044C12FB0CF244F2F47CC2F2000C62441A4405EB0603EF
:20E1C0001B78137045F2F478C2F2000898F8082840F6044312FB03F244F2F473C2F2000337
:20E1E0001A444FF0010382F8023C45F2F478C2F2000898F8082840F6044312FB03F244F2F2
:20E20000F473C2F20003134403F54068B8F8002002F1010292B203F54068A8F8002005F189
:20E22000010295B2A5428BD341B945F2F478C2F20008C8F8107800F009F901460846BDE882
:20E24000F08100002DE930414FF0000444F2F078C2F2000898F80000052800F2ED800FF20C
:20E260000808D8E800F000BFF104316F8BC84FF0000045F2F478C2F2000888F8090845F2D1
:20E28000F478C2F2000898F8090840F6044110FB01F044F2F471C2F20001084490F8020C0C
:20E2A000022808D14FF0020044F2F078C2F2000888F80000C8E04FF0040044F2F078C2F203
:20E2C000000888F80000BFE045F2F478C2F2000898F8090840F6044110FB01F044F2F47105
:20E2E000C2F200010844054621E000F01AFB45F2F478C2F20008D8F80C2828464FF4007147
:20E30000FAF7EAF944F2F471C2F2000141F60C088844D8F8000000F5007041F60C08884476
:20E32000C8F8000004F10100C4B205F50075042CDBD34FF0030044F2F078C2F2000888F848
:20E34000000081E045F2F478C2F2000898F8090840F6044110FB01F044F2F471C2F2000195
:20E3600008444FF0000180F8021C4FF0040044F2F078C2F2000888F8000065E045F2F47876
:20E38000C2F2000898F8090860BB4FF0010045F2F478C2F2000888F8090845F2F478C2F27E
:20E3A000000898F8090840F6044110FB01F044F2F471C2F20001084490F8020C022808D108
:20E3C0004FF0020044F2F078C2F2000888F800003AE04FF0050044F2F078C2F2000888F8EA
:20E3E000000031E04FF0050044F2F078C2F2000888F8000028E04FF0000044F2F078C2F255
:20E40000000888F8000045F2F478C2F20008D8F81008C8B145F2F478C2F20008D8F810185D
:20E420004FF0000088474FF0000045F2F478C2F20008C8F8100807E04FF0000044F2F07894
:20E44000C2F2000888F80000BDE830812DE930414FF000044FF000054FF0000042E040F685
:20E46000044110FB01F144F2F472C2F20002114491F8021C012932D140F6044110FB01F167
:20E4800044F2F472C2F20002114401F54068B8F80010B1F5007F22D340F6044110FB01F1E5
:20E4A00044F2F472C2F2000211444FF0020281F8022C4FF0FF0545F2F478C2F2000898F899
:20E4C0000818884202D1FFF79FFD04464FF0010044F2F078C2F2000888F8000004E000F1B4
:20E4E0000100C0B20228BAD3BDB945F2F478C2F20008D8F8100880B145F2F478C2F20008A5
:20E50000D8F810184FF0000088474FF0000045F2F478C2F20008C8F810082046BDE83081C3
:20E520004FF0010070472DE9004146F20808C2F2000898F80000072800F2EB800FF2040860
:20E54000D8E800F004153E617491C5DE4FF0000046F20808C2F2000888F800004FF00000A9
:20E5600046F20A08C2F20008A8F80000D9E040F63878C2F20008D8F8040046F21008C2F2C2
:20E580000008C8F8000040F63878C2F20008D8F8080046F20C08C2F20008C8F800004FF032
:20E5A000000046F20A08C2F20008A8F800004FF0020046F20808C2F2000888F80000B0E060
:20E5C00046F20A08C2F20008B8F80000022811D246F20A01C2F20001088800F1010080B2CC
:20E5E00008804FF0020046F20808C2F2000888F8000096E04FF0030046F20808C2F2000812
:20E6000088F800008DE000F08CF946F21008C2F20008D8F80000FAF747F84FF0040046F211
:20E620000808C2F2000888F800007AE0FFF778FF80B146F21001C2F20001086800F50050E3
:20E6400008604FF0050046F20808C2F2000888F8000066E04FF0040046F20808C2F20008FD
:20E6600088F800005DE046F20C08C2F20008D8F80000B0F5005F08D24FF0000046F20C089C
:20E68000C2F20008C8F8000007E046F20C01C2F200010868A0F50050086046F20C08C2F260
:20E6A0000008D8F80000002808D94FF0030046F20808C2F2000888F8000032E04FF006005C
:20E6C00046F20808C2F2000888F8000029E04FF0000046F20808C2F2000888F8000040F6B4
:20E6E0003878C2F20008D8F80C00D0B140F63878C2F20008D8F80C104FF00000884710E0C5
:20E700004FF0000046F20808C2F2000888F8000007E04FF0000046F20808C2F2000888F88C
:20E720000000BDE800814DF8048D4FF0FF0046F20808C2F2000898F8001049B94FF00100B9
:20E7400046F20808C2F2000888F800004FF000005DF8048B70474DF8048D46F20808C2F289
:20E76000000898F800005DF8048B704710B582B04FF00000ADF806004FF0000422E00DF142
:20E78000060320464FEA400040F64871C2F20001084400F1010220464FEA400040F64871DF
:20E7A000C2F20001084401464FF0010000F042F84FF47A7040F69371C2F20001884704F1C7
:20E7C0000100C4B2032CDAD302B010BD11B94FEA6000C0B200F080014FEAE11100F04002C4
:20E7E0004FEA621242EA010100F020024FEAE20242EA010100F010024FEA620242EA010114
:20E8000000F008024FEA420242EA010100F004024FEAC20242EA010100F002024FEA4212B1
:20E8200042EA010100F001004FEAC01040EA0100C0B2704770B51E464FF000054FF000044C
:20E84000E8BB08784FEA402080B2044604F47F404FEA2020C0B24FF00001FFF7B7FF4FEAB9
:20E86000002004F0FF0141EA000080B2044621464FF00000F8F70BFC4FF001014FF00000C1
:20E88000F8F71DFC0028F7D04FF003014FF00000F8F715FC0028F7D04FF00000F8F703FCE3
:20E8A000044604F0FF00C0B24FF00101FFF78EFF04F47F4141EA0004A0B230802FE008786D
:20E8C0004FEA402080B240F48070117841EA000080B2044604F47F404FEA2020C0B24FF038
:20E8E0000001FFF773FF4FEA002604F0FF00C0B24FF00101FFF76AFF40EA060040F48070F7
:20E9000080B2044621464FF00000F8F7C0FB4FF001014FF00000F8F7D2FB0028F7D0284692
:20E9200070BD10B582B04FF00000ADF806004FF0000426E020464FEA400040F64871C2F2FE
:20E94000000108440078032818D10DF1060320464FEA400040F64871C2F20001084400F117
:20E96000010220464FEA400040F64871C2F20001084401464FF00100FFF75CFF04F10100F7
:20E98000C4B2032CD6D302B010BD000000F020E300F020E31EFF2FE100BF7047016844F67E
:20E9A0006D62C4F2C612514343F23902C0F2000289180160C1F30E40704720B500F0EFF8DB
:20E9C00040F68C70C2F20000FFF7E8FF054600F0E7F8284620BD40F68C71C2F200010860BF
:20E9E0007047E1B5121F45DB4FF00305054012D0C5F10405022D11F8013B00F8013B08DBC1
:20EA000011F8013B00F8013B03DD11F8013B00F8013B521B2EDB4FF003050D403DD1083ACA
:20EA20001CDB143A11DBB1E86840A0E86840B1E86840A0E86840203AF5DA12F1100FA2BF17
:20EA4000B1E86840A0E86840103A1432A1BFB1E82840A0E82840B2F10C02F7E7083209DBB7
:20EA6000121FB9BF51F8043B40F8043B28C928C0A8BF121F121D00F08F80022A11F8013BDE
:20EA800000F8013BA4BF11F8013B00F8013BC4BF11F8013B00F8013B7EE021F0030151F8AE
:20EAA00004EB022D28DC4FD00C2A18DBA2F10C024FEA1E23B1E8E04043EA05634FEA152510
:20EAC00045EA06654FEA162646EA07664FEA172747EA0E67E8C0103AEADA0C3209DB4FEA5C
:20EAE0001E2551F804EB45EA0E6540F8045B121FF5DAA1F10301BDE70C2A18DBA2F10C025E
:20EB00004FEA1E63B1E8E04043EA05234FEA156545EA06254FEA166646EA07264FEA176757
:20EB200047EA0E27E8C0103AEADA0C3209DB4FEA1E6551F804EB45EA0E2540F8045B121F79
:20EB4000F5DAA1F1010195E70C2A18DBA2F10C024FEA1E43B1E8E04043EA05434FEA1545B1
:20EB600045EA06454FEA164646EA07464FEA174747EA0E47E8C0103AEADA0C3209DB4FEADB
:20EB80001E4551F804EB45EA0E4540F8045B121FF5DAA1F102016DE7BDE8E14070477047A4
:20EBA000704700000040024000500240008003400090034000400440005004400060054037
:20EBC000007005400040024000500240008003400090034000400440005004400060054019
:20EBE0000070054000800000004000000008000000040000000000400000008000000004D0
:20EC0000200000004000000080000000000008000000040000000100000001000000020004
:20EC2000040000000200000000000200000001000000080000001000010000002000000092
:20EC40004000000080000000000008000000040000000100000001000000020000000000E4
:20EC600001000000020000000300000000000200000001000000030000E003400020044001
:20EC80000030044000E00340002004400030044001000000020000000400000008000000F6
:20ECA000100000002000000040000000800000000001000000020000000400000008000055
:20ECC000001000000020000000400000008000000D00000007000000060000000500000025
:20ECE000040000000300000001000000000000000F00000000000F000000000F00000F0FC1
:20ED00008080008080808000808000000000400000000040000040400100000002000000F0
:20ED200004000000080000001000000020000000400000007F0000000100000002000000D5
:20ED40000400000008000000100000002000000040000000800000000001000000020000B4
:20ED6000000400000008000000100000002000000040000000800000000001000000020094
:20ED8000000004000000080000001000000020000000400000008000000000010000000274
:20EDA000000000040000000800000010000000200000004000000080FFFFFFFF100000004B
:20EDC0001000000000000001000000010090044000A0044000B004400000054000100540DB
:20EDE0000090044000A0044000B00440000005400010054000F00F4040F00F4080F00F4050
:20EE0000C0F00F4000F10F4000F00F4040F00F4080F00F40C0F00F4000F10F4001000000F6
:20EE20000200000004000000080000001000000020000000000040000000800000000001D3
:20EE400000000002000000040000000800000040000000803F00C0CF0060064000800540AB
:20EE6000006006400080054000000000010000000200000003000000040000000500000018
:20EE8000160000001700000018000000190000001A0000001B0000001E0000001F000000A2
:20EEA00010000000200000004000000080000000F0000000004005400050054000400540D3
:20EEC00000500540010000000200000004000000080000000F00000000E0004000A001407E
:20EEE00000E0004000A00140010000000200000004000000080000001000000020000000D2
:20EF00004000000080000000000100000002000000040000000800000010000000200000F2
:20EF2000004000000080000030000000FFFF00004000000080000000C00000002000000043
:20EF400004000000240000008000000000010000000800000020000080290000080000002F
:20EF60001000000020000000400000003800000000000100000000010000000200000004E1
:20EF80000000000800000010000000200080013F0000010000000001000000020000000471
:20EFA0000000000800000010000000200080013F010000000200000004000000080000004A
:20EFC000100000002000000040000000800000000001000000020000000400000008000032
:20EFE0000010000000200000004000000080000000000100FFFF010001000000020000001E
:20F00000040000000700000000C0024000D00240000003400010034000C0024000D0024027
:20F02000000003400010034001000000020000000400000008000000100000001F000000FC
:20F04000040000002000000040000000000200000004000000100000002000000080000096
:20F0600064B6000004000000200000004000000000020000000400000010000000200000DC
:20F0800000800000E4B6000001000000020000000400000008000000100000002000000017
:20F0A000000100003F01000000F0004000B0014000F0004000B0014000C0004000D00040BD
:20F0C000008001400090014000C0004000D0004000800140009001400100000002000000F9
:20F0E000040000000800000010000000200000004000000080000000000100000002000011
:20F1000010000000FF030000010000000200000004000000080000000F00000000000004BB
:20F1200000000004100000001000000000000000006A180000000000000000000100000028
:20F14000100000000100000020000000010000000100000000000020000800000E00000046
:20F1600000000000080000000400000003000000020000000300000000000000000000007B
:20F18000020000000300000002000000010000000100000000000000211000000000000035
:20F1A0000000000000000000080C101418203040000000000000000000000000000000006F
:20F1C000000000000000000084F102010A0003002FB00100DCF1010004000000311333225F
:20F1E000000007000200020000000000F4F1010002000000131200000100070002000600E7
:20F200000000000034F201000100000002000600020006000000000035F20100020000008C
:20F2200003000500020006000000000037F201000200000013137E137E0000000300070053
:20F24000020002000000000050F2010004000000131222338AF1070003000A00E5B80100BC
:20F260001CF301000300000089F00700030012001DB901001FF301000300000089F1070078
:20F280000300120055B9010022F301000300000087F107000300180087B9010025F301003D
:20F2A0000300000088F1070003001700BFB9010028F301000300000070F1070003000700A7
:20F2C000C3BA01002BF301000300000071F1070003000700F1B901002EF30100030000004B
:20F2E00010F0070003001B004DBA010031F301000300000084F1070003000A0085BA0100F0
:20F3000034F301000300000086F1070003000400A7BA010037F30100030000001322311334
:20F320002231132231132231132231132231132231132231132231132231503032373638F3
:20F340003739204141000000010000000000000001000200020006000000000078F3010023
:20F36000030000000200020006000200000000007BF3010003000000132237132224000047
:20F38000000004000300020000000000A8F3010002000000010004000300020000000000BC
:20F3A000AAF301000200000013221322FF000000000000000000000000000000020202013D
:20F3C00006000400000000000CF401000400000003020600040004000000000010F4010006
:20F3E0000400000000FF02010C0004000000000014F401000500000001FF020104000400DE
:20F400000000000019F40100030000003312132233121322331213312233121300000201E1
:20F420000B0004000000000030F4010005000000133133227000000000000201020801007C
:20F44000000000004CF40100040000001324717300000201010001000000000064F40100EE
:20F46000020000002413000001000400050002000000000090F401000200000002000400BA
:20F48000050002000000000092F4010002000000132213220080010100080000A20E002018
:20F4A000AC4700200080010110080000AA0E0020BC47002000800101200C0000B20E002016
:20F4C000CC4700200080010130040000A8470020DC470020E80300000050064004500640D6
:20F4E000085006400C5006401050064014500640185006401C5006402050064024500640AC
:20F50000285006402C5006403050064034500640385006403C50064040500640445006408B
:20F52000485006404C5006405050064054500640585006405C50064060500640645006406B
:20F54000685006406C5006407050064074500640785006407C50064080500640845006404B
:20F56000885006408C5006409050064094500640985006409C500640A0500640A45006402B
:20F58000A8500640AC500640B0500640B4500640B8500640BC500640C0500640C45006400B
:20F5A000C8500640CC500640D05006403FFFFFFF0050064004500640085006400C50064079
:20F5C0001050064014500640185006401C5006402050064024500640285006402C5006408B
:20F5E0003050064034500640385006403C5006404050064044500640485006404C5006406B
:20F600005050064054500640585006405C5006406050064064500640685006406C5006404A
:20F620007050064074500640785006407C5006408050064084500640885006408C5006402A
:20F640009050064094500640985006409C500640A0500640A4500640A8500640AC5006400A
:20F66000B0500640B4500640B8500640BC500640C0500640C4500640C8500640CC500640EA
:20F68000D0500640020600003000000001010000010400005000000001010000000102036D
:20F6A0000405060708090A0B0C0D0E0F101112131415161718191A1B1C1D1E1F20212223DA
:20F6C0002425262728292A2B2C2D2E2F303132333435363738393A3B3C3D3E3F40414243BA
:20F6E0004445464748494A4B4C4D4E4F505152535455565758595A5B5C5D5E5F606162639A
:20F700006465666768696A6B6C6D6E6F707172737475767778797A7B7C7D7E7F8081828379
:20F720008485868788898A8B8C8D8E8F909192939495969798999A9B9C9D9E9FA0A1A2A359
:20F74000A4A5A6A7A8A9AAABACADAEAFB0B1B2B3B4B5B6B7B8B9BABBBCBDBEBFC0C1C2C339
:20F76000C4C5C6C7C8C9CACBCCCDCECFD0D1D2D3D4D5D6D7D8D9DADBDCDDDEDFE0E1E2E319
:20F78000E4E5E6E7E8E9EAEBECEDEEEFF0F1F2F3F4F5F6F7F8F9FAFBFCFDFEFFE0A618243D
:20F7A000000C342C4C8008385144603E21BC549140638B574F3E4C853B928C8D0E4D5C3A22
:20F7C0009B1439AC359F1112132232425283232756987F7D938161507C900D0B48593F6FB4
:20F7E0008A8F7E9E1E0E5BFFF8AFBF1FDED8D0C3B9C8A8B0B1CDFC25747B7A9C68CFFE25A9
:20F80000359F1112131EC8DBC3B6C9AAB0BDCFFC28787D7C100002000100000001A30100A8
:20F8200011000200010000003DA30100220003000000000079A30100280003000100000065
:20F84000ABA301003E00020001000000E7A30100850002000100000023A40100010000003C
:20F86000040002000200000077A001000200000004000200020000008DA001000000000030
:20F880000400030005000000ED9F010003000000040003000500000021A0010001000000FD
:20F8A0000700020002000000AD9D0100020000000600020002000000139E01000300000031
:20F8C0000500020002000000759E01008AF100000200030003000000FD9E010089F0000073
:20F8E0000700030003000000259F010089F1000007000300030000004D9F010087F100004A
:20F900000700030003000000759F010088F1000007000300030000009D9F010070F10000A1
:20F920000700030003000000C59F0100010000000600020002000000D79E010000000000D4
:20F94000070002000200000055A00100010303001000020001000000C7B2010011000200FF
:20F960000100000071B50100220003000000000033B8010027000200000000008DC00100D7
:20F980002800030001000000B3C501002E000300000000007DAF010031000400000000002F
:20F9A000E1CC01003400010000000000BDD20100360002000000000015D501003700010079
:20F9C0000000000021D701003E0002000100000075B101008500050001000000B3D80100AF
:20F9E000A72364AA00000001000022222222FFFFFFFF0000FFFF0000FFFFFFFFFFFFFFFFB4
:20FA0000FFFFFFFFFFFF0000000000000000040000800100FF7F0500EFDD01000BDE01002D
:20FA20000000000065DE01000000000001000000010000000040030000C01C00FFFF1F0044
:20FA4000EFDD01000BDE01000000000065DE01000000000001000000020000000000002088
:20FA600000080000FF07002000000000000000000000000065DD0100000000000000000015
:20FA800000000000000005000000080000000000040302040317C021204128C12061010085
:20FAA0000200030004000600070008000B000C000E000F00170018001C001D001E001F004F
:20FAC0004000410042004300440046004800540055007E000100000001004FF000010A4695
:14FAE00001F101018242FAD370470000000000BF000000BF58
:020000040002F8
:203FE0005830315F414E3031325F535746425F423030312E533130312E30302E2E2E2E2E3D
:04000005000103747F
:00000001FF
